:020000040806ec
:10000000000006088a0c150800008c13200004016b
:100010000200d10700000000005000102100060877
:100020000d490e4a0e4b9b1a03dd043bc858d050b5
:10003000fbdc0b490b4a0020521a02dd043a8850bf
:10004000fcdc0949094a0a4b9b1a03dd043bc858ea
:10005000d050fbdc074880476098140820510010fe
:10006000e0c3001038c10110800006080000000243
:10007000e0970e02710000028809fa790100000081
:1000800038dc0c02a8640c0204650c020ce10c02c2
:10009000e0df0c0238df0c0234e20c0278de0c02e6
:1000a000d8e10c0294e20c0234660c02e4650c0206
:1000b000e4dd0c02dce20c02c0e10c02dcdd0c022f
:1000c00028df0c0284930c0288660c02c4e00c0248
:1000d000f4e00c0240e00c02a4e10c023ce30c0250
:1000e000a8dc0c0234e10c0284e20c02ffffffffeb
:1000f00046f0c0fb1af0d4fd1df046fe1af05afe81
:1001000081f0004102e000bf83f0004330b54feac8
:1001100041044fea430594ea050f08bf90ea020f35
:100120001fbf54ea000c55ea020c7fea645c7feac8
:10013000655c00f0e2804fea5454d4eb5555b8bfeb
:100140006d420cdd2c4480ea020281ea030382ea5c
:10015000000083ea010180ea020281ea0303362dee
:1001600088bf30bd11f0004f4fea01314ff4801cc1
:100170004cea113102d0404261eb410113f0004fd3
:100180004fea03334cea133302d0524263eb43038a
:1001900094ea050f00f0a780a4f10104d5f1200e28
:1001a0000ddb02fa0efc22fa05f2801841f1000183
:1001b00003fa0ef2801843fa05f359410ee0a5f157
:1001c00020050ef1200e012a03fa0efc28bf4cf088
:1001d000020c43fa05f3c01851ebe37101f000453e
:1001e00007d54ff0000edcf1000c7eeb00006eeb4b
:1001f0000101b1f5801f1bd3b1f5001f0cd34908d5
:100200005fea30004fea3c0c04f101044fea44522b
:1002100012f5800f80f09a80bcf1004f08bf5feab2
:10022000500c50f1000041eb045141ea050130bd92
:100230005fea4c0c404141eb0101013c28bfb1f5a4
:10024000801fe9d291f0000f04bf01460020b1faef
:1002500081f308bf2033a3f10b03b3f120020cdac2
:100260000c3208dd02f1140cc2f10c0201fa0cf0a0
:1002700021fa02f10ce002f11402d8bfc2f1200c05
:1002800001fa02f120fa0cfcdcbf41ea0c019040bb
:10029000e41aa2bf01eb0451294330bd6fea040404
:1002a0001f3c1cda0c340edc04f11404c4f12002ef
:1002b00020fa04f001fa02f340ea030021fa04f301
:1002c00045ea030130bdc4f10c04c4f1200220fa58
:1002d00002f001fa04f340ea0300294630bd21fa96
:1002e00004f0294630bd94f0000f83f4801306bf5c
:1002f00081f480110134013d4ee77fea645c18bf50
:100300007fea655c29d094ea050f08bf90ea020fe6
:1003100005d054ea000c04bf1946104630bd91eade
:10032000030f1ebf0021002030bd5fea545c05d1e1
:100330004000494128bf41f0004130bd14f5800420
:100340003cbf01f5801130bd01f0004545f0fe4194
:1003500041f470014ff0000030bd7fea645c1abfc9
:10036000194610467fea655c1cbf0b46024650ea00
:10037000013406bf52ea033591ea030f41f400212c
:1003800030bd00bf90f0000f04bf0021704730b5b2
:100390004ff4806404f132044ff000054ff0000187
:1003a00050e700bf90f0000f04bf0021704730b548
:1003b0004ff4806404f1320410f0004548bf40421d
:1003c0004ff000013ee700bf42004feae2014fea72
:1003d00031014fea02701fbf12f07f4393f07f4f4d
:1003e00081f06051704732f07f4208bf704793f050
:1003f0007f4f04bf41f40021704730b54ff4607463
:1004000001f0004521f000411ce700bf50ea010265
:1004100008bf704730b54ff000050ae050ea01020e
:1004200008bf704730b511f0004502d5404261eb7e
:1004300041014ff4806404f132045fea915c3ff4bf
:10044000d8ae4ff003025feadc0c18bf03325fea5c
:10045000dc0c18bf033202ebdc02c2f1200300fa0d
:1004600003fc20fa02f001fa03fe40ea0e0021fa32
:1004700002f11444bde600bf70b54ff0ff0c4cf420
:10048000e06c1cea11541dbf1cea135594ea0c0fd2
:1004900095ea0c0f00f0def82c4481ea030621ea0d
:1004a0004c5123ea4c5350ea013518bf52ea033548
:1004b00041f4801143f4801338d0a0fb02ce4ff0fa
:1004c0000005e1fb02e506f00042e0fb03e54ff02a
:1004d0000006e1fb03569cf0000f18bf4ef0010e22
:1004e000a4f1ff04b6f5007f64f5407404d25fea1e
:1004f0004e0e6d4146eb060642eac62141ea5551d1
:100500004feac52040ea5e504feace2eb4f1fd0c12
:1005100088bfbcf5e06f1ed8bef1004f08bf5fea90
:10052000500e50f1000041eb045170bd06f0004642
:1005300046ea010140ea020081ea0301b4eb5c04ef
:10054000c2bfd4eb0c0541ea045170bd41f48011e7
:100550004ff0000e013c00f3ab8014f1360fdebf0c
:10056000002001f0004170bdc4f10004203c35dae8
:100570000c341bdc04f11404c4f1200500fa05f36b
:1005800020fa04f001fa05f240ea020001f000420c
:1005900021f0004110ebd37021fa04f642eb060182
:1005a0005eea430e08bf20ead37070bdc4f10c04ac
:1005b000c4f1200500fa04f320fa05f001fa04f270
:1005c00040ea020001f0004110ebd37041f100015c
:1005d0005eea430e08bf20ead37070bdc4f1200567
:1005e00000fa05f24eea020e20fa04f301fa05f2cf
:1005f00043ea020321fa04f001f0004121fa04f277
:1006000020ea020000ebd3705eea430e08bf20ea46
:10061000d37070bd94f0000f0fd101f00046400080
:1006200041eb010111f4801f08bf013cf7d041ea02
:10063000060195f0000f18bf704703f00046520006
:1006400043eb030313f4801f08bf013df7d043ead7
:100650000603704794ea0c0f0cea135518bf95ea8d
:100660000c0f0cd050ea410618bf52ea4306d1d114
:1006700081ea030101f000414ff0000070bd50ea33
:10068000410606bf1046194652ea430619d094eabd
:100690000c0f02d150ea013613d195ea0c0f05d1a7
:1006a00052ea03361cbf104619460ad181ea0301fb
:1006b00001f0004141f0fe4141f470014ff00000b3
:1006c00070bd41f0fe4141f4780170bd70b54ff04e
:1006d000ff0c4cf4e06c1cea11541dbf1cea1355ce
:1006e00094ea0c0f95ea0c0f00f0a7f8a4eb0504b0
:1006f00081ea030e52ea03354fea013100f08880a7
:100700004fea03334ff0805545ea131343ea12636f
:100710004fea022245ea111545ea10654fea002624
:100720000ef000419d4208bf964244f1fd0404f5dd
:10073000407402d25b084fea3202b61a65eb030539
:100740005b084fea32024ff480104ff4002cb6ebf6
:10075000020e75eb030e22bfb61a754640ea0c0076
:100760005b084fea3202b6eb020e75eb030e22bfb6
:10077000b61a754640ea5c005b084fea3202b6ebf7
:10078000020e75eb030e22bfb61a754640ea9c00b6
:100790005b084fea3202b6eb020e75eb030e22bf86
:1007a000b61a754640eadc0055ea060e18d04fea44
:1007b000051545ea16754fea06164feac30343eae4
:1007c00052734feac2025fea1c1cc0d111f4801fb1
:1007d0000bd141ea00014ff000004ff0004cb6e7aa
:1007e00011f4801f04bf01430020b4f1fd0c88bf49
:1007f000bcf5e06f3ff6afaeb5eb030c04bfb6eb54
:10080000020c5fea500c50f1000041eb045170bd46
:100810000ef0004e4eea113114eb5c04c2bfd4eb73
:100820000c0541ea045170bd41f480114ff0000ef7
:10083000013c90e645ea060e8de60cea135594ea73
:100840000c0f08bf95ea0c0f3ff43baf94ea0c0f76
:100850000ad150ea01347ff434af95ea0c0f7ff4eb
:1008600025af104619462ce795ea0c0f06d152ea3f
:1008700003353ff4fdae1046194622e750ea410623
:1008800018bf52ea43067ff4c5ae50ea41047ff434
:100890000daf52ea43057ff4ebae12e74ff0ff3c99
:1008a00006e000bf4ff0010c02e000bf4ff0010c6a
:1008b0004df804cd4fea410c7fea6c5c4fea430ce3
:1008c00018bf7fea6c5c1bd001b050ea410c0cbf32
:1008d00052ea430c91ea030f02bf90ea020f002094
:1008e000704710f1000f91ea030f58bf994208bffb
:1008f00090422cbfd8176feae37040f001007047b8
:100900004fea410c7fea6c5c02d150ea013c07d10e
:100910004fea430c7fea6c5cd6d152ea033cd3d059
:100920005df8040b704700bf8446104662468c4653
:100930001946634600e000bf01b5fff7b7ff002886
:1009400048bf10f1000f01bd4df808edfff7f4ffaf
:100950000cbf012000205df808fb00bf4df808ed3a
:10096000fff7eaff34bf012000205df808fb00bf5d
:100970004df808edfff7e0ff94bf012000205df87f
:1009800008fb00bf4df808edfff7ceff94bf012034
:1009900000205df808fb00bf4df808edfff7c4ff2d
:1009a00034bf012000205df808fb00bf4fea410c76
:1009b0007fea6c5c02d150ea013c0ad14fea430c59
:1009c0007fea6c5c02d152ea033c02d14ff0000096
:1009d00070474ff0010070474fea410212f50012d4
:1009e00015d211d56ff47873b3eb625212d94fea76
:1009f000c12343f0004343ea505311f0004f23fa60
:100a000002f018bf404270474ff00000704750eab4
:100a1000013005d111f0004008bf6ff00040704771
:100a20004ff00000704700bf53b94ab9002908bf12
:100a300000281cbf4ff0ff314ff0ff3000f096b997
:100a4000adf1080c6de904ce00f01af8ddf804e011
:100a5000dde9022304b07047430803f05533c01aa0
:100a6000830800f0333003f03333184400eb1010e8
:100a700000f00f3000eb002000eb0040000e70474c
:100a80002de9f04f099d04460f46002b48d18a42bc
:100a9000944661d9b2fa82f343b1c3f120019f4079
:100aa00002fa03fc9c4020fa01f10f434fea1c417b
:100ab0001ffa8cfe220cb7fbf1f601fb167706fb42
:100ac0000ef042ea0742904208d91ceb020206f1fe
:100ad000ff3702d2904200f237813e46121aa4b28a
:100ae000b2fbf1f001fb102200fb0efe44ea0244cf
:100af000a64508d91ceb040400f1ff3202d2a6453a
:100b000000f21c81104640ea0640a4eb0e040026c9
:100b10001db1dc400023c5e900433146bde8f08f3c
:100b20008b4209d9002d00f0fd800026c5e90001a7
:100b300030463146bde8f08fb3fa83f6002e4bd134
:100b40008b42c0f0f280824240f2ef803046002dae
:100b5000e3d0c5e90047e0e702b9ffdeb2fa82f36d
:100b6000002b40f09d80891a4fea124e97b2012661
:100b7000200cb1fbfef20efb121140ea014107fb13
:100b800002f088420fd91ceb010102f1ff382cbfa3
:100b90004ff001094ff00009884203d9b9f1000f65
:100ba00000f0cf804246091aa4b2b1fbfef00efb62
:100bb000101100fb07f744ea0144a74208d91cebd7
:100bc000040400f1ff3102d2a74200f2b4800846cb
:100bd000e41b40ea02409be7c6f12007b34001fa5c
:100be00006f422fa07fcf940b2404cea030c20fa62
:100bf00007f34fea1c491c431ffa8cfe00fa06f368
:100c0000200cb1fbf9f809fb181140ea014108fb7f
:100c10000ef088420fd91ceb010108f1ff3a2cbffe
:100c20004ff0010b4ff0000b884203d9bbf1000fce
:100c300000f08d80d046091aa4b2b1fbf9f009fb8f
:100c4000101100fb0efe44ea01418e4507d91ceb52
:100c5000010100f1ff3401d28e457fd8204640eae1
:100c60000840a1eb0e01a0fb029841454c46c64648
:100c700002d306d14b4504d20138b9eb020468eb2c
:100c80000c0e002d70d01a1b61eb0e0122fa06f338
:100c900001fa07f7f14000261f43c5e900713ce760
:100ca00002fa03fcc3f1200001fa03f221fa00f674
:100cb0004fea1c4e24fa00f11ffa8cf79c401143b6
:100cc000b6fbfef00a0c0efb106642ea064200fb81
:100cd00007f696420ed91ceb020200f1ff382cbf3a
:100ce0004ff001094ff00009964202d9b9f1000f07
:100cf00031d04046921b89b2b2fbfef60efb1622a3
:100d000041ea024106fb07f28a4207d91ceb0101c6
:100d100006f1ff3801d28a4223d84646891a46eaac
:100d2000004625e72e462846f7e6841a61eb0303c2
:100d300001201f460be76444023849e76444023847
:100d4000e1e6023a61442ee7023e6244c6e6a8f1bb
:100d5000020861446fe702386244cbe7023861441d
:100d60007de7023e6144d9e72e46d6e6704700bfd4
:100d700010f8012b11f8013b012a28bf9a42f7d045
:100d8000d01a7047034613f8012b002afbd1181a1a
:100d9000013870477bb972b90029bebf00204ff0ff
:100da000004106e008bf00281cbf6ff000414ff073
:100db000ff30fff7dbbfadf1080c6de904ce002971
:100dc00009db002b1adbfff75bfeddf804e0dde951
:100dd000022304b07047404261eb4101002b1bdb52
:100de000fff74efeddf804e0dde9022304b04042e7
:100df00061eb4101524263eb43037047524263eba4
:100e00004303fff73dfeddf804e0dde9022304b013
:100e1000404261eb41017047524263eb4303fff7ed
:100e20002ffeddf804e0dde9022304b0524263eb5b
:100e30004303704709b504480068044b03441b682a
:100e40001b68029309bd000014ca001004000000d2
:100e500009b504480068044b03441b685b680293af
:100e600009bd000014ca00100400000009b50448c0
:100e70000068044b03441b689b68029309bd000093
:100e800014ca00100400000000b1807b704708b154
:100e9000c07b7047ff20704708b1408970474ff60c
:100ea000ff70704708b1808970474ff6ff70704738
:100eb00042680068101a704709b504480068044b7e
:100ec00003441b681b68029309bd000014ca00108c
:100ed000000000007047000010b50021012019f04b
:100ee0001dfd044619f09cfd24b9bde81040042006
:100ef0000bf07cba0028f8d1024826f061f90028ee
:100f0000f3d110bdecc9001008b50bf08dfa043810
:100f100018bf012008bd000010b5fff7f5ff20b194
:100f2000bde81040014bdb69184710bdecc900104b
:100f300010b5fff7e9ff20b1bde81040014b5b6a37
:100f4000184710bdecc9001010b5fff7ddff20b148
:100f5000bde81040014b1b6a184710bdecc90010da
:100f6000f8b504460e4617461d4624b92846bde886
:100f7000f8401ef064bbe72000f042f930461ef056
:100f80005efbe72000f060f938461ef058fb013c9c
:100f9000ebe70000014b1860704700bf18ca001053
:100fa0002de9ff4104460020039119f067ff234b10
:100fb0001b6813b12046039998474ff47f0000f057
:100fc0007ff8602000f09ef800f090f80023009376
:100fd00001231b4a18461b4901f0b0fbe72000f033
:100fe00033f94ff47f0000f06bf80226164ddff85e
:100ff0006880164f2b4641460320134afff7b0ff87
:101000002b4639460320104afff7aaff2a464146dd
:1010100003200f4bfff7a4ff3a4620460d4b0b4928
:10102000fff79eff012e07d100222146822004b047
:10103000bde8f04119f0c6bc0126dbe718ca001074
:10104000c9d30c0280660c02a0860100e093040064
:10105000a0bb0d0000350c00f049020037b500259b
:101060000195069d079c009500f074fa04b120607c
:101070007f28a8bf7f2040b203b030bd10b5054b1c
:101080001b7800fb03f4044b0020db6898476043a7
:10109000000c10bd3a5100102051001038b5054623
:1010a000c0f307400c46fff7e9ff2080c5f3072097
:1010b000fff7e4ff6080e8b2fff7e0ffa08038bdf3
:1010c000014b1860704700bf20ca0010014b186028
:1010d000704700bf24ca001010b9024b186870474f
:1010e000014bfbe720ca001024ca0010044b1a78f9
:1010f00022b100210120197001f03cbc704700bff3
:101100001cca0010014b1870704700bf3a51001004
:10111000014b1878704700bf3a510010024b18601d
:10112000024b1960704700bf28ca00102cca00107b
:1011300010b5054b0446db68002098472402b4fb39
:10114000f0f0c0b210bd00bf205100102de9f341f6
:10115000dff83480044600216846d8f80830984704
:101160006e46671e02340020d8f80c3036f8025b59
:1011700098472d02b5fbf0f507f8015fa742f2d1c1
:1011800002b0bde8f08100bf2051001010b4054b43
:1011900082885c684188a446002300885df8044b7f
:1011a000604700bf2051001030b50e4d85b0044699
:1011b000fff7ecff2b689bb12088fff7b9ff039086
:1011c0006088fff7b5ff0290a088fff7b1ffdde967
:1011d000022103460020009003482c680068a047c5
:1011e00005b030bd28ca00102cca001007b56946ea
:1011f000fff754ff6846fff7d7ff03b05df804fb25
:1012000008b510b1e72805d008bd0120bde80840a9
:101210001df047bc074b1b7853b1074b1868fff70d
:10122000e5ff6322054b1a70ff22054b1a70ebe7ae
:10123000044bf3e71cca001024ca001039510010f7
:101240003851001020ca001008b510b1e72804d0aa
:1012500008bdbde808401df024bc0020fff7c6ff14
:101260000022034b1a700122024b1a70f0e700bff4
:10127000395100103851001013b518b1e72807d0c4
:1012800002b010bd104b5b6902b0bde810401847ba
:101290000e4b1b78a3b10e4b1c680b4b00219b68b7
:1012a00068469847bdf80220bdf800301343bdf8ea
:1012b000042013439bb22bb10020fff797ffdfe719
:1012c000044be9e72046f8e7205100101cca001043
:1012d00024ca001020ca001038b5094b1a7802f051
:1012e000ff0462b90125214620461d7001f042fb32
:1012f0002046fff77bff034b1c70034b1d7038bd6e
:101300001cca0010395100103851001013b50446a2
:1013100008466946fff7c2fe6322bdf8003063430a
:10132000b3fbf2f3adf80030bdf802306343b3fb1a
:10133000f2f3adf80230bdf8043004fb03f0b0fb6b
:10134000f2f0adf804006846fff72eff02b010bdc2
:1013500010b40f4c024623780e4983b9012008705f
:101360000878e72a0344d8b220700ed10a4b1b78c4
:101370004bb10a4b19685df8044bfff7c7bf632bed
:10138000eed1ff20ebe7064bf4e75df8044b704726
:1013900039510010385100101cca001024ca001026
:1013a00020ca0010024b1878003818bf012070477f
:1013b0001cca001084b030b503ac84e80f00064ca2
:1013c00003ad0fcd0fc495e8030084e80300bde82a
:1013d000304004b0704700bf2051001070b5054682
:1013e00000200e4614462cf075f840b123463246d4
:1013f000696840304bf00cf8231a5842584170bdd0
:1014000070b5054600200e4614462cf063f840b136
:1014100023463246696840304bf0b5f9231a5842ea
:10142000584170bd01211020aef0a8bc08b510b124
:10143000aef09afe012008bd01210c20aef09ebc4a
:1014400008b510b1aef090fe012008bd30b50446dd
:1014500085b078b1684630f057f96a46234604ad46
:10146000144603ccac4218605960224603f10803cd
:10147000f6d1012005b030bd1fb5044648b101a822
:1014800030f0eefc01ab03cb206018686160a06017
:10149000012004b010bd000038b50d46044608b95f
:1014a000002038bd0029fbd000202cf013f80028c4
:1014b000f6d00023e360044b0120c4e900354ff06f
:1014c000ff33a360ede700bf5d130002f8b50e46e1
:1014d000054608b90020f8bd0029fbd000202bf0fc
:1014e000f9ff04460028f5d04034314620464af042
:1014f00094fd0746314620464af091fd002fe9db76
:101500000028e7db034bc01ba860c5e900360120bb
:10151000e1e700bf81130002002908bf3221024b1e
:101520001970024b186070473b51001034ca00100c
:1015300070470cb402b07047034b1860034b19603e
:10154000034b1a60704700bf38ca00103cca001035
:1015500030ca00102de9f04f4ff0010c00244ff07d
:10156000ff36d0f804e0964504d211f80e80b8f1a9
:10157000000f09d18268511e03eb0213002980f28b
:10158000a8812046bde8f08fb8f13a0f7dd033d85e
:10159000b8f1220f00f0a58010d8a8f109085ffa71
:1015a00088f8b8f1170f0dd8ac4d0cfa08f818ea06
:1015b000050f07d0456801354560d2e7b8f12c0f1b
:1015c00000f02981d0f8048042450ed911f8085066
:1015d0005db13a2d00f25e811f2d00f246810a2d89
:1015e00000f25581082d40f24b81002b40f05781cd
:1015f00008f1ff354560a4e0b8f17b0f1dd00ad893
:10160000b8f15b0f19d0b8f15d0fdbd1002bd1d051
:101610004ff0020906e0b8f17d0fd3d1002bc9d0fd
:101620004ff001098568013d03eb0518002d2fda05
:101630000135bfd16ff00104a3e70134002bb9d00d
:101640008568099faf4265d905f1010ec0f808e031
:101650004fea051a03eb051e0025cee90166cef818
:101660000c50c5686f1c1fbf03eb0519d9f80c504f
:101670000135c9f80c50b8f17b0f0cbf01250225cc
:1016800003f80a504568cef804508568013d1ce017
:10169000d8f8047001371ad0d8f808a0baf1ff3f83
:1016a00015d198f800b0cb45c4d10ef1010ec0f8a9
:1016b0000ca0c8f808e003eb051edef80470013743
:1016c00009d0def80870013705d1c56072e7013d29
:1016d000a8f11008aae7013d6f1caef1100eecd185
:1016e00068e70ef10109c0f80490d0f80480424583
:1016f00002d911f8085025b9c0f804e06ff00204cf
:101700003fe7222d2dd1e3b18568099faf4204d870
:10171000c0f804e04ff0ff3433e700274ff0030a2e
:1017200005f1010e4fea051803eb0515c0f808e0b6
:10173000c5e90166ef60d0f804e003f808a0c5e948
:10174000019ec56801346f1c3ff434af002b3ff499
:1017500031af03eb051edef80c500135cef80c500e
:1017600028e75c2d11d108f1010595420dd24560a5
:101770004d5d752d2cd86d2d0bd8662d28d85b2d81
:101780001ed8222d01d02f2d22d14568013545606c
:10179000abe76e3d072d1bd801a757f825f000bf1a
:1017a0000b170002511700025117000251170002d7
:1017b0000b170002511700020b1700025717000207
:1017c00040f241475c3dedb20cfa05f53d42dcd1fb
:1017d000c0f804e02ee74ff0040a08f10205456066
:1017e000d0f80480424512d911f808507db1a5f116
:1017f000300bbbf1090f04d925f02005413d052d23
:10180000e6d808f10105baf1010a4560e8d145685a
:10181000013d4560b9e7002b3ff4ccaec5682d0112
:101820005d5d013d012d7ff6c5ae856805f1ff3890
:1018300003eb051eb8f1000ffff6bcae1ef8105cfe
:10184000013d012d0cd85ef80c5c013508d05ef826
:10185000085c013504d1c0f80c80abe613008000b1
:1018600008f1ff38aef1100ee4e7a5f120091f4f93
:101870005ffa89f90cfa09f919ea070f7ff4b5ae96
:10188000203d5e2da4d808f1010545609ae60d2d96
:10189000f6d1aae605f0df09b9f15d0ff8e7856832
:1018a000099faf427ff634af002705f101084feae8
:1018b000051903eb0515c0f80880c5e90166ef605e
:1018c000d0f8048003f80970c5e901e84568013dd6
:1018d00090e653f80c2c013204d053f8082c013256
:1018e0003ff40caf0139103b48e600bf0110000483
:1018f0000023c0e901334ff0ff33c36070476ff03e
:10190000770070476ff0770070476ff0770070478f
:101910006ff0770070476ff07700704700207047d6
:10192000002070472bf030bd2bf00abd38b50d46b6
:10193000002104460171816038220c30aef061fc58
:1019400025b90a20074a0849fff72afb2846aff0c5
:1019500041fd206020b90a20024a0449fff720fb1c
:10196000204638bdbff501025c670c027d670c02a2
:1019700010b50446006808b1aef0f6fb204610bd75
:1019800010b58368044623b90a20034a0349fff7c8
:1019900007fba068403010bdbff501029f670c0235
:1019a00038b5044685682846fff7beff237963b142
:1019b0002046fff7e5ff04f10c014af030fb044636
:1019c0002846fff7afff204638bd6ff0d104f7e798
:1019d00070b5054686683046fff7a6ff2c794cb1f6
:1019e000002328462b71fff7cbff05f10c014bf0cc
:1019f000d7f904463046fff795ff204670bd2de924
:101a0000f0430c7807460e46c3b0acb30846fff768
:101a1000b9f92f2c804601d101282cd02f21701c20
:101a2000aff0b5fc002405464ff02f0925b3ab1be2
:101a3000434521d804bb2c703846fff7a1ff6a4606
:101a400031464af0f5fa041e0eda3846fff798ffe1
:101a500031464bf04bfb044628462f2100f8019bf2
:101a6000aff095fc0546e1e79df80030222b18bf4a
:101a70006ff0d104f0e70024204643b0bde8f083c6
:101a800037b50d4604460192fff77aff2a46019bbf
:101a900004f10c0103b0bde830404af0d8be37b5c0
:101aa0000d4604460192fff76bff2a46019b04f1a5
:101ab0000c0103b0bde830404af065be38b50446bd
:101ac0000d46fff76dff002802db0f2801dc0948f7
:101ad00038bda0f1100100222046fff7d1ff0028f9
:101ae000f5db102229462046fff7d9ff1028eed15a
:101af0000020ede7e8feffff1fb50446002110229d
:101b00006846aef07efb69462046fff7d7ff28b94e
:101b1000034a0399034b914218bf184604b010bd05
:101b2000e5114f71e8feffff2de9ff41054687688b
:101b30003846fff7f9fe95f80480b8f1000f07d09a
:101b400000243846fff7eefe204604b0bde8f081e1
:101b50002e462846fff714ff56f80c2b40f20313cd
:101b600031464bf0c1fb04460028ead1012301466f
:101b7000102268462b71aef044fb2846fff7bcffed
:101b80000028ddd0154b284603930194fff7f8fe9b
:101b9000224631464af074fe041e16db4246414698
:101ba0002846fff76dff041e0fdb2846fff7e8fe0f
:101bb00010236a4631464af02bfc041e05db2846fa
:101bc00000f04cf804460028bad02846fff7d8feab
:101bd00031464bf0e5f800232b71b2e7e5114f7168
:101be000f8b5064600202bf075fc054620b90a2002
:101bf000174a1849fff7d4f92846fff795fe2846fb
:101c0000b5602bf0e3fb20b10a20114a1249fff71f
:101c1000c7f937682f213846b0f089f9044640b932
:101c20003046fff781ff04462846fff77bfe20463b
:101c3000f8bd8742f4d00023037031683046fff7c7
:101c4000defe2f23237004460028e9d0ece700bf16
:101c5000bff50102b4670c02c8670c0270b50446f8
:101c600086683046fff760fe23799bb12046fff778
:101c700087fe04f10c014bf04bf8054628b12046d5
:101c8000fff7a6fe2046fff74fff3046fff74afe5c
:101c9000284670bd6ff0d105f7e737b50d4604460d
:101ca0000192fff76dfe2a46019b04f10c014af0f8
:101cb000affb051e09da2046fff7d0ff28b120460a
:101cc000fff786fe2046fff72fff284603b030bd02
:101cd0002de9f0430646856887b028461f468946a9
:101ce0009046fff721fe3379002b40d0304602a901
:101cf000fff7e4fe041e33db039c002c30db21469f
:101d000000223046fff7bcfe041e29db0023adf89d
:101d1000063044f6ad63082269463046adf800301f
:101d2000adf80290adf80470fff7b7ff041e17dba3
:101d30003a4641463046fff7b0ff041e10db0d4b1c
:101d400010220593039b304608331f4402a90397d2
:101d5000fff7a3ff041e03db3046fff77fff0446b7
:101d60002846fff7dffd204607b0bde8f0836ff09f
:101d7000d104f5e7e5114f712de9f04f89b00191dc
:101d800004a9814617469846fff798fe04460028a6
:101d900043d14ff0ff34054682462646059905f1aa
:101da00008028a42ab4617d8002229464846fff768
:101db00067fe002835db082248460deb0201fff7dd
:101dc0006efe07282fdd44f6ad62bdf80810914283
:101dd0000cd00235002de1da002f1ada01361ad0c4
:101de000b8f1000f19d0a8f800a016e0bdf80a104d
:101df000019bbdf80c20994208d10136b7429246aa
:101e000006d908322c4602eb0b05e3e72546f8e736
:101e10002c46b742e4d06ff0a904204609b0bde8d3
:101e2000f08f0446f9e7014cf7e700bfe8feffff3b
:101e30002de9ff410546d0f808801c46404616466d
:101e40000191fff771fd2b7923b3019906b924bbea
:101e500028460a9a0df10e03fff78eff011e1edbc6
:101e6000bdf80e70a74228bf2746c7b100222846fa
:101e70000831fff705fe041e05db3a4631462846c9
:101e8000fff70dfe04464046fff74cfd204604b028
:101e9000bde8f0816ff0d104f5e7024cf3e76ff095
:101ea000a904f0e7f2feffff2de9f04f0446d0f859
:101eb000089097b048460f461646fff735fd94f850
:101ec00004a0baf1000f00f08c804ff00008c34668
:101ed0003246394620460df10e03adf80eb0fff73d
:101ee0004bff051e0cda002e03dab8f1000f18bf05
:101ef00000254846fff716fd284617b0bde8f08fcd
:101f00002046fff74dfd04a980462046fff7d6fd89
:101f10000246002863d12046fff732fd22680123e4
:101f200008a94bf0e1f90246002858d1bdf80e305f
:101f3000294620460193fff7a3fd021e4fdb019bbc
:101f4000204608331d44fff71bfd2a46002308a93d
:101f50004af07dfc021e42db0599a94215d9aab3bd
:101f60002046fff70dfd0df10d02012308a94af0ef
:101f70000afc021e2adb012220460df10d01fff7ab
:101f80008cfe021e22db0135e6e7fab16ff0070591
:101f90001022bdf80e302046eb1a0b440deb020167
:101fa0000593fff77afe021e19db2046fff7e8fcd7
:101fb000bdf80e2004f10c01aa1a42444af060fc5c
:101fc000021e0cdb2046fff749fe02462046019226
:101fd000fff7d6fc08a94af0e3fe019a22b11546a4
:101fe00087e76ff0d10584e7002ef8dad0466fe777
:101ff0002de9f3410546d0f808801f4640461646b5
:102000000191fff791fc2b79bbb101992846089a01
:10201000fff74aff0199044610b110f1aa0f05d14c
:102020003b4632462846fff753fe04464046fff73c
:1020300079fc204602b0bde8f0816ff0d104f5e7ed
:102040000148fff795bc00bf44ca001010b5044614
:102050000249fff76bfc204610bd00bff0670c0281
:1020600010b50b4cd4e88f3fdb070cd420461ef094
:102070004dfc40b10748fff7e9ff20461ef080fc09
:102080000548adf070fe0348fff7aafd014810bdfa
:1020900040ca001044ca0010c11f000213b500243a
:1020a0009bb20094fff7c4fe02b010bdb3f5803fb1
:1020b00013b506d200249bb20094fff799ff02b03b
:1020c00010bd6ff0bd00fae72de9f0418046c2b0c7
:1020d00000200d4617462bf0fdf9044618b34ff4c7
:1020e0008472002168464034aef08bf86a46294677
:1020f000204649f09dff50b32f212846aff017ff2f
:10210000b8b1854215d0411b2846aff0e1fe064626
:10211000c8b1014620464af0e9ff38b1113005d078
:102120003046aef021f86ff0e0000de03046aef042
:102130001bf847f480773b462a46414620464bf041
:10214000d3f808b1efe7044842b0bde8f0819df84c
:102150000030112befd0e6e7fcfefffff8b5074695
:1021600000200d461646fff767f90446a0b100228d
:102170003946fff7abf928b132462946204630f000
:102180009ff938b96ff0e00500212046fff758f9b4
:102190002846f8bd0025f7e7004df9e7fcfefffff4
:1021a000f8b5074600200d461646fff73bf90446f2
:1021b000a0b100223946fff76ff928b1324629460f
:1021c00020462ff081fc38b96ff0e0050021204651
:1021d000fff72cf92846f8bd0025f7e7004df9e791
:1021e000fcfeffff0fb413b50a4b586a25f01dfe25
:1021f00058b1094c05ab80212046049a0193b0f0f8
:1022000043fa0028bcbf0023237002b0bde8104091
:1022100004b0704770cc001088ca001008b5044b99
:10222000586a25f002fe10b10022024b1a7008bd58
:1022300070cc001088ca0010021e80f2348112f5a2
:10224000967f00f0328100f3b580a64b9a4200f0f1
:102250002e8101339a4271da12f5c86f51dca3f571
:1022600080739a423edaa0487047c9320b2afad8e6
:1022700001a353f822f000bfff230002fb2300025a
:10228000e7210002e7210002e7210002e721000226
:10229000e7210002e7210002e7210002e721000216
:1022a000f723000233240002e6320b2adbd801a315
:1022b00053f822f00f240002e7210002e721000278
:1022c000e7210002e72100020b240002e7210002bf
:1022d000e7210002e7210002072400020324000294
:1022e0003724000202f24562052a00f2da80dfe8b4
:1022f00012f0d600d400d200d000e40006007b48e3
:1023000070477b4b9a4200f0da8001339a420ada36
:1023100012f5af6f00f0d5807649734b76488a424c
:1023200018bf18467047754b9a4200f0cc806e4833
:10233000734b12f5aa6f08bf18467047714b9a424b
:1023400000f0c38001339a421bda1f3b9a4200f02f
:10235000be806ff4a6639a420bda0b3b9a4200f000
:10236000b88009339a4200f0b68067495e4b6748ef
:10237000d5e712f5a56f00f0b08065495a4b654866
:10238000cde7654b9a4200f0aa8001339a4208da01
:102390004f3b9a4200f00a815348604b12f5966f0a
:1023a000c9e75f4b9a4200f003814f485d4b12f53d
:1023b0007a7fc0e712f1bd0f2eda12f1c90fbff616
:1023c00054af12f1da0f20da12f1e60fbff66caf5c
:1023d00012f5827f00f0ee800cdc12f58c7f00f0ad
:1023e000eb8012f5877f00f0e9803f484e4b12f5f5
:1023f000917fa0e712f1fa0f00f0e2803a4b4b48d0
:1024000012f1f00f18bf18467047374b484812f1c9
:10241000d20f18bf1846704712f18c0f00f0d2800f
:1024200012f18b0f18da12f1a00f00f0cd8012f12b
:102430009f0f0ada12f1b40f00f0c8802a4b3d4812
:1024400012f1aa0f18bf18467047274b3a4812f1ed
:10245000960f18bf1846704712f1780f00f0b88039
:1024600012f16e0f00f0b6801f4b344812f1820f4c
:1024700018bf184670473248704732487047324894
:102480007047324870473248704732487047324888
:102490007047324870473248704732487047324878
:1024a0007047324870473248704732487047324868
:1024b0007047324870473248704732487047324858
:1024c0007047324870473248704732487047324848
:1024d0007047324870473248704732487047324838
:1024e000704700bfb9faffff1f680c02d3680c02e7
:1024f0009cfaffff92faffffdc680c02a6faffffce
:10250000a7690c02ecfaffffbafaffff77690c0229
:10251000e2faffffe5690c0294fbfffff8690c0289
:10252000b4fbffff526a0c025d6a0c02ad6a0c023a
:10253000336b0c02296b0c02ff670c02636b0c02fd
:10254000d96a0c02ca6a0c02bc6a0c02a46a0c02a8
:10255000926a0c02876a0c02796a0c027a680c0291
:1025600068680c0256680c0244680c022d680c0264
:1025700047420d0208690c024f6b0c02e96a0c021b
:102580009e6a0c0295680c02a8680c02c6680c02d0
:10259000f2680c0266690c0229690c0247690c0298
:1025a00013690c028e690c02bf690c020a4870475d
:1025b0000a4870470a4870470a4870470a487047f7
:1025c0000a4870470a4870470a4870470a487047e7
:1025d0000a4870470a487047c9690c020b6a0c0226
:1025e000266a0c023e6a0c02156a0c026a6a0c0228
:1025f000156b0c02f86a0c02066b0c0211680c02d7
:10260000416b0c0210b5084b0446586a25f00dfcce
:1026100010b1064803782bb92046bde810400021d0
:10262000fff70abe10bd00bf70cc001088ca0010b2
:10263000a0f13003dab2092a01d818467047a0f198
:102640006103052b01d857387047a0f14103052bd2
:1026500094bf37384ff0ff307047102af8b5064660
:102660000c461bd900252078fff7e2ff071e15db7b
:102670006078fff7ddff031e10db43ea0713052d2b
:10268000735505d102340135062decd1012006e049
:10269000a278e31c3a2a01d11c46f4e70020f8bdd9
:1026a000034b1860034b1960034b1a60704700bf5f
:1026b00008cb00100ccb001010cb0010f0b5164b5f
:1026c00005461e680f461446abb036b9134b1b685f
:1026d00003b3134b1b7883421cdc23791b0706d4fe
:1026e0001ff0e5fe2379606143f0080323718eb18a
:1026f000dde93023a02102a8aff0c6ff9f28c4bfa8
:102700007e238df8a63000233a46009329462346bf
:1027100002a8b0472bb0f0bd08cb001034ca00109f
:102720003b51001030b585b008ac54f8045bcde9de
:1027300000540394fff7c2ff05b030bd70b40446e7
:102740000d46104619464bb1054b1e6836b10023a5
:1027500022460393b4462b4670bc604770bc70475a
:102760000ccb001070b51a46134b04461d680e467c
:10277000aab035b9114b1b68bbb1114b1b78834212
:1027800013dc2e9ba02102a8aff07eff9f28c8bfbc
:102790007e230146c4bf8df8a6309f213db10023a2
:1027a0002246009302a83346a8472ab070bd034bc7
:1027b00002a81b689847f8e70ccb001034ca001039
:1027c0003b51001008b410b585b007ac54f8043b79
:1027d00000940394fff7c6ff05b0bde8104001b0b8
:1027e000704700002de9f04f8846294907460d68db
:1027f000adb0002b3ad035b926490968b1b32649a6
:102800000978814232dc00211446dff89090dff82d
:1028100084b08df8ac10d61814f8013b2ca84fea00
:10282000131c19f80cc0084403f00f034a1c00f8ed
:10283000a4cc19f8033002312ca80244a02902f8d4
:10284000a43c09d1adb14ff0000a43463a46cdf859
:1028500000a003a8a8475146a642ddd131b175b109
:1028600000233a46009303a84346a8472db0bde88d
:10287000f08fdbf8003003a898472946ece72cab33
:102880001944044b01f8a45c1b6803a89847ede7c2
:102890000ccb001034ca00103b510010a46b0c028a
:1028a000074b02461b680bb100221847054b1868fe
:1028b00028b1054b1b789a42b4bf00200120704715
:1028c00010cb001034ca00103b5100104528dabf6d
:1028d0000a2390fbf3f00620034bd8bf20eae070f8
:1028e00053f82000704700bf886b0c0270b50d468e
:1028f000044620b90a201c4a1c49fef751fb17f078
:1029000009ffa37bdb070bd563680bb1a2689a6054
:10291000d4e9013282b15360a37b03f0fe03a373b9
:1029200013490b686db1002283b11e7b257bae423b
:102930000bd91a465b68f7e70d4a1360ece70c60a9
:1029400007e063b901238b7409e09c60002af6d08c
:102950005460c4e90132a37b43f00103a373bde8d3
:10296000704017f0dbbe00bfbff50102b56b0c0273
:1029700014cb001010b5044617f0ccfe094b1a8a90
:102980005cb1013a92b21a821a8a92b20ab9012251
:102990009a74bde8104017f0c1be013292b21a829b
:1029a000f7e700bf14cb001010b517f0b3fe044bcf
:1029b0001c8a17f0b3fea4b2b4fa84f0400910bd2b
:1029c00014cb00102de9f04f85b04ff000090546fb
:1029d00017f0a0feca4683464b46012049464f46a3
:1029e0004e464a46614cd4f8008010b3b8f1000f4f
:1029f0001fd098f80d300f2b5ffa83fa15d1d8e964
:102a00000531284698470022d8f8106098f80e1033
:102a1000238a94f812909bb2b3fa83f30020c9b2d0
:102a20005b095ffa89f9a274dde7b8f81470bfb2e8
:102a3000eae75846cde9021317f070fedde902130c
:102a4000a27a524502d1a289ba4261d0002284f80a
:102a50000aa0a781e281002b57d011f0020067d1b4
:102a6000434bc6f307481f78424bffb2db689847d9
:102a70007843f5b2c6f3072700fb08f84743454300
:102a8000b4f80cc04fea18413a0c280c8846174697
:102a90000546bcf1000f05d0a67ae389022e44d08a
:102aa000032e49d0b9f1000f08d1a388434505d1c1
:102ab000e388bb4202d12389ab4226d0dff8b49031
:102ac0000023d9f804602a4639464046b0472a4eca
:102ad0003368b3b1d9f80c30002098474fea082189
:102ae0002b023a02b3fbf0f3b2fbf0f2b1fbf0f0d1
:102af00000210091c1b2214836680068dbb2d2b231
:102b0000b047a4f80480e780258105b0bde8f08fc8
:102b1000002fa0d0e0890544adb2bd4224bfb5fb73
:102b2000f7f207fb1255e58195e7b3eb5c0fb9d3dc
:102b300000252f46a846b5e74fea5c06b3eb5c0fcd
:102b400034bff31a9b1b9bb203fb01f803fb02f794
:102b500003fb00f5b8fbf6f8b7fbf6f7b5fbf6f5a7
:102b60001ffa88f8bfb2adb29ce700bf14cb0010cb
:102b70003a5100102051001028ca00102cca001031
:102b8000064b0022194641f8042b5a601a828a80ab
:102b90005a81da6001229a74704700bf14cb00108a
:102ba00070b5d0e90043204643f31d03002b0ddd33
:102bb0005a1050f8226000eb8205b6888e4203d28c
:102bc0009b1a281d013bf1e71346efe7001b80101d
:102bd00070bd000070b51048d0e88f5f15f001059a
:102be0000e4e16d11df092fe98b110201bf0f0fd94
:102bf000044650b1c0e90055856005738020adf0f2
:102c0000abfa10b120232060a360034834601df0ac
:102c1000b7fe306870bd00bf28cb00102ccb001071
:102c2000f8b50746fff7d6ff037b044673bbb988a8
:102c3000fff7b6ff0546d4e90006b54204da50f8be
:102c400025309b888b4224d0a3689e420ddb013641
:102c5000002e05ddb100aef055fa20b90e4814e0a3
:102c6000adf082fa00202060a6602668626806eb5c
:102c700085019200a2eb8502081dadf0a8fa0020a4
:102c800046f82570636801336360f8bd6ff0d100ca
:102c9000fbe76ff0b300f8e7fcfeffff2de9f84318
:102ca00007460e469046fff795ff037b0546a3b106
:102cb00077b1d0e9004304eb83094c45234607d0a4
:102cc000414618680434b8470028f6d0bde8f883b8
:102cd00036b16b6800203360f8e76ff0d100f5e79c
:102ce0003046f3e770b506460c46fff773ff037beb
:102cf00005467bb13146fff753ff6b6898420cda0b
:102d00002b6853f820309a88b24206d144b1002093
:102d1000236070bd6ff0d100fbe76ff0a900f8e70a
:102d20002046f6e710b50446fff754ff022c05bf16
:102d3000012303736ff07700002010bd38b53822ef
:102d40000d4600210446adf05cfa4ff0ff3200233f
:102d50002046c4e90f23a56338bd000030b5054601
:102d60008db000202af0b6fb044618b32af0e8fa2a
:102d70002b6c990706d4002520462af005fb28462f
:102d80000db030bd294604f1400049f0c1ff0028d4
:102d9000f1da202200230290cde90423aa6b32202d
:102da0000192064a0649009204aafff7bbfc6ff0a5
:102db000e005e1e76ff0e005e1e700bfd56b0c024d
:102dc000cd6b0c02002370b501f1400604460146ac
:102dd0001a4630468eb049f03afd00284ff0000503
:102de00011da2023cde90635a36b029001930f4b36
:102df000322000930e492b4606aafff793fc6ff092
:102e0000e0000eb070bd04232146304605aa0595aa
:102e100049f0b9fc042807d02023cde90635a36b7f
:102e200002900193034be3e70598eae7f46b0c0289
:102e3000cd6b0c02136c0c0210b50446236c0846d3
:102e40008cb0abb12146403049f0aaff00280dda22
:102e500020220023cde90423a26b02900192054aaf
:102e600032200092044904aafff75cfc002323648b
:102e70000cb010bd326c0c02cd6b0c0238b505469f
:102e800000202af027fb044650b12af059fa2846c0
:102e90002146fff7d1ff2046bde838402af074ba3a
:102ea00038bd000030b505468db000202af012fb79
:102eb000044610b32af044fa21462846fff7bcff27
:102ec000a96b04f140004af017fa00280fda811cc0
:102ed0000dd020220023cde90423aa6b0290019299
:102ee000074a32200092074904aafff71bfc20463c
:102ef0000db0bde830402af047ba0db030bd00bf7c
:102f0000526c0c02cd6b0c02002a70b540f6031512
:102f100018bf0125036c044635ea03030e468cb046
:102f20001fd0fff789ff2b462146a26b06f1400018
:102f30004af0daf9002813da811c14d02022002389
:102f4000cde90423a26b02900192084a322000923c
:102f5000074904aafff7e6fb6ff0e0000cb070bd74
:102f600025640020fae76ff0a900f7e76e6c0c0209
:102f7000cd6b0c022de9f04705468cb00020894648
:102f800090462af0a7fa0746002863d02af0d8f91d
:102f9000012239462846fff7b7ff041e1bdb07f165
:102fa000400a2946504649f03af8061e10da202019
:102fb0000023aa6bcde904030192284a02960092ed
:102fc0003220274904aafff7adfb6ff0e00402e0ce
:102fd000032e07dc234c38462af0d6f920460cb0e5
:102fe000bde8f087eb6b002b09da39462846fff77e
:102ff000e9fe041eefdb17d1042eebd1ec63ea6b84
:1030000000239045a8bf904629465046b21a49f081
:103010001efc00280cda20210023aa6bcde9041342
:1030200001920290104acae7f31ea342e6dcd1e700
:1030300043464a462946504649f0a5fb804504468a
:10304000c9d020220023cde90423aa6b029001926b
:10305000064ab4e76ff0e004c0e700bf8d6c0c02d5
:10306000cd6b0c02e8fefffff46b0c02136c0c023c
:103070002de9f04705468eb00020894616462af015
:1030800029fa804600287fd02af05af900224146ca
:103090002846fff739ff041e18db08f1400a2946cd
:1030a000504648f0bcff071e17da4ff0200c0023f3
:1030b000aa6bcde906c30192354a029700923220ed
:1030c000344906aafff72efb6ff0e00440462af0d1
:1030d0005bf920460eb0bde8f087032f0fdc00221d
:1030e0002946504649f0ccfb002828da2026002348
:1030f000aa6bcde9066301920290274adee7eb6beb
:10310000002b06da41462846fff75cfe041edddb95
:10311000ec63eb6bb342e2d13744b7f5805fdedca2
:1031200033464a462946504649f072f986420446db
:10313000ccd0202200230290cde906231ee00023fc
:1031400029461a46504649f082fb002808da202416
:103150000023aa6bcde90643019202900f4aade726
:1031600004232946504605aa059649f051f904283a
:1031700008d020210023cde906130290aa6b01920a
:10318000074a9be7ee63cbe76ff0e004a1e700bfdf
:103190008d6c0c02cd6b0c02ac6c0c02f46b0c024f
:1031a000cf6c0c027047704770470000074b1a78cd
:1031b00012b10021064a11705a7812b10121054a54
:1031c00011709b780bb109f0e1b8704730cb00105b
:1031d00076cf001074cf0010fff7e8bf10b5c368ba
:1031e00004460bb9acf066fa036904309847002135
:1031f000a0616069bde8104024f050bf10b509f02f
:10320000edf8124b124c1b780246b3fa83f35b09bc
:10321000a070237080b1012000220521607010464b
:1032200004f072fa09f0d4f8bde8104000231a4601
:103230001946184604f004bb014604f03ff9024663
:103240000028e8d1014604f088f9e5e776cf0010c0
:1032500030cb0010012af8b5064603d10b68036095
:103260000020f8bd022a08d0032af9d100680028fe
:10327000f6d01c211bf0b4faf2e71c200c681bf0fe
:10328000a7fa074630b105460fcc0fc594e80700f2
:1032900085e807003760e3e7012a70b5054603d1ea
:1032a0000b680360002070bd022a08d0032af9d100
:1032b00000680028f6d010211bf092faf2e71020e7
:1032c0000e681bf085fa044618b196e80f0084e8f2
:1032d0000f002c60e6e7000070b5037d04460e4643
:1032e000154683b10368db6873b19a88012a06d05a
:1032f0009b68f9e79b683bb19a88012afad19a89c1
:10330000b242f7d19d7370bd002110200bf0e4fe96
:1033100008b92075f7e7054b036001238380236913
:103320008681836085732061ede700bf1000030094
:1033300038b5037d04460d466bb10368db6823b1e5
:103340009a88042a11d09b68f9e7002110200bf01d
:10335000c3fe08b9207538bd054b03600423838084
:103360002369c0e902352061f5e7dd60f3e700bfbe
:103370001000030010b58368044613b10322014610
:103380009847204610bd000010b50446034b40f896
:10339000043bfff7efff204610bd00bf80720c0218
:1033a00010b50446fff7f0ff204614211bf018fa71
:1033b000204610bd10b5074b04460360406918b1a4
:1033c00024f047fe002363612046fff7ddff20461f
:1033d00010bd00bf94720c0210b50446fff7eaff5f
:1033e000204618211bf0fcf9204610bd10b50446fc
:1033f000024b0360fff7deff204610bda8720c02ef
:1034000010b50446fff7f2ff20461c211bf0e8f937
:10341000204610bd38b50446006928b185680021f2
:103420000bf06cfe2846f8e7204638bd002330b587
:1034300087b0cde90233049301238df814301023b3
:10344000adf80430032301ad00280c460095adf81b
:1034500006308df8083005dd4ff47a714143684637
:10346000fff766ffa30704d401220a216846fff78d
:1034700033ff0120fff797fe0022284611461af07d
:103480009bfd04466846fff7c5ff204607b030bde8
:103490002de9f0470e4698461021002388b0cde96b
:1034a00004330693adf80c10012303211746109a3c
:1034b0000df10c09002a0546cdf808908df81c3056
:1034c000adf80e108df8103005dd4ff47a7102a8ba
:1034d0005143fff72dffb5b1beb1002f3cd0b8f17d
:1034e000000f39d0002407eb080ab4420dd0444540
:1034f00035f8141034bf3a5d1af8012c02a8fff712
:10350000ebfe0134f1e72c46ede700270120fff741
:103510004afe3a46484601a901971af04dfd041e9d
:1035200011dbfff741fe0198c0b183883c46012bb7
:1035300007d1b4420ed035f81430828901349a4252
:10354000f7d1acf011fe02a8fff764ff204608b0e7
:10355000bde8f0870024f4e7014cf4e70446f2e705
:10356000f2feffff73b506461c200d461bf030f936
:10357000044628b3144b03600023c360ab683bb11f
:103580000222294604309847eb682361ab68e36068
:10359000002220460d4b0121236040f8142f24f017
:1035a0004dfd0b4b30462360336801945b6801a9e5
:1035b0009847054620b9236820469b6898472c46c3
:1035c000204602b070bd00bf80720c0294720c02e3
:1035d000a8720c02f0b51f463c4b164693f82c20ff
:1035e00005460c4689b0f2b1586a24f01efcd0b9e9
:1035f000069010201bf0ecf818b1c0e901460570e8
:10360000c760334b04900793324b304804a90693ac
:10361000fff7a8ff0546b8b9044604a8fff7aafebd
:10362000204609b0f0bd02f0a1fbc8b9f34313f086
:10363000010300d195bbfff7e1fd012d3ed0022d26
:103640003cd0bdb10024ebe700224ff0ff314069d0
:1036500024f004fd2b6828469b68ac699847dce79a
:1036600016f00403e2d11a460621012000940bf063
:10367000bffadbe7002cd3d0e317cde904430121e7
:103680002b46154a009504a8cde906551ff05cf8b5
:1036900004460028c4d0fff789fdc1e7012d0dd0f5
:1036a000022dcfd11a4618460521039304f02cf8b9
:1036b000039b1a461946184604f0c2f831462046c4
:1036c00009b0bde8f040fff7b1be00bf70cc0010fc
:1036d0005d3600021932000259310002006841686b
:1036e000d0e902230078fff775bf2de9f0411f46ae
:1036f000002304460d46164601211a46184603f0db
:103700004aff3b46324629462046bde8f041fff7d6
:1037100061bf00002de9f04f9846504b174693f8d3
:103720002c2087b00546dde910940e4622b3586a76
:1037300024f07bfb00bb04901c201bf049f838b13f
:10374000129bc0e90056c0e90278c0e90494836185
:10375000434b02900593434b404802a90493fff763
:1037600001ff0446002853d1054602a8fff702fed8
:10377000284607b0bde8f08f02f0f8fa824600282c
:1037800052d1e44314f0010403d0fff737fd4ff0aa
:10379000000a00210846fff7edf8e720fdf754fd89
:1037a00043463a4631462846cdf80090fff770fe72
:1037b000002105460120fff7ddf8e720fdf720fd99
:1037c0000cb1fff7f3fc08f02ffe0446002008f0d0
:1037d00037fe0646b8bb013ce4b2012c33d808f0f2
:1037e000fdfd80b330461ef055fe4ef660260446c1
:1037f00000201ef04ffe001b61f10001b04271f18c
:1038000000031ed202f0b2fad8b902f0bffaefe715
:1038100000224ff0ff31406924f020fc236820464d
:103820009b68a5699847a0e714f0040ba9d15b46f3
:103830005a4606210120cdf800900bf0d9f9da465e
:103840009fe702f093fabaf1000f91d006f006fd5f
:10385000002304211a4610f0fafa89e770cc001010
:10386000e9370002d53100021fb500688369029371
:103870004369019303690093d0e90223d0e9000171
:10388000fff748ff05b05df804fb2de9f0471f4640
:10389000dde90889002304460d461646ddf828a018
:1038a0001a460121184603f076fe3b463246294669
:1038b0002046cde9099acdf82080bde8f047fff712
:1038c00029bf70b51d46002388b00e461446adf8da
:1038d00016001a460121184603f05dfe0c9b009469
:1038e000cde9015301230df11f0219460df1160018
:1038f0008df81f60fff7c9ff08b070bd38b51546d9
:10390000d0e902239342044607d2d21a4068aa4261
:1039100028bf2a461844acf04dfce26801202a4436
:10392000e26038bd012a02d1016000207047022afe
:1039300004bf0b680360f8e713b50446084601911d
:10394000fdf720fa02462046236801991b6802b061
:10395000bde810401847000004281fb50346144670
:103960000cd14ff6ff7345f61b210920002a08bf32
:10397000194604b0bde8104017f0aeba01280ed1c8
:1039800000233c220093112312481349002c18bf36
:1039900001461248006802f0abfd04b010bd0928d2
:1039a0000ad100230b480c490093002c18bf014694
:1039b00011233c220a48ede70028eed1002aecd082
:1039c0000246cde90100009000214ff4007003f0a1
:1039d000c7f9e2e7b4720c02cbd40c023c510010e0
:1039e0004051001009280a4608b50dd8084b195c4b
:1039f000914203d1042801d0082803d1195c1a543c
:103a0000fff7aaff002001e04ff0ff3008bd00bf24
:103a10004d510010092838b50c4613d8a9b1042817
:103a20000b4d0cd1092017f061fa45f61b2380b22b
:103a3000c31a5842584120702871002038bd2b5cb1
:103a40000b70fae74ff0ff30f8e70846f6e700bfe3
:103a50004d51001037b500220df107010546fff763
:103a6000d9ff044628b99df8072028461146fff7dc
:103a700073ff204603b030bd014b1860704700bf94
:103a80003ccb001038b50b4b45681c6864b100f1a5
:103a9000080100222846a047044618b106492846d6
:103aa0000ff090fc204638bd044928460ff08afcf0
:103ab0000349f4e73ccb0010b9720c02e7720c0228
:103ac0001d730c020c4a0d4b00b51a601c2389b003
:103ad0000021adf804301423029001a8cde90311b0
:103ae000cde90511adf806100791adf80c30fff7e0
:103af000c9ff09b05df804fb455500023ccb00103e
:103b000010b50f4b04461b68834208d100230121e6
:103b10001a46184603f03ffd00200ff0effd00228b
:103b20001146104603f087fd024640b9054b1b685d
:103b3000a34204d1bde81040014603f031bf10bddf
:103b4000445100104851001030b50d4b05469b788c
:103b500085b003f0ff0483b9224601210220fff75c
:103b600041ff084b22461d704ff480602346002120
:103b7000cde90144009403f0f3f805b030bd00bf77
:103b80004d5100104c51001013b500240220224664
:103b90000df107018df80740fff73cff9df8070086
:103ba00060b1224603200df107018df80740fff7b1
:103bb00031ff9df80700001b18bf012002b010bda7
:103bc00007b5fff7e1ffa0b10b4b1a7802f0ff0336
:103bd00042b1002302201a46194603b05df804ebf7
:103be000fff783bd054900931a460120097808f0c4
:103bf0002dfc03b05df804fbc5d200104c51001041
:103c0000f0b585b0fff7c0ff48b3164d2b7833bb36
:103c100001222a70144a4ff400600021cde90133db
:103c200000921a4603f09cf81ef041fc47f22f5711
:103c300004460e4efff7a8ff30b90020287005b0eb
:103c4000bde8f040fff7bcbf1ef031fc001bb842de
:103c5000f3d802f09bf8304604f016f8eae705b016
:103c6000f0bd00bf40cb0010413b000270cc001003
:103c700037b5837a04460d46ebb91ff0f3f9636854
:103c800018442389206113b91ff0f8f92081e368f3
:103c900013b91ff0edf9e06015f0010f0cbf00251e
:103ca000042504f00bfd0023e1681a46009505f099
:103cb0001bf803b030bd0148fbe700bfe2faffff8d
:103cc0002de9f0411646ca0788b038d511f0020f29
:103cd0000cbf0024042404f0f1fc214604f080fe13
:103ce00014f00805074626d106b34ff0ff08294611
:103cf00042463046acf085fa124b134904a8cde990
:103d00000436cde90685fff717fe3b460c210f4a26
:103d100001a8cde901550395adf0aafa01a904a8bf
:103d2000fff70afe0a4904a8fff706fe630702d45c
:103d30004620fff709ff384608b0bde8f0810824a7
:103d4000c9e700bf6c730c025a730c02c27f0c02ed
:103d500060730c0230b50446002585b0039104f071
:103d6000adfc626823690399d31a0095228904f097
:103d700077fe05b030bd000070b5324e044696f8af
:103d80002c3086b0002b49d0706a24f04ef80546de
:103d9000002843d12c4b1c2005932c4b02940493f8
:103da0001af016fd0446002831d0294bc560036087
:103db000049b3bb1022202a904309847059b236172
:103dc000049be36000252046224b2a462360012104
:103dd00040f8145f24f032f91f4b01a92360f26907
:103de0002b46306b019424f07ef8014650b9706a7e
:103df00008b124f047f800224ff0ff31606924f049
:103e00002df9a569236820469b68984700e0054680
:103e100002a8fff7affa284606b070bd04f04efcca
:103e2000037e63b90d4b1b7803f0ff05002bf2d026
:103e30000b4b1b78002b0cbf01250225ebe703255c
:103e4000e9e700bf70cc0010e53d0002a538000294
:103e500080720c0294720c02a8720c0238cb001013
:103e60004d5100100068fff787bfc1684a6950686c
:103e700003681b681847000038b50c461546c8682b
:103e80003ab11146adf03ef938b1e060002025614d
:103e900038bdacf069f9e560f8e70148f8e700bf24
:103ea000fcfeffff10b591f843300c46db07486875
:103eb0000cd500210bf022f994f8433023f00103d4
:103ec00084f843300023c4e9013310bdacf04cf951
:103ed000f8e708b508b108f07bfa002301211a467b
:103ee000184603f058fbbde8084001f017b910b5bb
:103ef000c468a068acf030f9606016f00bfc94f870
:103f000042202ab963687bb1022384f84230144608
:103f100016f004fc6cb16068acf026f92046bde8f0
:103f2000104000210bf0eab8012284f842201c4620
:103f3000eee710bd136810b5032b17d90b685c1c96
:103f40000c6018700b685c1c0c60040a1c700b6819
:103f50005c1c0c60040c1c700b68000e5c1c0c607c
:103f6000187001201368043b136010bd0020fce7ab
:103f700073b58b6804460d4600931bb90026304686
:103f800002b070bdcb880068694601aa0193fff7b3
:103f9000d1ff06460028f1d0019b012beed9009af3
:103fa000a389511c00911370009a1b0a511c0091a7
:103fb0001370019b2268023b910701930ed5012be0
:103fc000dcd9009ae389511c00911370009a1b0af6
:103fd000511c00911370019b023b019323685a0707
:103fe0000ed423681b0706d56946606801aafff74f
:103ff000a1ff0028c2d0aa68009b9b1aeb80bee7f5
:104000006946a06801aafff795ff0028e9d1b5e746
:1040100038b50c4b416003600023c0e902330361f3
:10402000044616f077fb05462146074822f092ff2a
:104030002146064822f09aff284616f06ffb2046dc
:1040400038bd00bfc0730c0237440002594400025f
:104050002de9ff41cb8806463f2b0f4640f2938067
:10406000886860b1338a032b0cd9002301220293a4
:10407000cde90023032303936846fff779ff04b0db
:10408000bde8f081002144200bf026f8044638b941
:104090000123cde900300423029003933946ebe776
:1040a00018230380bb884ff0000843807b88c0e959
:1040b000038883606ff06303c0e90c884661406247
:1040c000c0f83880c363738a01339bb273828568fa
:1040d000a0f8403080f84380002d35d12b4b00f103
:1040e0001801c3612a4803f0fbfd032384f8423022
:1040f00063886560462b0ed010d8322b07d004d8c9
:10410000283b012b03d9002508e03c2bfbd10120e3
:10411000fff7dffef7e72846fff7dbfe0023a36289
:10412000b368e36203b19c62338ab46001333382c3
:104130000023cde90133b4f84030adf80c50adf8b0
:104140000e3003230093a9e7402d0fd8414628469f
:104150000af0c2ff606048b194f8433043f00103b5
:1041600084f84330022384f84230cce7094b0848f6
:10417000e36104f1180103f0b3fd0023022563603d
:1041800084f84230cae7002079e700bfeb3d000227
:10419000f4d600106f3e000270b58b8884685cb165
:1041a000b4f840209a4209d0e46af8e7d8b96368c5
:1041b00033448b60012070bd0020fce794f842304e
:1041c000022bf9d1cd88a66ba36872199a42f3d855
:1041d000402d8868ead80028edd0636801462a4659
:1041e0009819abf0e7ffa26ba36815449d42a56345
:1041f000e0d1064b0648e36104f1180103f070fdbd
:104200000023a363032384f84230d3e7eb3d00028d
:10421000f4d60010f8b506468b8884684cb1b4f823
:1042200040209a4207d0e46af8e7e3683b448b6099
:1042300016e0002019e094f84230042bf9d1cd8823
:10424000002df6d0a76b23697a199a42f1d8402d38
:10425000ebd8886848b1e1682a463944abf0aaff38
:10426000a06b2844a0630120f460f8bdf0b54b7842
:104270000c46502b85b00cd191f90030002b41da5f
:10428000cb8833b1886888b38a88142a03d01e2a61
:104290002ed000202ae01021684619f0d5fe102803
:1042a000f7d8e3884500b3eb400ff2d36b46a26822
:1042b0005619b24218d01f4619780232090901f185
:1042c0003000392888bf01f1370002f8020c397834
:1042d000013301f00f0101f13000392888bf01f1ed
:1042e000370002f8010ce4e7e580012005b0f0bddd
:1042f000042bced90b4b1a681b790260037105237e
:10430000cb80f2e78b88282b06d0b3f5977fc0d1fe
:104310000120fff7defde8e700228c20114616f0b1
:1043200051fbe2e7af730c0210b5cb6a0c460bb140
:104330008a6a9a62d4e90a2362b1d362038a013b92
:10434000038294f842300bb1032b05d1042384f887
:10435000423010bd8360f1e7606840b194f84330ab
:10436000db070dd500210af0c9fe00236360e36876
:1043700033b9216b21b92046bde810400af0bebe1a
:10438000044b04f11801e3610348bde8104003f059
:10439000a7bc00bf19450002f4d600101fb5cb889a
:1043a0000c463f2b38d98b68002b37d08b8881681f
:1043b00029b1b1f840209a4201d0c96af8e7002338
:1043c0000122cde90233cde9002319b391f842303f
:1043d000042b0dd8dfe803f003070c0312000223bf
:1043e000adf80c3004e00423adf80c30fff79cff6f
:1043f00021466846fff7bcfd04b010bdcb6b0193ae
:10440000092300930b691bb102930d230093efe77f
:10441000c160ede70523e3e70020ede71846ebe791
:104420007fb5cb8804463f2b0d4615d98868a0b1cf
:104430008b884bb96ff08b06a368e3b1de6320462f
:10444000a168fff771fff7e7a16841b1b1f840201b
:104450009a420ad0c96af8e7002004b070bd01236f
:104460000291cde9003105230ae06ff08b0320466d
:10447000cb63fff759ff00230122cde9002302930c
:10448000294668460393fff773fde6e74b78013b47
:10449000042b0ed8dfe803f0030507090b00fff734
:1044a000d7bdfff77bbffff777befff7b3befff7c0
:1044b000b7bf0020704708b503465a780846013a4e
:1044c0000e2a194605d8fff7e1ff80f00100c0b2bf
:1044d00008bdfff7cbfef8e7012838b50c460bd036
:1044e000022815d16ff09505a3689bb1dd632046c6
:1044f000a168fff719fff7e7c96849b18a6b0b6933
:104500009a4205d100252046cd63fff70dffe560f7
:10451000002038bde360fbe738b54b6805460c4624
:1045200013b103685b689847e3682bb12b680022de
:10453000214628461b689847236b13b1616be06bdb
:1045400098472046bde8384000210af0d7bd2de944
:10455000f0411f464b6805460c461646ddf81880ac
:1045600013b103685b689847c4e90c7816f0d2f879
:1045700094f84230032b01bf0423e66384f84230f1
:10458000002416f0cbf82cb121462846bde8f041b6
:10459000fff7c2bfbde8f081c1684869fff7bcbf43
:1045a00003681b681847000007b50022044bcde9db
:1045b00000021146104604f09fff03b05df804fbb3
:1045c0002145000208b54ff47a701bf036f8bde8bb
:1045d000084000200ff092b808b54ff47a701bf035
:1045e0002cf8bde808400ff0a1b810b5c368044628
:1045f0000bb9abf05ff80369043098472368204695
:10460000bde810409b68184708b54ff47a701bf05e
:1046100014f8bde8084000200ff08bb808b54ff43f
:104620007a701bf00af8bde8084000200ff050b87f
:1046300037b5446925680093ad6813460a460146bc
:104640002046a84703b030bd012a38b5044602d140
:104650000b68236003e0022a03d0032a0dd0002058
:1046600038bd0c200d681af0b3f803460028f0d0ce
:1046700095e8070083e80700ebe700680028eed024
:104680000c211af0adf8eae7012a034602d10160d5
:1046900000207047022a04bfd1e90001c3e90001ec
:1046a000f6e7000010b50446034b40f8043bfef764
:1046b00061fe204610bd00bff4730c0210b5044625
:1046c000fff7f0ff204614211af08af8204610bdab
:1046d00010b50446024b0360fff7e4ff204610bd0f
:1046e00008740c0210b50446fff7f2ff20461421af
:1046f0001af076f8204610bd10b50446074b214647
:1047000040f8043bfff784fc214604f118000bf04d
:1047100069fb00232046c4f8f43010bd1c740c0261
:1047200010b5044607f080fe042805d104f11800f6
:10473000bde810400bf038bd092016f085fa0028be
:10474000f4d0002010bd18300cf058bd0048704760
:1047500044cb0010024bc3f8f4000020704700bfa8
:1047600044cb001010b443690a4619680c6801462e
:10477000184623465df8044b184701464069036814
:104780005b681847fff754bff0b5354e074696f8fb
:104790002c300d46144687b0002b51d0706a23f0a0
:1047a00044fb00284cd104900c201af011f810b1f1
:1047b000c0e9015407702b4b029005932a4b1c2033
:1047c00004931af005f80446002832d0274b036002
:1047d0000023c360049b3bb1022202a90430984726
:1047e000059b2361049be36000252046204b2a465d
:1047f0002360012140f8145f23f020fc1d4b01a928
:104800002360f2692b46306b019423f06cfb014668
:1048100050b9706a08b123f035fb00224ff0ff3128
:10482000606923f01bfca569236820469b689847b4
:1048300000e0054602a8fef79dfd284607b0f0bd42
:104840000d4c84f8fc70d4f8f80028b18368c4f8e3
:10485000f830abf089fcf6e7c4f8f8500546ece711
:1048600070cc0010fd470002c945000280720c02a6
:1048700094720c02a8720c0244cb001003681878e2
:10488000d3e90112fff780bf73b5064614200d4629
:1048900019f09eff0446d0b10e4b03600023c360a5
:1048a000ab683bb10222294604309847eb6823618c
:1048b000ab68e360084b30462360336801945b6863
:1048c00001a9984718b9236820469b68984702b009
:1048d00070bd00bff4730c0208740c027fb5144e57
:1048e000044696f82c300d4693b1706a23f09dfa79
:1048f00070b9104b694603930f4b30460293cde9d4
:104900000054fff7c1ff6846fef734fd04b070bde8
:10491000d4f8f43023b90a20084a0949fcf740fbcf
:104920002846d4f8f43004b0bde87040184700bf02
:1049300044d20010354d000209460002bff50102c5
:10494000cc730c02f0b50c46d0f8f83085b0002bd3
:1049500000f0238299886288914200f010829b685f
:10496000f5e76388d32b00f2bf80c72b25d8322b05
:1049700000f0558100f2a280012b00f07181143b00
:104980009ab2152a68d9d0f8f430002b00f0a7802d
:10499000214605b0bde8f040fff7a0bf6ff4fa7202
:1049a00013442046052b00f2d581dfe813f0d60131
:1049b000d901dc01df01e201e501c83b0b2be2d8a4
:1049c00001a252f823f000bf414c0002494c000202
:1049d000074900020749000207490002074900028f
:1049e000074900020749000207490002074900027f
:1049f000514c0002594c0002463b142bc3d801a273
:104a000052f823f0a54b0002b14b0002c14b00024b
:104a1000c94b0002d14b0002d94b000207490002ea
:104a2000074900020749000207490002074900023e
:104a3000074900020749000207490002074900022e
:104a4000074900020749000207490002074900021e
:104a500007490002e94b0002152b94d801a252f835
:104a600023f000bf534b0002614b000207490002d4
:104a700007490002074900020749000207490002ee
:104a8000074900020749000207490002694b00027a
:104a9000714b0002794b0002814b0002894b0002ee
:104aa00007490002074900020749000207490002be
:104ab00007490002914b0002994b00025a2b07d87c
:104ac000452b99d83c2b7ff45eaf0023b44aa1e07c
:104ad000642b7ff458afa368002b00f0c98000233b
:104ae0006ff077011a4652e1b3f5967f00f0268108
:104af0004cd8e72b22d8db2b7ff645afdc3b0b2bca
:104b00003ff641af01a252f823f000bf614c000212
:104b1000694c0002714c0002794c00020749000206
:104b2000074900020749000207490002074900023d
:104b300007490002814c0002894c0002f03b9ab206
:104b40000d2a3ff620af0d2b3ff61daf01a252f804
:104b500023f000bf914c0002074900020749000200
:104b600007490002074900020749000207490002fd
:104b7000074900020749000207490002994c000258
:104b8000a14c0002ad4c0002b54c0002b3f5fd7f14
:104b90003ff6f9aeb3f5fa7fbff400afb3f5c87fc7
:104ba00000f0d4800cd840f22d12934200f0ca805d
:104bb000b3f5977f7ff4e7ae20460cf030fe0be0b4
:104bc00040f2911293427ff4deae20460cf050fd8d
:104bd00002e020460cf08afe002301461a46d6e089
:104be00020460cf0bdfef7e720460cf0d1fef3e7bf
:104bf00020460cf0e3feefe720460cf035ffebe734
:104c000020460cf0c5ffe7e720460cf0dfffe3e7a6
:104c10000023644a1946bae00023634afae70023f6
:104c2000624af7e700221146104602f05bfed3e726
:104c300000220121104602f0b3fe00231a46e9e7e4
:104c400020460cf057ffc7e720460cf065ffc3e78e
:104c500020460cf075ffbfe720460cf07fffbbe756
:104c600020460cf0d9ffb7e720460df0abfeb3e7c6
:104c700080264f4f60693246036821461b6898477b
:104c8000054640b1002211462046fff76bfd002388
:104c900029461a467be0e368014603906846cde961
:104ca00000730296fff780fc002205460028ead137
:104cb000039b9e4202d203eb1316dbe72361e6e778
:104cc00020460cf0dffe87e720460cf0f1fe83e77c
:104cd00020460cf0b0ff7fe720460cf0afff7be7eb
:104ce00020460cf0aeff77e720460cf0adff73e7ef
:104cf00020460cf0acff6fe720460cf0abff6be7f3
:104d000020460cf0e7fe67e720460cf0ebfe63e779
:104d100020460cf0a2ff5fe720460df06bfd5be73d
:104d2000204605b0bde8f0400df0debd20460df098
:104d30000bfe51e720460df00dfe4de720460cf02e
:104d400039fd49e720460cf065fd45e720460cf0ab
:104d50006ffc41e70df0bcf93ee70df07ff83be753
:104d60000df0e6f838e70df019f935e70df03af9ee
:104d700032e70df043f92fe70df014fb2ce79b7998
:104d8000022b7ff4eead00236ff081011a4620461e
:104d900005b0bde8f040fff74bbc90f8fc30efe702
:104da00089450002594500029d4500024545000223
:104db0006c730c02d0e90010fff790bd0148fff7bb
:104dc0009bbc00bf44cb00100023202200b58bb059
:104dd000cde90223054a01200092054902aafdf708
:104de000a1fc4ff0ff300bb05df804fb27740c0200
:104df00020740c02f0b5002420274ff4837605467a
:104e00000e4bc5b0009302aa23461e200c49cde9e3
:104e10000274fdf787fc3246214602a8abf0f1f997
:104e20003a4621462846abf0ecf923462246314665
:104e300002a804f087fc45b0f0bd00bf83740c02eb
:104e400020740c022de9f041ceb04ff48372044679
:104e50000e460ca80021abf0d4f900234ff4837167
:104e60001a460ca804f090fcb0f5837f2dd1bdf854
:104e70003030b3f5837f28d180213046149d15f062
:104e80003ffe854234d00025202780213046ddf8c2
:104e90005080cde9047515f033fe214bcde901803a
:104ea000009304aa2b4632201e49fdf73bfc9df8d7
:104eb0003530322001931c4b1a49009304aa2b462b
:104ec000cde90475fdf72efc0ae020210023174ae6
:104ed000cde9041300922820124904aafdf722fc10
:104ee0002046fff787ff4ff0ff304eb0bde8f0815e
:104ef0009df83530002bc6d00dad0fcd0fc495e811
:104f00000700002384e807002022cde90423084a93
:104f10001e200092034904aafdf704fce3e700bf4a
:104f2000cf740c0220740c02f4740c029b740c02fb
:104f300007750c0210b504460846802115f0e0fd07
:104f4000e061002010bd0000f0b50020b3b003f018
:104f50001dfb032015f078fe0446002837d05f4b78
:104f60001d888022002112a8abf04bf912a81ef078
:104f7000b3f99df84830012b16d920220023cde942
:104f80000a23574a2820009256490aaafdf7cafb6d
:104f90002cb1554b55491a6812a8abf00bf9544a7d
:104fa000136843f0040313609df8482020218ab160
:104fb000012a4ff0000360d001924e4acde90a1356
:104fc0000092282047490aaafdf7acfb1fe041f2f6
:104fd0003365c6e7ddf84a30cde90a12bdf88a101c
:104fe0001e200791d9b20691c3f307210591c3f39f
:104ff00007411b0e03930df14a03cde901233e4bfc
:1050000004910093374913460aaafdf78bfb4ff62c
:10501000fd71bdf88a20531e9bb28b4202d81cb191
:10502000aa4201d0adf88a5012a93448fff70aff0e
:10503000002c14bf11200620304a12a903f028f8d2
:105040000646002842d14ff4a06512a92b48fff76d
:1050500071ff09a8099629f037fd099cdcb1606849
:1050600048b10aa90a962af065f920b90a9b13b13a
:105070009d4228bf1d462468f0e7cde90a130df1d3
:105080004a01cde901211e4a1e20009215490aaab3
:10509000fdf748fbbbe7099829f042fdb5f5a06f85
:1050a000184f16d02023cde90a34174b803d0093ca
:1050b0000aaa23461e200b490195fdf733fb234620
:1050c0002a460094072138680ef061fe304633b05e
:1050d000f0bd234622460094f4e700bf6051001063
:1050e0003e750c0220740c02086d0c02ef6c0c0271
:1050f00010d10010d4750c026a750c0248cc001057
:10510000ac750c0218d1001010760c0203f03ebaf8
:1051100008b5002003f07cfac0b208bd0122014ba3
:105120001a70704744cc001013b50f4b04461b781f
:1051300023b102b0bde81040fff746be0b4b019112
:105140001b78002bf5d1fff7e3ff0028f1d1084bc6
:105150001b7803f0ff02002bebd12046019902b02f
:10516000bde8104003f0aeb975cf001076cf001047
:1051700044cc0010fff7d8bf13b50f4b04461b7883
:1051800023b102b0bde81040fff71ebe0b4b0191ea
:105190001b78002bf5d1fff7bbff0028f1d1084b9e
:1051a0001b7803f0ff02002bebd12046019902b0df
:1051b000bde8104003f0b2b975cf001076cf0010f3
:1051c00044cc0010fff7d8bf08b5002003f00afa5e
:1051d00010f1780f08bf002008bd002003f014baba
:1051e000f0b5022806460d4614468db005d00a28b3
:1051f00034d01f4c20460db0f0bd202000231d4fa1
:10520000cde904033a68cde901211b4a009201204f
:105210001a4904aafdf786fa3d6000f0a7fd10b90f
:1052200014f00104e6d0164b00245b78b342e1d1c0
:105230002023cde90434134b04aa00930120234614
:105240000e49fdf76ffa082202232946cde904230f
:105250002046234604aa00f07ffecbe7202100234e
:10526000094fcde904133a68cde90125074acde796
:10527000f2feffff5851001038760c0220740c0229
:1052800048cc00109b760c025c51001069760c0231
:1052900019b1022803d00a2806d004487047044bed
:1052a0001b6800200b607047024bf9e7f2feffff1e
:1052b000585100105c51001003689b6818470eb4e9
:1052c00003b503ab53f8042b002101930ef0a2f8b1
:1052d00002b05df804eb03b070472de9f0410646db
:1052e0000d4690461df0e3f807461df0e0f8c01ba0
:1052f00040450ed83468236820461b69984700282b
:10530000f3d0236820465b69984728700020bde8e9
:10531000f0814ff0ff30fae72de9f04f16461a46bc
:10532000002385b00f4633600df10f0101928246d4
:10533000fff7d3ff019a044628b14ff0ff3420460f
:1053400005b0bde8f08f9df80f50182d13d008d888
:10535000022d20d0042df2d0012deed14ff0800887
:105360001be005f0df03412b35d0202d14bf4ff09b
:10537000ff340224e3e750460df10f01fff7adffc4
:1053800004460028d9d19df80f30182bd5d14ff005
:10539000ff333360d3e74ff48068b94609f8015b07
:1053a000012508f1040b5d450cd849465046019291
:1053b000fff793ff09f101090028bed10135019ad9
:1053c000adb2f0e7bb787a78db43dbb29a42b4d176
:1053d000c6f80080b3e70124b1e738b50d460021d7
:1053e00002f58070033313f8014b2cb1b1f5807fc7
:1053f00002d054540131f6e700245454ff32195db1
:10540000202905d0102c03d0013402f8011ff6e743
:1054100000210a220155acf0b1fe4ff48063e86030
:105420002b8138bdf8b51d46531c04460cd08ab1fb
:10543000d0f818644f78f3b29f4213d0006815215a
:10544000fff73aff012004e000680621fff734ff70
:105450000020f8bd00680621fff72eff0120c4f8e8
:105460001404f6e786bbcb7803b30b46069a2946ad
:10547000fff7b3ff324631462846fef7f9fb50b13d
:1054800018212068fff718ff20681821fff714ff84
:105490004ff0ff30dde72b6906216b602068fff7d6
:1054a0000bff43212068fff707ff04e00123c0f84a
:1054b0001434c0f810340120d4f81834c4f820048f
:1054c0000133c4f81834c4e72a8128460022033186
:1054d000fef740fc50b118212068fff7edfe206870
:1054e0001821fff7e9fe6ff00100b2e76b682a8927
:1054f000062113446b60d5e72de9ff4117460446aa
:1055000000250e464ff4887200213846aaf079fe35
:1055100004f10808c4f81054c4f81c54c4f820540a
:10552000c4f81854c4f8145441462046636803aaca
:10553000fff7f2fe012810d0022819d030bbc4f8c2
:105540001c04334641462046039a0097fff76aff42
:10555000002811dc04b0bde8f08118212068fff7b5
:10556000abfe20681821fff7a7fe6ff00200f1e7fd
:1055700006212068fff7a0fed4f81434002bd3d006
:10558000d4f81034002bcbd0f068e3e7d4f8203403
:10559000002b08dbd4f81c34432101332068c4f805
:1055a0001c34fff789fed4f81c34052be4dd1821e8
:1055b0002068fff781fe20681821fff77dfe00209c
:1055c000c8e70000f0b50446c7b040f224400f46db
:1055d00019f0fef8054618b141f2883304604360c3
:1055e0003946284602aafff787ff061e48dd00223b
:1055f00001213846fef764fb021e31db06212868d4
:10560000fff75afe20462a490df0dcfe20462949c4
:105610000df0c5fe204602a90df0c1fe2046264928
:105620000df0d0fe204625490df0b9fe0a22314684
:1056300020460df0d1fe224920460df0c3fe23681e
:105640002046db6998474ff47a7019f0f6ff012481
:10565000284640f2244119f0c3f8204647b0f0bd77
:10566000182128680192fff727fe18212868fff704
:1056700023fe2046019a1349fff721fe0024e7e7a5
:1056800018212868fff718fe18212868fff714fe74
:10569000721c04d10c4920460df094feeee7b31cb9
:1056a00001d10a49f7e703360cbf09490949f2e776
:1056b000bf760c02df760c0247420d02e6760c0242
:1056c0005aa10c02ed760c0205770c023c770c0215
:1056d00052770c0263770c02012009f05dbc08b51b
:1056e0000023c269006b22f0fefbb0fa80f0400993
:1056f00008bd70b505460e468069002122f0befb4c
:10570000002304461a463146286b22f00dfc18b1de
:10571000201e18bf012070bd0120fce708b5002342
:105720008269006b22f000fcb0fa80f0400908bded
:1057300038b50546fff7d3ff044620b1686a10b1bb
:10574000002122f09ffb204638bd012a02d10160d2
:1057500000207047022a04bf0b680360f8e7036863
:1057600018470000014b186822f01dbcb8cc00108f
:1057700010b5044c236813b9204622f030fc206891
:1057800010bd00bfa4cc001010b50a4cd4e88f3f68
:10579000db070cd420461bf0b9f840b1064822f0d4
:1057a000f8fb20461bf0ecf80448aaf0dcfa0248ab
:1057b00010bd00bf6ccc0010b8cc0010e556000244
:1057c000014b1860704700bf68cc001038b500234b
:1057d00083608b6804460d462bb102229847eb6824
:1057e000e360ab68a360204638bd000030b5214bb4
:1057f0008db00093204b69460393204b04a802937d
:10580000fff7e4ff4ff4a0526423cde908236ff0c3
:1058100000430a9332231a4cadf82c300223204661
:1058200000258df82e30174b04a940f8043bfff7f4
:10583000cdff089b04f128006361099b6562a361a9
:105840000a9be361bdf82c3023849df82e3084f848
:10585000223022f09efb0c4b04a8236084f82c50cd
:105860002563fdf787fd6846fdf784fd074b9d60c6
:105870000db030bd59560002df560002cb56000273
:1058800070cc001088770c0298770c02a8cc00101e
:1058900010b5c36804460bb9a9f00cff03690430c6
:1058a00098470021a0616069bde8104022f0f6bb76
:1058b00010b5c36804460bb9a9f0fcfe03690430b7
:1058c0009847002120766069bde8104022f0e6bbd1
:1058d00008b504f057fc002008bd000007b51346ca
:1058e000002200920a460146054800680ef085fa3b
:1058f000002818bf6ff0ef0003b05df804fb00bf95
:1059000018d10010012a70b5054603d10b68036059
:10591000002070bd022a08d0032af9d100680028af
:10592000f6d0102118f05cfff2e710200e6818f096
:105930004fff044618b196e80f0084e80f002c6072
:10594000e6e7012a70b5054603d10b680360002025
:1059500070bd022a08d0032af9d100680028f6d0c9
:10596000102118f03dfff2e710200e6818f030ff0c
:10597000044618b196e80f0084e80f002c60e6e7b3
:10598000012a08bf016000207047012a38b504468b
:1059900002d10b68236003e0022a03d0032a0dd052
:1059a000002038bd0c200d6818f012ff03460028b7
:1059b000f0d095e8070083e80700ebe700680028cf
:1059c000eed00c2118f00cffeae7012a70b505466d
:1059d00003d10b680360002070bd022a08d0032a9f
:1059e000f9d100680028f6d0102118f0f9fef2e78e
:1059f00010200e6818f0ecfe044618b196e80f006f
:105a000084e80f002c60e6e7012af8b5064603d1ca
:105a10000b6803600020f8bd022a08d0032af9d1e0
:105a200000680028f6d0142118f0dafef2e71420fe
:105a30000c6818f0cdfe074620b105460fcc0fc507
:105a400023682b603760e5e7012af8b5064603d1e5
:105a50000b6803600020f8bd022a08d0032af9d1a0
:105a600000680028f6d0142118f0bafef2e71420de
:105a70000c6818f0adfe074620b105460fcc0fc5e7
:105a800023682b603760e5e7012a034602d10160f5
:105a900000207047022a04bfd1e90001c3e90001d8
:105aa000f6e7012a02d1016000207047022a04bff4
:105ab0000b680360f8e7012a08bf01600020704707
:105ac000012a02d1016000207047022a04bf0b683e
:105ad0000360f8e7012af8b5064603d10b680360b6
:105ae0000020f8bd022a08d0032af9d10068002856
:105af000f6d0182118f074fef2e718200c6818f0a0
:105b000067fe074630b105460fcc0fc594e8030089
:105b100085e803003760e3e7012a034602d101600c
:105b200000207047022a04bfd1e90001c3e9000147
:105b3000f6e700224ff0ff3122f090ba00224ff03a
:105b4000ff3122f08bba000010b50446034b40f839
:105b5000043bfdf70ffc204610bd00bfa8770c02e8
:105b600010b50446fff7f0ff2046142118f038fe68
:105b7000204610bd10b5074b04460360406918b1bc
:105b800022f067fa002363612046fff7ddff20461d
:105b900010bd00bfbc770c0210b50446fff7eaff4a
:105ba0002046182118f01cfe204610bd10b50446f2
:105bb000024b0360fff7deff204610bdd0770c02da
:105bc00010b50446fff7f2ff20461c2118f008fe2e
:105bd000204610bd10b50446034b40f8043bfdf7ca
:105be000c9fb204610bd00bfe4770c0210b5044687
:105bf000fff7f0ff2046142118f0f2fd204610bdfb
:105c000010b5074b04460360406918b122f021fa31
:105c1000002363612046fff7ddff204610bd00bf73
:105c2000f8770c0210b50446fff7eaff204618216a
:105c300018f0d6fd204610bd10b50446024b036097
:105c4000fff7deff204610bd0c780c0210b50446ad
:105c5000fff7f2ff20461c2118f0c2fd204610bdc0
:105c6000406a22f0e2b8000010b404460748134628
:105c700000682ab1214600235df8044b0df0a2bf55
:105c80000a4621465df8044b0df0a3bf18d1001061
:105c9000f0b52e4e044696f82c300d4687b0002bfa
:105ca0004ad03046fff7dcff0746002844d1284b96
:105cb0001c200593274bcde90245049318f088fd7d
:105cc0000446002831d0244bc7600360049b3bb1dd
:105cd000022202a904309847059b2361049be360dc
:105ce000002520461d4b2a462360012140f8145f01
:105cf00022f0a4f91a4b01a92360f2692b46306bfc
:105d0000019422f0f0f8014650b9706a08b122f00f
:105d1000b9f800224ff0ff31606922f09ff9a569c0
:105d2000236820469b68984700e0054602a8fdf7d7
:105d300021fb284607b0f0bd04f090fa2a46214620
:105d400007b0bde8f0400ef08cb800bf70cc00107a
:105d5000e55c0002095a0002e4770c02f8770c02b5
:105d60000c780c02d0e90001fff792bf054b1b78bd
:105d700003f0ff0023b1044b1878003818bf01204e
:105d8000704700bf36cb001033cb001008b5094870
:105d9000fff766ff68b1002006f052fb20b1bde8b6
:105da0000840044801f070bf0120bde8084009f038
:105db000f3b808bd44d20010002190b583b004466a
:105dc00000af084618f040f9c31d23f00703adeb00
:105dd000030d01467860684618f036f920467a6867
:105de000694604f0b9ff20460c37bd4690bd00005f
:105df000014b18600020704714d100107fb51d4d75
:105e0000044695f82c300e46b3b12846fff728ff1c
:105e100090b9194b69460393184b2846cde90046c3
:105e20000293fdf79ffb044688b905466846fdf7d7
:105e3000a1fa284604b070bd94b1631c13d021466a
:105e40000f4802f0dff80e4802f0c9f80be0406995
:105e5000fff774fe236820469b68a5699847e5e72d
:105e6000074802f0b7f8064804b0bde8704002f0f9
:105e70000db900bf70cc0010055e0002995a0002f7
:105e8000bccc0010d0e90001fff7b8bf2de9ff41fd
:105e9000014640b368460df0c1f9009e9df80940e7
:105ea000ddf804809df80850fff760ff00b304f0b0
:105eb0007fff4ff00103d0e8cf7fc0e8423f002ac8
:105ec000f9d1ffb2002ff6d1c660c0f81080057579
:105ed00044750023c0e88f3f06f07afa002420467c
:105ee00004b0bde8f0810546804604460646dbe77f
:105ef00006f06efa16f0040625d0002cefd0134cf5
:105f000094f82c3013b904f03df9e7e72046fff789
:105f1000a7fe0028f7d10e4b694603930d4b204690
:105f20000293fdf71ffb054658b14069fff706fed7
:105f30002b6828469b68ac6998476846fdf71afab3
:105f4000cde70446f9e73446c9e700bf70cc00103e
:105f50005158000201590002f0b504462c481f4672
:105f600090f82c300e46154687b0dbb1fff778fe6f
:105f7000c0b90490102018f02bfc18b1c0e90046fd
:105f8000c0e90257234b02900593234b204802a9f6
:105f90000493fdf7e7fa044660b9054602a8fdf749
:105fa000e9f904e0012c25d9022c0cd01b4d284620
:105fb00007b0f0bd4069fff7c1fd236820469b682c
:105fc000a5699847eae7294602a80df027f904f0e9
:105fd000effe029b0025d90744bf9df810200272f6
:105fe0009a0744bf039a42605b0744bf9df8113093
:105ff0004372dce70a4800972b4632462146006888
:106000000df0c5fe07b0bde8f0400df0f7bc00bfd5
:1060100070cc0010a55f0002c3580002f2feffff23
:1060200018d100100068d0e90223d0e90001fff781
:1060300093bf000030b5044628481d4690f82c3028
:1060400087b00bb3cde90012fff70afedde90012bd
:10605000d0b90490102018f0bbfb28b1019a009928
:10606000c0e90225046041601d4b029005931d4b61
:106070001a4802a90493fdf775fa044670b905465b
:1060800002a8fdf777f906e0042c19d0052c1cd0e6
:10609000032c0cd0144d284607b030bd4069fff7e3
:1060a0004dfd236820469b68a5699847e8e70f4b9c
:1060b0001b787bb1082007b0bde83040fff70ebc6d
:1060c0000a4b1b7833b10920f5e7084b1b780bb15d
:1060d0000a20f0e76ff0d105dde700bf70cc0010bb
:1060e0007160000285580002f2feffff33cb001002
:1060f0000068d0e90223d0e90001fff79bbf000050
:1061000073b506461c200d4618f062fb044628b302
:10611000144b03600023c360ab683bb102222946e5
:1061200004309847eb682361ab68e36000222046a7
:106130000d4b0121236040f8142f21f07fff0b4b02
:1061400030462360336801945b6801a9984705468f
:1061500020b9236820469b6898472c46204602b009
:1061600070bd00bfa8770c02bc770c02d0770c0280
:106170002de9f04305462e48994690f82c3087b01b
:106180000e4690460e9f2bb3fff76afd10bb04909e
:10619000182018f01dfb40b10f9bc0e90056c0f855
:1061a000088080f80c9007614361224b02900593b0
:1061b000214b1f4802a90493fff7a2ff054670bbbd
:1061c000044602a804f00104fdf7d4f8204607b005
:1061d000bde8f083b9f1000918bf4ff00109cde91e
:1061e000007816484b463246294600680df0f8fc08
:1061f00004460028ead0fff7b9fd06460028e5d09e
:1062000006f012f9012803d10d4b1b78002bddd0cd
:106210003a4649462846fff727fd3446d6e7406907
:10622000fff787fc2b6828469b682c7e9847c8e7b9
:1062300070cc0010c5610002555a000218d1001040
:10624000c4d2001007b500684269037b019202695d
:106250000092d0e901120068fff78aff03b05df8f1
:1062600004fb000030b5174c054694f82c3085b07f
:1062700003b32046fff7f4fce0b9134b2046039329
:10628000124b694600950293fff73aff044678b136
:106290004069fff74efc236820469b68257e98479f
:1062a000684605f00105fdf765f8284605b030bde4
:1062b0000546f5e703f0d2ff002105b0bde8304008
:1062c0000df0ccbd70cc001051620002235a0002c8
:1062d0000068fff7c7bf0000f0b5044622481f461c
:1062e00090f82c300d46164685b0fbb1fff7b8fc90
:1062f000e0b90290102018f06bfa18b1c0e900451f
:106300000672c760194b00900393194b69461648f3
:106310000293fff7f5fe054658b90446684604f0b7
:106320000104fdf727f8204605b0f0bd55b900245b
:1063300015e04069fff7fdfb2b6828469b682c7e23
:106340009847ebe75cb12046faf71cfd4028eed8f1
:1063500020463b463246294603f0a6ff0446003c51
:1063600018bf0124dfe700bf70cc0010f562000207
:106370004b5900020068c368027ad0e90001fff7b8
:10638000abbf00007fb5054622480c4690f82c3084
:106390001646f3b1fff764fcd8b902900c2018f050
:1063a00017fa10b1c0e9005486601b4b00900393ac
:1063b0001a4b694617480293fff7a2fe044680b9bc
:1063c0000546684605f00105fcf7d4ff284604b0f1
:1063d00070bd7db93146204604b0bde8704004f080
:1063e0001cb94069fff7a5fb236820469b68257e02
:1063f0009847e6e710230021adf80030084b6846c7
:106400000195cde90234adf8021004f006f9054615
:10641000dce700bf70cc0010a56300020b5900023e
:1064200059a4000203681868d3e90112fff7aabf54
:1064300030b5114c054694f82c3085b08bb1204610
:10644000fff70efc68b90d4b694603930c4b2046d1
:1064500002930095fef718fa6846fcf78bff05b02b
:1064600030bd0022074b114618680df07efc05b0c8
:10647000bde8304003f0f8bc70cc001009640002a5
:10648000415a000218d100100068fff7d1bf000088
:106490001fb50e4c94f82c3083b12046fff7e0fb7b
:1064a00060b90b4b694603930a4b20460293fef7f3
:1064b000ebf96846fcf75eff04b010bd0021064b07
:1064c000186804b0bde810400df024bc70cc00107a
:1064d0006b640002375a000218d1001008b5fff7ac
:1064e000d7ffbde80840fff741bcfff7d1bf000070
:1064f0002de9f04705463d4886b013f0100f1c46c5
:106500000e461746ddf8389090f82c300df108084b
:1065100022d003f0ff0a002b46d0fff7a1fb002892
:1065200042d10490142018f053f928b1c0e9005664
:10653000c0e90274c0f810902d4b029005932d4bca
:1065400041462a480493fef79ff94046fcf712ffa4
:10655000504606b0bde8f08733b3fff781fb18bba8
:106560000490142018f034f928b1c0e90056c0e9ad
:106570000274c0f81090204b029005931f4b4146c7
:106580001a480493fff7bcfd044658b14069fff771
:10659000d0fa236820469b6894f818a098470af020
:1065a000010ad2e78246fae70023cde903330c2340
:1065b0000293b9f1000f05d0d9f804300393d9f84c
:1065c0000830049314f0010f14bf4522652224f013
:1065d000010313430a480093cdf804803b4632463a
:1065e000294600680df090fa8246b1e770cc0010a1
:1065f00085650002c95900029f65000289590002a1
:1066000018d1001007b5006803690093d0e9022390
:10661000d0e90001fff76cff03b05df804fb07b59c
:10662000006803690093d0e90223d0e90001fff775
:106630005fff03b05df804fb0021014801f06cbc72
:10664000bccc001030b5cc1c2a3114f8035c0334e8
:1066500005f00f0205f0f00342ea021243ea1515b5
:10666000130243ea0543436014f8052c02f0f005d9
:1066700045ea12152b4302f00f024360827214f8b0
:10668000043ca14203eb830303eb83034fea430380
:1066900020f8083fd9d130bd002138b5044608465e
:1066a000fcf768f91c2500232046094c05fb034232
:1066b000416801331161817a0d2b517330f8081f45
:1066c0009182f3d10021bde838400120fcf752b996
:1066d000cccc00100c2808b50ad81c22054b02fbb4
:1066e0000030002201730121fcf700f9002008bdf1
:1066f0000120fce7cccc001011f0040238b50cd01e
:1067000000240b4d0022284611460134fcf7eef818
:106710000d2c05f11c05f5d138bd0c28fcd81c2426
:10672000034b114604fb0030bde83840fcf7deb8ef
:10673000cccc00100c289fbf1c22044b02fb003065
:10674000807b94bf00f0010000207047cccc00108b
:10675000f0b58a0705460c469db01cd50125682278
:10676000002102a8a9f04dfd214901a80195fff7dc
:1067700069ff01a8fff790ffe30709d5ff232a4629
:1067800040f6af618df803300df1030019f07bf88e
:1067900000201db0f0bd0368012b27d1fff77cff5f
:1067a00014f00100f5d001a9084632262b466835c1
:1067b0005a68c2f30357c2f3033444ea07144c7017
:1067c0009c7a02f0f00204f00f0422438a7033f83e
:1067d000082fb2fbf6f29d4201f8032fe8d1012306
:1067e000402240f6af618df80430cfe70120d0e7ba
:1067f00018780c0270b50268012a18d111f0020154
:1068000005d00c49fff71eff0021084670bd0b465e
:106810001c26094d06fb0352146901334460547b66
:106820000d2b8472928a20f8082ff3d1ede7012115
:10683000ebe700bf18780c02cccc00100c289dbff1
:106840001c22024b02fb003000207047cccc001011
:10685000022803d0032807d000207047142909d04c
:106860000adc4ff4fa707047142907d009dc4ff4a2
:10687000fa507047c8207047642070474ff47a6020
:1068800070474ff47a7070470021224a30b50b46aa
:1068900015461c24adb004fb015001310d29c2e99d
:1068a00000439360037302f11c024373837303611b
:1068b0008382f0d16822002112a8a9f0a2fc012352
:1068c000402240f6af6001a9119318f0a7ff18b954
:1068d0009df80430012b1ad00f4b01aa03f12005bb
:1068e000144618685968083303c4ab422246f7d1ee
:1068f000998818689b79a1802060a37101a911a8cb
:10690000fff7a0fe11a8fff7c7fe2db030bd0df1b7
:106910000501f4e7cccc001024610c022de9f04f06
:106920004ff0180a91469b460e46154985b0d1e9ad
:10693000004103900afb014adde90e780c34a4f112
:106940000c018a4511d054e90301039b31401840e2
:1069500050ea010307d000945b464a46314603984b
:1069600054f8045ca8471834e9e72fb140463b4689
:1069700005b0bde8f04f184705b0bde8f08f00bf87
:1069800038ce001030b5d1e90054d0e900232a40b8
:10699000234013430cd0836813b18a68934207d114
:1069a000c3683bb158680b69c31a5842584130bd9f
:1069b0000020fce70120fae7704710b504462821c3
:1069c00017f00eff204610bd012af8b5064603d188
:1069d0000b6803600020f8bd022a08d0032af9d111
:1069e00000680028f6d0182117f0fafef2e7182008
:1069f0000c6817f0edfe074630b105460fcc0fc509
:106a000094e8030085e803003760e3e72de9f043ed
:106a1000dff8d88093b08146d8f800000e461546be
:106a20001c4621f0ebfa13f075fe00230746cde972
:106a30000096cde90333029505933cb16288214667
:106a40000c2a28bf0c2203a8a9f0b4fb6d4606aca3
:106a50000fcd0fc495e803000cae0df1180c84e8bf
:106a60000300bce80f001f4d0fc694e80300d5f8e3
:106a70000490ab6886e8030099451adb09f101042c
:106a8000002c286810dd18216143aaf03bfb70b987
:106a9000154c384613f042fed8f8000021f0bdfa3c
:106aa000204613b0bde8f083a9f05efb002028600b
:106ab000ac6018236a6803fb09f95a432c68a2ebff
:106ac00009024c442146e0180caea9f080fb0fce21
:106ad0000fc496e803006b6884e8030001330024c8
:106ae0006b60d6e738ce0010fcfeffff44ce0010ee
:106af0002de9f04f8fb00193574b834618688946b4
:106b0000164621f07bfa13f005fe1822534fcde90b
:106b100002b9d7e90045019b554304960deb020ce1
:106b200005930df108090aae824699e80f008ce83a
:106b30000f0086e80f004a4b04eb0508ed105d439b
:106b4000ad10002d1ddd21463046fff71bff30bb89
:106b5000a346183421463046fff714fff8b90bf16d
:106b6000300421463046fff70dffc0b90bf1480451
:106b700021463046fff706ff88b90bf16004013d5e
:106b8000dfe7a8eb0403302b27d0482b1ed0182baf
:106b90004cd121463046fff7f5fe002846d0a045ef
:106ba00045d004f11806b04541d031464846fff7bc
:106bb000e9fe48b92546b446bce80f000fc59ce87d
:106bc000030085e8030018341836ece72146304608
:106bd000fff7d8fe0028e2d1183421463046fff7ef
:106be000d1fe0028dbd11834d3e71d48e31adb10af
:106bf000151b00fb03f304d4ed10454358198142e3
:106c000000dacd1a182101fb05412046521aa9f0dd
:106c1000defa7b685b1b7b60504613f07ffd0e4bfa
:106c200018680fb0bde8f04f21f0f7b944461826b8
:106c30007a683b6806fb02339c42edd02546d7e9d3
:106c4000003106fb01329542cfd0286910b16b6943
:106c500003b198471835f2e744ce001038ce001043
:106c6000abaaaaaa2de9f0471f461e4b164693f879
:106c70002c2086b00546dde90e890c46eab1586a3b
:106c800021f0d3f8c8b90490182017f0a1fd28b15d
:106c9000c0e90054c0e90267c0e90489124b0290c0
:106ca0000593124b02a90f480493fdf7edfd02a8ce
:106cb000fcf760fb06b0bde8f087dff834a0daf837
:106cc000000021f09bf928463b4632462146cde99b
:106cd0000089fff723fedaf8000006b0bde8f047b0
:106ce00021f09bb944d20010396d000249690002bd
:106cf00044ce00102de9f047dff860c00746dde91b
:106d00000898dcf804c00e46ccf3080c15461c4667
:106d1000bcf1000f16d00021282008f0ddf9014653
:106d2000a0b1002383600a4bc0e904760360c0e988
:106d30000654c0e90898074b4360bde8f047064891
:106d400000f0cebfbde8f047fff78cbfbde8f0878d
:106d500048780c02136d0002f4d6001000ed00e03c
:106d600010b4039ce40703d55df8044bfff7d6bdd0
:106d70005df8044bfff7bebf002307b502460021b4
:106d80004ff48040cde90033fff7b4ff03b05df866
:106d900004fb13b50446436a0193036a0093d0e9e8
:106da0000623d0e90401fff75dff0021204602b071
:106db000bde8104008f0a2b907b501684b6901931e
:106dc0000b690093d1e90223d1e90001fff74affe3
:106dd00003b05df804fb00000023044a0448c2e944
:106de00000339360036021f0fab800bf38ce001082
:106df00044ce0010002210b51146044600f05efba0
:106e0000024638b1002320461a46194600f018fd04
:106e1000012010bd0146204600f09ffb0028f8d05d
:106e2000f0e7002337b5062200930321012007f085
:106e3000dffe0320fff7deff05460420fff7daff41
:106e40000023044625b11a461946032000f032fefd
:106e500044b1002304201a46194603b0bde830406f
:106e600000f028be03b030bd10b401291346c0683d
:106e700008d102685968146803f1080223465df8d6
:106e8000044b18476ff077005df8044b704738b536
:106e9000144619b904220846226038bd1368032b32
:106ea00007d903685b6898470028f6d1042323605c
:106eb000f3e76ff0bd00f0e7836900200b607047d7
:106ec00038b5144619b904220846226038bd136843
:106ed000032b07d903685b6898470028f6d1042381
:106ee0002360f3e76ff0bd00f0e7836900200b60db
:106ef00070471830036800200b6070471830036833
:106f000000200b60704738b505460c4613f002fcb4
:106f1000ab69236013f002fc002038bd70b5104e41
:106f20008ab01bf0c4fa736a1bb1c01ab0f57a7f3d
:106f300012d30c4901a80cf01df8029b0a4c736097
:106f4000039b04adb3600fcd0fc495e8030084e844
:106f500003001bf0acfa706201480ab070bd00bfbc
:106f60004ccf001044d7001058cf001038b50d4654
:106f7000fff7d4ff044688b103685b699847b5ee14
:106f8000c00af1ee10fa0cd4236820469b6998479a
:106f9000beeec80a002085ed000a38bd6ff077000c
:106fa000fbe76ff06300f8e738b50d46fff7b6ff73
:106fb000044688b10368db689847b5eec00af1ee75
:106fc00010fa0cd4236820461b699847beeec80a05
:106fd000002085ed000a38bd6ff07700fbe76ff009
:106fe0006300f8e738b50d46fff798ff0446b8b1df
:106ff00003685b699847b5eec00af1ee10fa12d447
:10700000236820465b699847dfed087a20ee270a5f
:10701000bceec00a10ee103a00209bb22b6038bdc7
:107020006ff07700fbe76ff06300f8e70000804344
:1070300038b50d46fff772ff0446b8b10368db6848
:107040009847b5eec00af1ee10fa12d42368204634
:10705000db689847dfed087a20ee270abceec00a0d
:1070600010ee103a00209bb22b6038bd6ff0770015
:10707000fbe76ff06300f8e70000804310b50c46b3
:10708000fff74cff28b103689b68984720600020f9
:1070900010bd6ff07700fbe70a4b10b503601423b7
:1070a0004360012304464381074bc0e9032001816b
:1070b000436100210430fbf7b3fd044b20462360fd
:1070c00010bd00bfc4780c02e96d0002d0780c023c
:1070d0000048704748ce00102de9f0413d4c082192
:1070e00020463d4a0025fff7d7ff1c2114273b4bc4
:1070f0003b4a23606018a561fff7ceff394bdff8ec
:107100005081e361384b394ec4e90f73384b29463f
:10711000636404f13803a3646563c4f83880e664eb
:1071200004f13c00fbf77cfd324b2946a363324b54
:10713000c4e91458e365314ba765236604f1540391
:10714000c4e9193604f15800fbf76afd2c4b0921fc
:1071500063652c4ae56604f17000fff79dff2a4b3a
:10716000c4f888502367294c294b18222360022336
:107170002946c4e9013504f10c00a9f042f8656222
:10718000244c21212046244afff786ff234b25214a
:107190002360234c234a2046fff77eff224b222107
:1071a0002360224c224a2046fff776ff214b232101
:1071b0002360214c214a2046fff76eff204b2421fb
:1071c0002360204c204a2046fff766ff1f4b2360b8
:1071d000bde8f08148ce001050780c02e0780c0237
:1071e00059780c02f0780c020c000200e96d0002e4
:1071f00066780c0200790c021b00020070780c0209
:1072000010790c027c780c0220790c024ccf001013
:10721000b4910c02ecce001084780c0240790c0280
:107220001ccf00108f780c0260790c02d4ce0010b5
:107230009b780c0230790c0204cf0010a7780c0266
:1072400050790c0234cf0010b4780c0270790c0223
:10725000c4780c0230b5134b8db01d78e5b1002415
:10726000042022460df10f011c708df80f40fcf731
:10727000d1fb9df80f3093b12023cde904340a4ba4
:107280001e200a49009304aa2346fbf74bfa224624
:1072900021460420fcf7a6fb28460db030bd1d4654
:1072a000fae700bf6251001078790c0220740c02da
:1072b000012a38b5044602d10b68236003e0022a94
:1072c00003d0032a0dd0002038bd0c200d6817f024
:1072d0007ffa03460028f0d095e8070083e807000e
:1072e000ebe700680028eed00c2117f079faeae706
:1072f000012a02d1016000207047022a04bf0b68f6
:107300000360f8e7012a034602d1016000207047bc
:10731000022a04bfd1e90001c3e90001f6e7012a0e
:1073200002d1016000207047022a04bf0b6803608d
:10733000f8e7012a034602d1016000207047022ac3
:1073400004bfd1e90001c3e90001f6e7012a02d137
:10735000016000207047022a04bf0b680360f8e751
:1073600007b5016811f00101019107d105f020fd79
:10737000019903b05df804eb05f0e8bd05f018fdd8
:1073800003b05df804eb05f043be000007b50068ec
:1073900050b101a9c0b227f009fc28b904f086f861
:1073a0000122019904f052fe04f080f804f050fc30
:1073b0000122044b1a700022034b1a7003b05df8cf
:1073c00004fb00bf77cf001076cf001030b50d461c
:1073d000044685b010bb03460a46009003210120f5
:1073e00007f006fc194b1c700122194bc3e88f2fc4
:1073f00004f05cf80722214604f060ff04f056f820
:10740000294604f09cfcf0b904f050f804f0eafac4
:10741000022818d0012018f010f9f5e703a9c0b22e
:1074200027f0c4fb48b904f041f82a46039904f058
:1074300045ff04f03bf804f086fa04f037f804f056
:1074400030fa0028dad005b030bd00bf77cf001089
:1074500078cf001001790068fff7b8bf08b504f0d5
:1074600025f804f0dbfb04f021f8bde80840072212
:10747000002104f023bf0000042810b519d10e4ce0
:107480007e2200212046a8f0bcfe4ff0ff33c4f856
:107490007e30a4f88230c4f85730a4f85b306ff027
:1074a0007b03237000232046637015f034fa2046d6
:1074b00010bd0020fce700bf79cf001073b50d466a
:1074c000d8b911f0ff0506d103f0f0ff02b0bde816
:1074d000704004f030ba012d06d103f0e7ff02b08e
:1074e000bde8704004f014b8022d34d103f0deff83
:1074f00002b0bde8704004f012b801a9c0b227f094
:1075000055fb30bb03f0d2ff019904f08ff904461c
:10751000f8b103f0cbff019904f0d4f9064603f06b
:10752000c5ff019904f0d6f915f0ff0506d1022e2a
:1075300001d002280dd1204602b070bd012d04d12a
:10754000022e14bf00240124f5e7022d01d10228e8
:10755000f7e70024efe70446ede713b530b903f091
:10756000a5ff02b0bde8104004f0dbb96946c0b227
:1075700027f01cfb68b9019001a9009827f0dbfbfc
:10758000002806db019800f04100012801d102b07b
:1075900010bd0020fbe70020704713b5044638b942
:1075a00003f084ff214602b0bde8104004f021b989
:1075b00001a9c0b227f0fafa30b903f077ff0199b8
:1075c00004f017f902b010bd0020fbe713b5044624
:1075d00038b903f06bff214602b0bde8104004f05b
:1075e00016b901a9c0b227f0e1fa30b903f05eff85
:1075f000019904f00cf902b010bd0120fbe713b5ae
:10760000044638b903f052ff214602b0bde81040ed
:1076100003f0eebf01a9c0b227f0c8fa30b903f0f9
:1076200045ff019903f0e4ff02b010bd0020fbe725
:1076300070470020704708b505f0bafbbde8084068
:1076400005f0babb07b50c4b5b68cde90012c3f37c
:10765000080343b905f0acfbdde9001203b05df8a7
:1076600004eb05f00dbd05f0a3fbdde9001203b04e
:107670005df804eb05f0cabb00ed00e010b504288e
:1076800086b011d11046059215f0a6f8059b044668
:1076900038b9cde901000090012210200021fff748
:1076a0005ffb204606b010bd004cfae7f2feffff7c
:1076b00013b5044648b903f0f9fe214603f0c4ffb0
:1076c000b0fa80f0400902b010bd01a9c0b227f0a5
:1076d0006dfa40b903f0eafe019903f0b5ff0038f6
:1076e00018bf0120efe70020ede74ff0ff307047b3
:1076f0004ff0ff30704708b505f05afbbde8084071
:1077000005f05ebb704700007fb5104e044696f84a
:107710002c300d4693b1706a20f087fb70b90c4b8a
:10772000694603930b4b30460293cde90045fdf7c4
:10773000abf86846fbf71efe04b070bd2046e9b208
:1077400004b0bde87040fff741be00bf70cc001030
:10775000d5730002b372000237b504460068a8b9b9
:1077600000220121174b10461a70174b1970032184
:10777000fff7caff03f09afe04f078fa6368db07ac
:107780001dd503b0bde8304004f022be0022032125
:10779000fff7baff207801a927f008fa054628b9b3
:1077a00003f084fe2a46019904f050fc2368002b64
:1077b000d6d003f07bfe04f074f80028d0d003b0dc
:1077c00030bd00bf77cf001076cf001030b5174d19
:1077d000044695f82c3085b08bb1686a20f025fb03
:1077e00068b9134b28460393124b694600940293e1
:1077f000fdf74af86846fbf7bdfd05b030bd54b152
:107800006946e0b227f0d2f928b903f04ffe012211
:10781000009904f01bfc03f049fe04f019fa012260
:10782000054b1a700022054b1a70e6e770cc001069
:107830000d7300029f72000277cf001076cf001008
:107840007fb5234e044696f82c300d4693b1706aee
:1078500020f0ebfa70b91f4b304603931e4b69467c
:10786000cde900450293fdf70ff86846fbf782fd6e
:1078700004b070bda4b900220121184b10461a7043
:10788000174b19700321fff73fff03f00ffe04f0c1
:10789000edf9eb07ecd504b0bde8704004f098bdfd
:1078a000204600220321fff72fffe0b2694627f0b0
:1078b0007df9044628b903f0f9fd2246009904f049
:1078c000c5fb03f0f3fd03f0ecff0028d3d0cfe7b6
:1078d00070cc0010d97600028572000277cf0010bc
:1078e00076cf001070b52a4b0c465b6886b0c3f3a8
:1078f0000803002b39d1274e96f82c30b3b1706aab
:1079000020f093fa054688b9234b30460593234b64
:1079100002a902940493fbf725fe0446c8b9054664
:1079200002a8fbf727fd284606b070bd14f0010140
:10793000019107d105f03cfa019906b0bde870400d
:1079400005f004bb05f034fa06b0bde8704005f060
:107950005fbb2a464ff0ff31406920f07ffb236870
:1079600020469b68a5699847dae711f00102019269
:1079700008d105f01dfa0121019a06b0bde870405a
:1079800005f044ba05f014fa00220221f5e700bf21
:1079900000ed00e070cc0010e17200027172000294
:1079a0007fb5174b04465b680d46c3f308031646c4
:1079b000ebb9144b93f82c20cab1586a20f035fa71
:1079c000a8b902900c2016f003ff10b1c0e90045e1
:1079d00086600d4b694603930c4b00900948029357
:1079e000fcf752ff6846fbf7c5fc04b070bd324699
:1079f0002946204604b0bde87040fff773bf00bfc2
:107a000000ed00e070cc0010b97b00023172000282
:107a100037b50122244b05681a700022234b1a70d7
:107a2000234bc3e88f2ffff715fc044638b1002223
:107a30001146104603b0bde83040fff7b1bf03f078
:107a400035fd214603f0d4fd0028f0d01db301a977
:107a5000e8b227f0abf840b903f028fd019904f033
:107a60001dfc03f023fd03f06eff03f01ffd03f088
:107a700050ff18b903f01afd04f0eaf803f016fd00
:107a8000002103f0b5fd60b103f010fd03b0bde8c7
:107a9000304004f0fdb803f009fd294604f0fefb78
:107aa000e3e703b030bd00bf77cf001076cf001002
:107ab00078cf001030b5304d044695f82c3085b0a5
:107ac0008bb1686a20f0b1f968b92c4b2846039352
:107ad0002b4b694600940293fcf7d6fe6846fbf7f1
:107ae00049fc05b030bd0122264b1a700022264bfe
:107af0001a70264bc3e88f2ffff7acfb054638b151
:107b000000221146104605b0bde83040fff748bfdf
:107b100003f0ccfc294603f06bfd0028f0d024b321
:107b20006946e0b227f042f840b903f0bffc009983
:107b300004f0b4fb03f0bafc03f005ff03f0b6fc5d
:107b400003f0e7fe18b903f0b1fc04f081f803f08c
:107b5000adfc002103f04cfd0028c2d003f0a6fcd0
:107b600005b0bde8304004f093b803f09ffc214617
:107b700004f094fbe2e700bf70cc001091790002a2
:107b8000cd72000277cf001076cf001078cf0010b2
:107b900070b505f00df905f00ff900283cd1224e23
:107ba0003378ebb9214c2378d3b904f017fc98b3a0
:107bb0001f4bd3e88f3fdbb20bb1237863bb03f0dd
:107bc00075fc03f0b8fe38bb03f070fc03f0a9feaf
:107bd000034608bbbde8704002460146fff76abf96
:107be00003f064fc03f0a7feb8b100220f4c10466e
:107bf00025782378edb2002b14bf07210621fff76b
:107c000083fd00231a4619461846fff719fe002384
:107c1000084a33701360257070bd03f047fc03f011
:107c200080fe0028e1d1f7e775cf001076cf001075
:107c300078cf001028d7001003681868d3e9011224
:107c4000fff7aebe13b543690446cde900030a4908
:107c500090f82220094b243020f0d0f820b10a20df
:107c6000074a0849f9f79cf994f82c3013b920f029
:107c7000e4f8f9e702b010bd85790c02597c0002e6
:107c8000bff5010293790c02002313b50193036839
:107c900001a91b689847044620b1019828b10368e0
:107ca0001b689847204602b010bd0446fae708b5a5
:107cb000012380f82c30044617f012f8a9f092f94d
:107cc000251d2046fff7e0ffe3680bb9a7f0f2fca3
:107cd000284623699847f4e708b5fff7e8ff000056
:107ce00070b505460c4612f015fd6b686bb19c60d3
:107cf0000026a6606c6012f011fd054b586a30b189
:107d00003146bde8704020f0bdb82c60f0e770bd92
:107d100070cc001038b50446006868b112f0fafc67
:107d20002568ab682360236803b9636012f0f6fc32
:107d300028466b689847012038bd704710b5044647
:107d40000c2116f04dfd204610bd436913b1836927
:107d50000c301847704713b500210446084620f040
:107d600063f90023204601a9019320f0cdf9019c7d
:107d70000cb1012323710021012020f055f92cb111
:107d8000236820469b6898470023237102b010bdea
:107d900008b5fdf7ebff48b10cf064fa00220421ae
:107da0000bf0affebde808400bf028be6ff0d1002d
:107db00008bd000009490c2008b5a7f077fc014672
:107dc00050b1074b036000238360064b4360bde85e
:107dd00008400548fff784bf08bd00bf55860e0266
:107de000dc790c02cd7d0002f4d6001010b40368db
:107df0005a689968541001eb6200d20748bf0a59cb
:107e00001b685df8044b48bfd3581847012a38b5a2
:107e1000044602d10b68236003e0022a03d0032a40
:107e20000dd0002038bd0c200d6816f0d1fc0346a3
:107e30000028f0d095e8070083e80700ebe700682a
:107e40000028eed00c2116f0cbfceae708b510b103
:107e500003685b689847bde80840fff799bf07b51e
:107e6000806830b10023cde900131a46022120f0ca
:107e700057f903b05df804fb38b5836804469bb13d
:107e80006ff00041fff7ebff0021a06820f043f9fd
:107e9000237903f0ff0513b11ff0cffff8e7294660
:107ea000a06820f087f9a56038bd000038b5054608
:107eb0000446054b45f80c3bfff7deff2846fbf771
:107ec00059fa204638bd00bfec790c0210b50446c3
:107ed000fff7ecff20461c2116f082fc204610bd67
:107ee00010b50446064b03608068fff7c5ff237b8f
:107ef00023b1a06810b103685b689847204610bda5
:107f0000007a0c0210b50446fff7eaff2046102164
:107f100016f066fc204610bd284b2de9f0410360a9
:107f20004ff0ff3306460d4688b04360002943d129
:107f30001c2016f04dfc0446002834d00c20d6f846
:107f40000480069516f044fc18b11d4b8660c0e90c
:107f500000351c4b0490236000230df1080c04af86
:107f600097e803008ce803002371a36004f10c027e
:107f700092e8030087e803009ce8030082e803001e
:107f8000114a06936261a269414607920f4a04f1c1
:107f90000800a261cde900330d4a234620f0a2f883
:107fa0003846fbf7e7f9b5fa85f530466d09b46058
:107fb000357308b0bde8f0810c46f4e7007a0c0296
:107fc000357d0002ec790c028d7d00026d7d000292
:107fd000d77c00026ff000418068fff740bf13b507
:107fe000846800212046fff73affa06840b10023d3
:107ff0006ff000421946cde900231a4620f090f8b0
:1080000002b010bdf0b58368054698680e468bb087
:10801000f0b1002120f0ddf8041e18bf0124ab6888
:108020009868b8b100226ff000474ff47a730321cb
:108030007343cde9007220f073f8034650b9a86885
:108040006e60a4b939460bb0bde8f040fff707bf3a
:108050000446e4e720220023cde90223094a322026
:108060000092094902aafaf75dfb0bb0f0bd8068e7
:108070000028fad01a460121cde9007320f050f80b
:10808000f3e700bfab790c0220740c02fff780be4f
:108090002de9f04f0025b5b081460c469246099572
:1080a000002a78d05378002b75d029462a221da8a3
:1080b0001c95a8f0a6f808230c20cde90130cde9e5
:1080c0000c550cad00959af800102e2350461caab2
:1080d00026f044f9014600285dd1102218a8a8f026
:1080e00090f84c2314939af80130b9f1110f1593bd
:1080f0000cbf022301232946169314aa09ab1ca81e
:10810000cdf85c9026f0f0f8002844d10125099bb9
:108110004bb92022cde91c23a44a32200092a44965
:108120001caafaf7fffa202100236ff0e508a14a04
:10813000cde91c13009201209d4901951caafaf774
:10814000f1fadff86cb2099c002c00f0aa81d4e9a6
:108150000212606826f00afb00262023071ecde9e4
:108160001c3680f29880d4e90173e2680793069286
:10817000a7f01afe079b0168069acde901738e4ba2
:108180000491039200935946334632201caafaf711
:10819000c9fae469d8e7894b5a6822b19b6813b1e0
:1081a00002250993b3e7002c73d025781db1012d6a
:1081b00035d00025abe71022294620a8a8f021f8e9
:1081c00002264c23b9f1110fcde91c360cbf334602
:1081d0000123d4f802001e93cde91455cde91655bc
:1081e000cde90c55cdf87c900a9527f050fc102372
:1081f0000a9014aa30460aa927f045fc002886d028
:108200000821b4f842306e4a0ca8a9f031f809ab45
:108210001caa0ca914a826f067f8032577e71c22ee
:1082200000210da8a7f0edff4823b9f1110f4ff081
:1082300000060c930cbf022301235c2231461da8cb
:108240000aaf0e93cdf83c901c96a7f0daff60229f
:108250005c4b1ca9a01ccde90a6607f0acfc082108
:10826000b4f84230564a3846a9f002f82023cde946
:1082700014361cab0193544b28464d49009314aa65
:1082800033460297faf74efa394609ab0caa1ca8f6
:10829000c1e725463be7e36859460493a3680120fc
:1082a000039363681caacde90173484b00933346de
:1082b000faf738fa2a2231461da81c96a7f0a1ff2a
:1082c0006068022846d00a2850d020220023cde939
:1082d00014231caacde901723d4a594600921e2082
:1082e000039614aafaf71efab9f1110f76d1626853
:1082f00000230a2a72d11c2219460ca8a7f081ff7c
:108300001c228df830206368022b8df8313032d07a
:108310000a2b30d0012304220a9340f6ff7138461d
:1083200000920aab26f0edf960b320230026cde9d8
:108330001436a7f039fd03685946cde90173254b82
:108340003220009314aa3346faf7ecf9384626f0a7
:10835000fff91ee72e2361691caa043127f093fb65
:108360006369588827f099fb0646aee761692e23ba
:108370001caa0831f2e741f2346027f08cfbadf81b
:108380003200c7e706901c2238460ca926f07af97d
:10839000069b18b32022cde914230f4a59460092b8
:1083a000322014aafaf7bef9d0e700bf187a0c02ff
:1083b00020740c023b7a0c024c7a0c0264510010bf
:1083c000a0a30c0271a70002087a0c028b7a0c029f
:1083d000bc7a0c02e17a0c02177b0c023846d4e915
:1083e000042126f0b7f920238046149390b100238e
:1083f0001593a7f0d9fc02681cabcde903622c4aa7
:10840000cde90173009200235946322014aafaf7ed
:1084100089f99be71cabcde90173264b15900093be
:10842000254903460396012014aafaf77bf9b9f10e
:10843000110f224b0ad1023d012d07d85968e2697c
:1084400031b19a604ab90991c3f80480012505e069
:10845000002afbd00999c3e9011245461f60baf111
:10846000000f04d0d4e904215046a7f0a3fe002653
:108470000c960ca96068fcf70bff01220c99606850
:10848000fcf7aefe304603f0dbff012808d1304692
:108490001ff0c9fc0a49149014aa384626f0a1f925
:1084a00015b1099825f01eff404635b0bde8f08fa4
:1084b000417b0c02777b0c0220740c02645100108b
:1084c0000873048030b50a4601461148002300684d
:1084d0008db026f047f9041e15daa7f065fc036895
:1084e00000250c2b12d02023cde90435a7f05cfc2d
:1084f00003680849cde90143074b3220009304aae1
:108500002b46faf70ff920460db030bd2c46fae79e
:108510006451001020740c029b7b0c0230b50a469b
:1085200001461748082300688db026f017f9041e8d
:1085300007daa7f039fc03680b2b05d1a7f034fc50
:10854000002420460db030bda7f02efc03680b2b95
:10855000f4d0a7f029fc03680c2befd020230025d2
:10856000cde90435a7f020fc03680649cde90143b5
:10857000054b3220009304aa2b46faf7d3f8e0e724
:108580006451001020740c02b47b0c0230b5144c02
:1085900089b02368002b1fdbc20715d501211846bf
:1085a00026f072f880b919f082ff054600222021da
:1085b0006846fff7b3ff002806db19f078ff41f2a9
:1085c0008732431b9342f1d9206826f0c1f84ff05f
:1085d000ff33236009b030bd6ff0d100fae700bf70
:1085e0006451001013b501a828f0d2fa002242f21b
:1085f0001073114601a828f05ffb044601a828f07b
:10860000d8fa204602b010bd6ff077007047000026
:10861000014b1868c017704764510010014b18686f
:10862000704700bf6451001010b50446503052f03e
:108630003afe04f1440052f036fe2046faf71efce2
:108640002046bde81040b02116f0cab838b504463f
:10865000062052f017fe054668b1204652f01efe75
:1086600000222946204652f071fe034628b1bde89b
:10867000384028f083bf6ff07703184638bd08b53f
:1086800052f0a4fe18b1bde8084028f077bf08bd3d
:1086900008b552f0b7fe18b1bde8084028f06ebf2b
:1086a00008bd00221421c0e90022c0e902220261b3
:1086b0000180426102764276c261704710b50a4c71
:1086c000d4e88f3fdb070cd4204618f01ff940b1e7
:1086d0000648fff7e6ff204618f052f90448a7f0d5
:1086e00042fb024810bd00bf04d0001008d00010ab
:1086f000c58700022de9f047c469a0b0289f002c6f
:1087000000f09480d4f8a0509d4211d39e18ae4240
:108710000ed9eb1a761b3246194404f14400fff7d8
:10872000b7ff002869dbd4f8a0303344c4f8a03088
:10873000d4f8a030bb4229d200217c2201a80091ac
:10874000a7f05ffd1af08efcd4f8a030c61900eb3c
:10875000030904f14408b14516d2a6eb090abaf19f
:10876000800f28bf4ff0800a6946524648461af0eb
:10877000abfc002841db524669464046fff788ffc4
:1087800000283adbd144e6e7c4f8a070d4f8a03062
:10879000ab4229d904f15006304604f1440152f0ad
:1087a000affd30bb304604f17c0152f045fe18b1fc
:1087b00028f0e4fe002820db4822204604f15c017a
:1087c000faf756fc002818dbd4f8ac30ab4203d1e2
:1087d00019f06dfec4f8a400d4f8a830d4f8a02095
:1087e00013445d1bc4f8a850d4f8a83043b9002046
:1087f00003e028f0c3fe0028d4da20b0bde8f087fb
:1088000019f055fed4f8a430c01a47f22f539842fd
:10881000edd92046faf7a2fa0028eedb19f047fe60
:10882000c4f8a4000020c4f8a800e6e76ff0d10067
:10883000e3e710b50446006808b1fff7f5fe2046ef
:1088400010bd000008b50248fff7f3ff08bd00bfe8
:1088500024d000100368016013b11846fff7e4be8e
:108860007047000070b5c56906468ab03db3d5e9ca
:1088700027329a4226d1202205f15c0105f17c00c5
:10888000a7f088fc044688b1002320220e4ccde9d5
:10889000022332200d49009402aaf9f743ff204633
:1088a000f9f7a0fc0a4c20460ab070bd2846faf73a
:1088b000e5fa214606f11c00fff7ccfff3e76ff065
:1088c000d104f0e7034ceee7d87b0c02cd7b0c0221
:1088d000cdfaffffb9faffff10b50446c06992b0a8
:1088e00040b1faf7dffa002104f11c00fff7b2fff4
:1088f00012b010bd054901a8faf720fa01a8faf74d
:10890000d1fa01a8faf7bafaf2e700bf077c0c0225
:1089100070b5037e05468ab0c3b1c469b4b1d4f85a
:10892000a8309bb119f0c3fdd4f8a430c01a47f2a7
:108930002f5398420ad92046faf710fa00284ff030
:10894000000605db19f0b3fdc4e929060ab070bdc5
:108950002023cde90236074b0190009332203346a5
:10896000054902aaf9f7defe28460ab0bde87040c4
:10897000fff7b2bf187c0c02cd7b0c027fb5037ee3
:1089800005460e463bb31c300021fff763ff687eaf
:1089900008b90af058fc0024104ba6421c7018bffe
:1089a00001222b4608bf4ff0ff3200214ff48070a8
:1089b000cde901442c760094fef7d2f92046fbf76e
:1089c000dbf92346024600214ff48010cde9014433
:1089d0000094fef7c5f904b070bd00bf37cb00109e
:1089e00070b511f008020546047e01f0040301f0a1
:1089f000010626d18cb3e3b9c4691cb1fff732ff7d
:108a0000041e10db7eb900201af092fb0446e143fd
:108a10002846c90ffff7b2ff002c10db4620fbf7fa
:108a200093f800240be02846fff756ff002ceedbfe
:108a3000e9e7422101201af049fb00eae0742046f0
:108a400070bd002cfbd0002bebd10eb1fff744ff23
:108a500000212846fff792ffe3e76ff0d104eee72d
:108a60002de9f0411f46037e0446884616468cb029
:108a7000002b56d01af0f6fa0023c11932464046b0
:108a80001af012fb0546d0b100262023264f04aa77
:108a9000cde9043625493346019000973220f9f795
:108aa00041fe29463846f9f79dfb31462046fff73f
:108ab00065ff6ff0da0528460cb0bde8f081e36988
:108ac000bbb1129b3246009341463b462046fff71e
:108ad00011fe70b12023cde90435154b01900093b0
:108ae00032202b46114904aaf9f71cfe2046fff755
:108af000f3fe637e13b9e720f8f7befb2369022279
:108b00003b44636000234ff480700021cde90133c2
:108b1000009326812346fef723f919f0c8fc606113
:108b2000c9e76ff0d105c6e73c7c0c02cd7b0c0297
:108b3000187c0c022de9f04fa5b001908846b020ba
:108b400066491646a6f0b2fd044698b10025644970
:108b5000faf7f4f848222946c4e91155c4e9135537
:108b6000c4e9155504f15c00a7f04bfbc4e9295595
:108b7000c4f8ac500394002c00f0ad8004f1440024
:108b8000fff764fd041ec0f2968003985030fff793
:108b90005dfd041ec0f28f80039d482205f15c0735
:108ba00039462846faf7e6f94828044640f08a8014
:108bb000d5f89c30434552d1d5f8a03043454ed826
:108bc000202231463846a7f0e5fa8246002846d1f1
:108bd00003984430fff753fd041e6cdb51467c22a2
:108be00005a8cdf810a0a7f00cfb1af03bfa8346bd
:108bf000d5f8a03000eb030ad34517d2aaeb0b0936
:108c0000b9f1800f28bf4ff0800958464a4604a9a1
:108c10001af05afa041e4edb03984a4604a944305f
:108c2000fff736fd041e46dbcb44e5e7039800f171
:108c30004401503052f064fb002838d1039804a955
:108c4000503052f0f9fb18b128f098fc041e32dbca
:108c5000202204a905f17c00a7f09cfad8b1039862
:108c6000faf720f906f1200356f8042b9e4247f844
:108c7000042bf9d12022002105f17c00a7f0c1fad4
:108c800000230398c5f89c80c5f8a0304430fff756
:108c9000f6fc041e0fdb00240399d5f8a0300198e0
:108ca000c1f8ac301c300394fff7d4fd03e028f08a
:108cb00065fc041ec2da03a8fff7bbfd204625b001
:108cc000bde8f08f0028cada10f1aa0fc7d010f55e
:108cd0008c7ff0d1c3e7034cede700bf55860e0251
:108ce000077c0c02fcfeffff2de9f0478cb0149dc1
:108cf00004460f461e46904605f0040905f0010a99
:108d0000bab1b3b1c5f34005227ea2b10023202140
:108d10006b4ccde9041332206a4904aa0094f9f798
:108d200001fd2046f9f75efa6ff0d1000cb0bde806
:108d3000f0870125e8e7012004a98df81020faf753
:108d400069fe9df8102012b16fb95f48eee7092067
:108d500004a98df81020faf75dfe9df81030002b65
:108d6000f2d15a48e2e71af083f9b842edd3baf1ea
:108d7000000f1bd1d5b9424639462046fff7dafe2f
:108d8000002877da20220023cde90423504a0190fd
:108d9000009232204b4904aaf9f7c4fcb9f1000f44
:108da00040f087802046fff797fd07e0b9f1000ffc
:108db0007ad12046fff790fd002ddcd01af052f951
:108dc000394600221af05ef9014600285ed04ff0c5
:108dd0000008002211461046faf704fef8f7e2fafe
:108de0000546607658b901200af02dfa29460b2075
:108df000fdf724fd002850d000690af047fa01234e
:108e00000025344a237613701423a446cde9045573
:108e1000cde907550695adf810300df1100ebee8fe
:108e20000f00ace80f00ccf80050e7601af01af918
:108e300020611af023f92369208163602a462346c2
:108e40000021a5724ff48070cde901550095fdf722
:108e500087ff2846faf790ff2b46024600214ff481
:108e60008010cde901550095fdf77aff19f01ffb41
:108e7000606120e0e369d3f8a080b9f1000f0fd062
:108e8000002104f11c00fff7e5fc14e004f11c00d4
:108e9000fff7e0fc6ff0da0048e74ff0ff10ace7b7
:108ea000b8f1000f95d189e71db9baf1000f3ff471
:108eb00062af4ff000080eb1c6f80080002035e721
:108ec0005d7c0c02cd7b0c02b9faffff9cfaffff20
:108ed000847c0c0237cb001048b10138222896bfa1
:108ee00005230723b0fbf3f34ff47a7098407047e3
:108ef00008b580b103881b2b0dd94ff0ff330371e8
:108f0000002343710123837105231422c371034994
:108f10000830a8f0c9ff1c2008bd00bfaf730c02c9
:108f200010b50446007c10b1d4e902309847207493
:108f300010bd036802224068184770470eb4f0b5b0
:108f4000002692b017ad55f8047b3c22314604460a
:108f500003a80296a7f055f93a462b46402102a8ed
:108f60000195a9f091fb3f28024605dd267412b059
:108f7000bde8f04003b07047204602a9fff7d0ffdc
:108f8000f5e710b50446142115f02afc204610bd63
:108f900013b5044608460191f7f7f4fe0246204651
:108fa000019902b0bde8104009f064be37b56fea20
:108fb00041416fea5141adf8041001a9044615463c
:108fc000fff7b7ff30b104222368606801950deb0d
:108fd0000201984703b030bd7fb50e4615460446e2
:108fe00008b1036923b90a20094a0a49f7f7d8ffeb
:108ff0000c23cde901362b68012103932046236918
:1090000001aa984708b9039b2b6004b070bd00bf4c
:10901000bff50102b77c0c0237b5c3880446012bab
:109020000d4604d00a20074a0749f7f7b9ff042381
:10903000294620460deb03020193fff7cdff03b055
:1090400030bd00bfbff50102dd7c0c0237b5c3881f
:109050000446022b0d4604d00a20074a0749f7f7b9
:109060009fff0423294620460deb03020193fff7df
:10907000b3ff03b030bd00bfbff50102097d0c0294
:1090800073b5cb880546012b0c4605d0022b17d0b3
:109090006ff0770002b070bd002369462046009350
:1090a000fff7baff0246f0b9a388286801a9009e1d
:1090b000adf80430fff73dff48b96ff0bd00e9e7b8
:1090c0000023694620460093fff7c0ffeae7042229
:1090d0002b6801961c6858680deb0201a047002818
:1090e000ebd00020d6e7a1882868fff75ffff6e7fe
:1090f0000b4601461846fff7c3bf13b504460846a2
:109100000191f7f73ffe02462046019902b0bde803
:10911000104009f09fbd000038b5044615460068b0
:10912000fff7ebff206809f0e3fc06492068fff732
:10913000e4ff294609f0e8fc206809f0b7fc236841
:10914000187c38bd3f820c0273b5054688680c4612
:1091500030b1cb88012b05d0022b19d06ff07700ee
:1091600002b070bd0023204601a90193fff754ff10
:109170000246f0b9019ea1682868fff7beff31469c
:1091800009f0e6fc2b681b7ccbb96ff0bd00e7e76c
:109190000023204601a90193fff758ff024640b97a
:1091a000019ea1682868fff7a8ff314609f0e2fc9c
:1091b000e8e72846a168fff7afff0028e5d00020c8
:1091c000cee70b4601461846fff7bebf2de9f04f2c
:1091d0009a4b99b01546039300240123cde905016c
:1091e000974903a88df81c308df81040fff785ffd4
:1091f000698809f089fc24272b8aa3420dd907fb33
:1092000004f6eb6803a89959fff777ffe968013482
:1092100031440431fff7bcfeeee78a4903a8fff7ab
:109220006cff03a809f058fc4ff00008dff84892e3
:109230002b89434540f2f980782606fb08f6d5f8dd
:1092400004b00beb060494f82230052b00f2d28018
:10925000002b00f0d380a37b012b04d1b4f8703035
:109260009b0740f1cb8004f114073846f7f70cfe5a
:10927000824603a809f03cfc734903a8fff73dffb1
:109280005bf8061009f076fc704903a8fff735ff7c
:10929000a37b032b96bf6e4a6e4952f82310fff74b
:1092a00077fe6d4903a8fff728ffb4f86e1009f0a8
:1092b0002bfc6a4903a8fff720ffb4f8701009f0ef
:1092c00023fcbaf1050f2ed100213c2209a80891f8
:1092d000a6f097ff624903a8fff70fff04f16c06a1
:1092e00004f14c0308aa13f8011b0232090901f129
:1092f000300cbcf1390f88bf01f1370c02f802ccf9
:1093000013f8011c01f00f0101f1300cbcf1390f11
:1093100088bf01f1370c9e4202f801cce3d1402214
:1093200008a909f0a7fc4f4903a8fff7e6fe064687
:109330003846f7f7a9fd082898bf59f8201030469d
:109340004ff0000688bf4349fff722fe38460896d3
:10935000f7f79dfd444a0346042108a8a7f088ffbb
:10936000424903a8fff7c9fe08a9fff711fe4049cb
:1093700003a8fff7c2fe82463846f7f78dfd014687
:10938000504609f0c1fb3b4903a8fff7b6fe03a80e
:1093900009f0a2fbdff8ccb094f8247094f82530e3
:1093a000b4f826a0052f34d8002f35d003a8019398
:1093b00009f09efb594603a8fff79ffe59f82710b6
:1093c000fff7e6fd019b284a042108a8a7f050fffb
:1093d000264903a8fff791fe08a9fff7d9fd244904
:1093e00003a8fff78afe514609f08efb03a809f097
:1093f0005dfb11e0073b012b7ff62daf08f1010863
:1094000016e7012694f8287094f82930b4f82aa0b9
:10941000c8e7f91f0129c9d9002ef2d003a809f025
:109420003cfb03a809f042fbe8e703a809f035fb81
:109430009df81c0019b0bde8f08f00bf987d0c02ac
:10944000958d0e02c86a0c0214810c0262cd0c02ca
:10945000807d0c02ff8e0c0289f30c02367d0c021b
:10946000a1a30c02948b0e02a0a30c02a88e0e02e4
:10947000b2780c02c37f0c025c7d0c0218b1002292
:10948000012119f0febc0148704700bff2feffff4a
:1094900018b10022114619f0f4bc0148704700bf12
:1094a000f2feffff30b587b004460d4612220021c0
:1094b00001a8a6f0a6fe14230022adf80430012373
:1094c000114601a8adf81630fff7d8ff294601aaca
:1094d0002046fff77bfe0446002101a8fff7d8ffd6
:1094e000204607b030bd000003681f221b680149f9
:1094f000184700bf397d0c02f0b512f0010489b0a5
:109500000e4605460e9933d0cde9033103ab0193e6
:10951000022302a903a8adf80830fff70afd10b92d
:109520006ff0bd0022e00423019802a9adf80830d5
:10953000fff7fffc0028f3d095b100242746a64290
:1095400033d0002235f8140002a90297f9f7cafbbc
:1095500060b9029901a8fff793fd38b90134eee72d
:109560002b4629461f4801aaf9f798fb09b0f0bd20
:10957000cde905311c4b8df81040039301238df884
:109580001c3003ab1846019309f0b2fa019b1b7c17
:10959000002bc5d0e5b12746a64208d1019809f0b5
:1095a00085fa019b1b7c002bbad00020dee700224d
:1095b00035f8140002a90297f9f794fb0028d5d1d9
:1095c000029901a8fff7c0fd0028cfd10134e3e7dd
:1095d0002b462946054801aaf9f760fb0028ddd093
:1095e000c4e700bf71900002987d0c024391000215
:1095f00013b500240346cde9001420462146fff7a9
:109600007bffb0fa80f0400902b010bd70b5264b68
:1096100088b0002403930123cde90501234903a861
:109620008df81c308df81040fff767fd09f054faf3
:1096300000f0fafd26460546ac420ed0204602a9af
:10964000029600f0f7fd10b1002008b070bd02993d
:1096500003a8fff79dfc0134eee703a809f01dfa0b
:10966000134903a8fff749fd09f042fa002400f06e
:10967000bbfd26460546ac4211d0204602aa01a9f0
:10968000cde9016600f0b6fd0028ddd1019903a8ff
:10969000fff733fd029909f037fa0134ebe703a82d
:1096a00009f004fa0120d0e7987d0c02948b0e0299
:1096b000b2780c0270470368c1f8d030d1f8e030be
:1096c00043f00403c1f8e03070470368c1f8dc30b0
:1096d000d1f8e03043f00803c1f8e0307047036888
:1096e000a1f8e830d1f8e03043f01003c1f8e030e1
:1096f00070470368a1f8ea30d1f8e03043f0200366
:10970000c1f8e03070470368c1f8e430d1f8e030c8
:1097100043f04003c1f8e03070470368a1f8ec3033
:10972000d1f8e03043f08003c1f8e0307047002307
:1097300081f8e03081f8e13081f8e23081f8e330ff
:1097400070470000f0b404460f46bab90388b3f579
:10975000837f0cd10b4e051d06f12002334603cb4f
:109760009342286069601e4605f10805f6d1002382
:109770003a462146f0bc184611f084bb4ff0ff304a
:10978000f0bc704748cc00101fb500240a46009476
:10979000014603ab2046039411f084fb00b103940f
:1097a000039804b010bd10b5002488b02146cde95f
:1097b000040404a8cde9064418f0c4ff234601229e
:1097c0004ff480400021cde901440094fdf7c8fa30
:1097d00008b010bdf7b50d4616461f460446fef705
:1097e0006dff33462a4621460097fff739f903b04b
:1097f000f0bd07b50190fef761ff019903b05df878
:1098000004ebfff7edb8f7b50d4616461f460446c4
:10981000fef754ff33462a4621460097fff764fac5
:1098200003b0f0bd1830036800200b60704718309b
:10983000036800200b60704700b50b4a8bb01378ab
:1098400073b10121094b1e201970002313702022cf
:10985000cde90223064a0749009202aaf8f762ffff
:109860000bb05df804fb00bf35cb001034cb00100b
:10987000a87d0c0220740c0208b510b103685b6867
:109880009847bde80840fdf7ccba13b504460191ee
:10989000f7f778fa0199a0f1180204f11800a8f07e
:1098a000effab0fa80f0400902b010bdf0b5efb0a9
:1098b00005460c46f7f766fa172842d918222846bb
:1098c0006e49a8f0ddfa074600283ad12046f7f79e
:1098d00059fa6b4902462046a8f0d2fa6949b0fa13
:1098e00080f62846fff7d1ff7609044638b13a469c
:1098f000314609206fb0bde8f040faf773b828464a
:109900006149fff7c2ffd0b12046faf735fa0122cc
:109910005e4b05461a70314622462046faf762f839
:109920002046faf729fa8542024608d023464ff42a
:1099300080100021cde901440094fdf711fa6fb0c9
:10994000f0bd132228465249a8f09afa064680b97b
:109950002023cde924304f4b4f49009324aa0346de
:109960000120f8f7dffe30466fb0bde8f04019f097
:1099700055bd28464949f7f7fbf9002846d1002c88
:10998000ddd02378002bdad021464548f7f7f0f9ef
:1099900020b96fb0bde8f04009f0cbbe2146414888
:1099a000f7f7e6f920b96fb0bde8f04009f0a6bec0
:1099b00021463d48f7f7dcf920b96fb0bde8f0402b
:1099c00009f0b4be21463948f7f7d2f90446002819
:1099d000b5d12023cde92430354b2f49009324aa5b
:1099e00003462820f8f79efe32490c20a5f05efec3
:1099f00001460028a3d0304b846003602f4b4360a6
:109a00002f486fb0bde8f040fef76ab9182228462b
:109a10002c49a8f035fa002891d12023cde9243033
:109a2000294b1d4924aa009303461e20f8f77afe0d
:109a3000032011f009f904464ff49372ff2124a882
:109a4000a6f0dffb8022ff2104a8a6f0dafb5cb1c0
:109a50001e4b1f491a6824a8a6f0acfb1d4b1e49db
:109a60001a6804a8a6f0a6fb214624a819f029fd2f
:109a7000214604a819f030fd61e700bf73830c0292
:109a8000b4720c0253830c028c830c0238cb00108e
:109a90003f830c02d37d0c0220740c022c830c0239
:109aa000097e0c02137e0c02177e0c023e7e0c0215
:109ab0001e7e0c0255860e02dc790c02f99700021c
:109ac000f4d600105a830c02467e0c02686d0c021c
:109ad0000c6d0c02086d0c02ef6c0c02f7b506461b
:109ae000184fd7e88f5f15f0010522d1384616f0e0
:109af0000dfff0b12a4614210f20fcf7a9fe1e220b
:109b00000221114c0346cde9002120460f226ff0bf
:109b10007f4109f031fe0d4b384623600c4b84f831
:109b2000225063616423238416f02aff0948a6f0bb
:109b30001af900223146084803b0bde8f040f8f7b2
:109b4000d5be00bf28d00010ecd000109c830c02c2
:109b5000ee82ee00059d0002f0d00010012a38b51b
:109b6000044602d10b68236003e0022a03d0032ad3
:109b70000dd0002038bd0c200d6814f029fe0346de
:109b80000028f0d095e8070083e80700ebe70068bd
:109b90000028eed00c2114f023feeae7012af8b5e4
:109ba000064603d10b6803600020f8bd022a08d0e6
:109bb000032af9d100680028f6d0182114f010fe0d
:109bc000f2e718200c6814f003fe074630b1054692
:109bd0000fcc0fc594e8030085e803003760e3e786
:109be000012a08bf016000207047012a02d10160ec
:109bf00000207047022a04bf0b680360f8e7012abf
:109c000002d1016000207047022a04bf0b68036084
:109c1000f8e7012a02d1016000207047022a04bf40
:109c20000b680360f8e7012a02d101600020704749
:109c3000022a04bf0b680360f8e7012a02d1016021
:109c400000207047022a04bf0b680360f8e7012a6e
:109c500002d1016000207047022a04bf0b68036034
:109c6000f8e7012a08bf016000207047012a08bff9
:109c7000016000207047012a70b5054603d10b68ca
:109c80000360002070bd022a11d0032af9d10468b4
:109c9000002cf6d004f1180009f0f6fb04f10800de
:109ca00009f0f2fb2c21204614f09afde9e72c2064
:109cb0000e6814f08dfd044688b1338806f1080162
:109cc00003807368083040f8043c09f073fc06f127
:109cd000180104f1180009f06dfcb36aa3622c604e
:109ce000cfe7002307b5009342f001033c22fcf7c5
:109cf000fffb03b05df804fb10b58ab002f094fbe3
:109d0000042813d100242023cde90234084b02aaf1
:109d100000931e2023460749f8f704fd2246064912
:109d200006480ab0bde81040fff7dbbf0ab010bd1f
:109d30007e7e0c0220740c0247420d02967e0c02bd
:109d4000002210b50446044b114640f8043bf8f7d6
:109d5000cdfd204610bd00bfa4820c0210b5044604
:109d6000fff7eeff2046202114f03afd204610bdfb
:109d700010b50446024b0360fff7e2ff204610bd1a
:109d80009c830c020148fff7f3bf00bfecd000102a
:109d900010b50446fff7ecff2046242114f020fd07
:109da000204610bd038c8b4211d890f8223001332d
:109db000dbb2072b08bf002380f8223090f8222066
:109dc000044b53f8223043616423038470475b1ac9
:109dd000fbe700bf10830c0207b50068036901931d
:109de00002238df8033083680bb9a5f063fcc368c8
:109df0000df1030201a9984703b05df804fb0000d0
:109e000070b500242026144b8ab0144d1e2014492e
:109e1000009302aa2346cde90264f8f783fc2246a8
:109e20000221286809f06dfe044620b10ab0bde8a1
:109e3000704009f0e3bd0b4bcde90260009302aa2c
:109e4000034607491e20f8f76dfc2868214609f0f3
:109e500089ff20460ab070bdac7e0c0218d10010fc
:109e600020740c02c97e0c0230b500248bb023464e
:109e700022460f49cde900440e48fcf779f9234604
:109e800005462246cde9004409490b48fcf770f924
:109e900000b155b920220023cde90223074a322020
:109ea0000092074902aaf8f73dfc0bb030bd00bf95
:109eb0002d980002df7e0c02e87e0c02ee7e0c0282
:109ec00020740c022de9f041adf58a6d08238e4d0a
:109ed00002af00222868391dbb8009f050ff02f054
:109ee000a3fa042800f0ec80f98800201cf041f966
:109ef000012039891cf03df9032010f0a5fe38241b
:109f000080462246002107f14400a6f07af9b8f114
:109f1000000f14bf02230123a7f8444087f84630fe
:109f200000f0ec80794bbb64794bfb64794bfb66aa
:109f3000794b3b67794b7b67794b1c223b65794baf
:109f400000217b65784b07f18000bb65774b07f1fb
:109f50007c04fb65764b07f1bc063b66754b7b6664
:109f6000754bbb66754bbb67a6f04bf9402323606e
:109f7000734b4ff49372e360724bff21a363724bf8
:109f800030462362714b6362714ba362714be36392
:109f9000714b6363714be362714b2363a6f031f93c
:109fa00007f5f27318464ff41972ff21a6f029f94c
:109fb0001022ba820822fa60012207f10c013a74d9
:109fc000c7e9060619f0e4f9304619f0caf997f81e
:109fd000bc30ff2b19d120220023c7e90923614a95
:109fe00028200092604907f12402f8f79bfbb8f1a2
:109ff000000f05d05d4b30461a685d49a6f0daf8cf
:10a000005c4a136843f0010313600021084614f012
:10a010001bf80026c1b2cb1d03f4fc73adeb030d9e
:10a020000df10808404614f00ff84146286807f182
:10a03000440307f11402cde9004609f045fd33461b
:10a04000324602212868009609f0a1fe1ef0eaf8c7
:10a05000b0f57a7f06d333460122032128680096a3
:10a0600009f095fe002441f28c3223460421286831
:10a07000009409f08cfe2e6818f0faff2346024681
:10a0800005213046009409f082fe2e6818f0f6ff94
:10a090002346024606213046009409f078fe082344
:10a0a000bb84354b07f124011b682868bb6209f0ab
:10a0b00005fdfff7d9fe07f58967bd46bde8f081cc
:10a0c00000201cf059f8f88001201cf055f84ff6dc
:10a0d000ff73f9883881994204d0002328681a4612
:10a0e00009f049fe4ff6ff73398999423ff404aff6
:10a0f000002328681a4609f040fefde61f4bbb64aa
:10a100001f4bfb6418e700bf18d10010f550000288
:10a110004551000248cc0010c59600020997000284
:10a1200087970002739700025597000281aa0102e7
:10a130005d9a00022f24020227970002b9970002bd
:10a14000b9b10002c1af0002db320202df3202020b
:10a15000259400028d9500027195000239ad000230
:10a160005da600020a7f0c0220740c02686d0c02ce
:10a170000c6d0c0210d1001014d10010a950000277
:10a18000f950000210b500232024144accb01e2040
:10a19000134900920aaacde90a43f8f7c3fa00234b
:10a1a0004ff4837219460aa8a6f02bf800234ff447
:10a1b00083711a460aa8fff7c5fa00284ff000037a
:10a1c00009da084a019000923220054902aacde935
:10a1d0000243f8f7a7fa4cb010bd00bf327f0c0263
:10a1e00020740c02487f0c02014b5868704700bf76
:10a1f000d4d0001010b50a4b5c6884420bd95024af
:10a200001b6804fb003009b1431d0b602ab10379c0
:10a210000020136010bd0348fce71046fae700bfba
:10a22000d4d00010defeffff014b5868704700bf1e
:10a23000e0d00010074b5a68824208d929b14c225d
:10a240001b6802fb0030083008600020704702489d
:10a25000704700bfe0d00010defeffff10b5044cd9
:10a26000236813b909f0feff2060206810bd00bf0d
:10a2700018d10010f8b50b4b0546d3e90046502322
:10a2800003fb0646b442274609d0601d40222946fa
:10a29000a7f0f6fd50340028f4d13846f8bd002769
:10a2a000fbe700bfd4d000102de9f0410f46164661
:10a2b0001c46beb005464c22002103a8a5f0a1ff14
:10a2c00002978df80c6034b16368149323880b2bcc
:10a2d00084bfa36815932846f6f754fd402802462c
:10a2e000294628bf40220df10d00a5f063ff284646
:10a2f000fff7c0ff044638b1502202a9a5f05aff6b
:10a3000020463eb0bde8f081254d6e68632e41d8f1
:10a31000502402a9224616a8a5f04cff224616a9f1
:10a320002aa8a5f047ffab689e4215db06fb044157
:10a330002868a6f0e7fe771c044658b92023cde92b
:10a340002a30184b00933220234617492aaaf8f7df
:10a35000e9f9d5e72860af604ff050086a6808fb5c
:10a3600006f608fb02f22f68921b3744394607ebca
:10a370000800a5f02cff424638462aa9a5f01aff8e
:10a380006c6801346c6008fb04f4a4f150002c6884
:10a390000444b5e72023cde92a30044bd2e700bfbf
:10a3a000d4d00010266a0c0220740c02607f0c02cc
:10a3b000f8b50b4b0546d3e900464c2303fb064694
:10a3c000b44227460ad004f1080040222946a7f0eb
:10a3d00057fd4c340028f3d13846f8bd0027fbe781
:10a3e000e0d000102de9f0410d460446bcb04422f7
:10a3f000002105a8a5f005ffab6820460493eb6893
:10a400000393f6f7bffc40280246214628bf4022ae
:10a4100005a8a5f0cffe2046fff7caff044638b1d5
:10a420004c2203a9a5f0c6fe20463cb0bde8f08151
:10a43000254d6e68632e41d84c2403a9224616a8e8
:10a44000a5f0b8fe224616a929a8a5f0b3feab6870
:10a450009e4215db06fb04412868a6f053fe771cdc
:10a46000044658b92023cde92930184b00933220f7
:10a470002346174929aaf8f755f9d5e72860af60b0
:10a480004ff04c086a6808fb06f608fb02f22f68da
:10a49000921b3744394607eb0800a5f098fe424668
:10a4a000384629a9a5f086fe6c6801346c6008fb6b
:10a4b00004f4a4f14c002c680444b5e72023cde952
:10a4c0002930044bd2e700bfe0d00010266a0c020e
:10a4d00020740c02797f0c0210b588b004466846df
:10a4e00009f01df8694604a809f064f804a8a0471b
:10a4f000044604a808f0c8ff684608f0c5ff2046d7
:10a5000008b010bd10b50446f6f73cfc01462046e5
:10a51000bde8104010f0f4ba70b5094b0025d3e93e
:10a5200000464c2303fb0646a64206d004f1080071
:10a53000fff7e8ff4c340544f6e7284670bd00bf3e
:10a54000e0d00010f8b50b4b0026d3e900475023ac
:10a5500003fb0747a7420bd0601dfff7d3ff012184
:10a560000546201d10f0ccfa284406445034f1e78b
:10a570003046f8bdd4d0001007b5fff7e3ff0090d8
:10a58000fff7caff08210190684610f0b9fa03b03e
:10a590005df804fb10b50c46fff7eeffd4f8e03091
:10a5a000c4f8d40043f00203c4f8e03010bd70b525
:10a5b000142486b02246002101a8a5f022fe7826a8
:10a5c000adf8044000240022012101a818f059fc34
:10a5d000bdf80650bdf80c30a34209dd02982021d9
:10a5e00006fb04004c3010f08bfa01340544f1e70f
:10a5f000002201a8114618f044fc284606b070bda0
:10a6000010b50c46fff7d3ffd4f8e030c4f8d800fb
:10a6100043f00103c4f8e03010bd38b58468054646
:10a620005cb144684cb12046f6f7acfb402808d832
:10a6300020462946fff7d6fe0446201e18bf0120fb
:10a6400038bd0024f9e710b410461a46d1e9103499
:10a6500024b1014620465df8044b184711465df8c9
:10a66000044b18471b681268fff7edbf07b5016878
:10a670000a468b6a32f8080b009301f11803496807
:10a68000fff7f0ff03b05df804fb30b5c3b04ff443
:10a690008372002104466846a5f0b3fd00234ff401
:10a6a00083711a466846fff76ff8b0f5837f12d1c1
:10a6b000bdf80050b5f5837f0dd1a3680bb9a4f0a8
:10a6c000f9ff69462046e3689847002329461a4661
:10a6d0006846fff737f843b030bd000003291fb5c7
:10a6e00015d128b101280ed0002005b05df804fb7b
:10a6f0002d4b03932d4b68460293fff7c6ff684628
:10a70000f8f738fef0e72a4b03932a4bf3e70229c8
:10a7100032d102380628e7d801a353f820f000bf51
:10a72000bda60002c7a6000269a60002d1a60002cb
:10a73000dba60002e5a60002efa600021e4b009277
:10a7400003931e4bd7e71e4b009203931d4bd2e79a
:10a750001d4b009203931d4bcde71d4b00920393bd
:10a760001c4bc8e71c4b009203931c4bc3e71c4bcc
:10a77000009203931b4bbee701290cd130b1012895
:10a78000b2d105b05df804ebfff711bf05b05df87d
:10a7900004ebfff7f1be0429a6d10428a4d1124b83
:10a7a0000393124ba7e700bf15a50002ed9b000223
:10a7b00081a50002e39b000237960002cf9b0002b6
:10a7c0004b960002bb9b00025f960002a79b000213
:10a7d00073960002939b0002879600027f9b000203
:10a7e0009b9600026b9b0002af960002619b0002e9
:10a7f0002de9f04302291646984691b03dd10a460c
:10a8000001461f48a5f0c6fc0446002835d11c258a
:10a8100001a8fbf7d1fa2a46214609a8039fa5f013
:10a82000f0fc214609a8adf82450fef761fb9df825
:10a830002b20144905a808f0edfeddf81c9007eb6d
:10a840000905a84513d93a4601993046a5f0b2fc4e
:10a850004a460599f019a5f0adfc05a808f014fecc
:10a8600001a808f011fe284611b0bde8f08305a844
:10a8700008f00afe01a808f007fe0025f3e700bf74
:10a88000fd840c02927f0c020138c0b208289abfe6
:10a89000014b185c0220704704830c02042906d087
:10a8a000092907d0012914bf04200120704718b1dd
:10a8b000f6f768ba082070477047000010b5184bcb
:10a8c0008cb01b7803f0ff001bb1164b1c7814b141
:10a8d00001200cb010bd17f0eafd134b1b78002bc4
:10a8e000f6d043f69821114a1368c31a8b42efd968
:10a8f0002023cde9043413680d49cde901030d4b44
:10a900002820009304aa2346f7f70cff204623468d
:10a9100022462146009404f06bf92046d9e700bf97
:10a9200036cb00102cd7001033cb00102cd00010e9
:10a9300020740c02977f0c0208b5fff78ffc054bc3
:10a94000186809f0d5f818b9bde80840fff7baba99
:10a9500008bd00bf18d1001008b50120f9f77af83a
:10a960000920f9f777f8002008bd00002de9f04331
:10a9700000244ff02008b14bb1b01c70b04bb14e69
:10a9800020ad2a46b04901900093074623461e2079
:10a99000cde92084f7f7c6fe2146306809f09bf820
:10a9a0000d28034657d12346032240200021cde93c
:10a9b00001440094fcf7d4f9a44ba3492a461e2075
:10a9c00000932346cde92084f7f7acfefff794f916
:10a9d000fff7c2ff204617f09bfe014628b9fbf7a0
:10a9e00057f90146002800f0e58001f01dfd01281f
:10a9f00040f00081964b1b78002b40f0fb80954b7c
:10aa00001868b0b101230a22294608f03cfe002450
:10aa10002023cde91034904b1e208b49009310aabf
:10aa200023460195f7f77efe224629468b48fff71d
:10aa300058f900220823306810a9cde91022adf89a
:10aa4000403009f01efa0446002800f0dd8008f0ce
:10aa5000d5ff0446d4e020b131b0bde8f04308f0a2
:10aa6000cdbf02220021cde9010000900df1400987
:10aa70004020fcf775f94021484618f0fcfc0446dc
:10aa8000b0b99df84030013bdbb2fd2b10d8744bc0
:10aa90002a46cde920806c490093cdf80490034606
:10aaa0001e20f7f73ffe224649466e48fff719f988
:10aab0000023402249461846009313f0ebfa04465f
:10aac00090b99df840307bb12023cde92030664b12
:10aad0002a465d49009303461e20f7f723fe2246cf
:10aae00049466248fff7fdf8fff706f90022062005
:10aaf0000df117018df81720f8f78cff0446002898
:10ab000052d19df81730002b4ed002460146062048
:10ab1000f8f768ff224607a906a8cde906440ff01a
:10ab2000e3ff002840d1ddf81880b8f1000f3bd0da
:10ab30005ffa88f3502b079c7bd047d8282b7bd01b
:10ab40003cd8142b00f0b2801e2b00f0b1800a2bf1
:10ab500000f0b0804346464a40212846a6f088fbd4
:10ab6000b8f1820f01460ed1631edbb20c2b2844d4
:10ab7000c1f140013bd83f4a52f82330002b36d078
:10ab80003d4aa6f075fb00242023cde908343b4b59
:10ab90001e202d49009308aa2346f7f7c3fd22463d
:10aba00029463748fff79df8fff7d6fe0fb1faf7b1
:10abb00014fb0021306809f0adf816e73c2b7bd080
:10abc000462b7bd0322bc5d12e4b33e0782b77d060
:10abd00007d8642b76d06e2b76d05a2bbad12a4b5d
:10abe00028e0822b72d08c2bb4d1284b22e0234654
:10abf000274ac6e7fff704f9044600283ff4ffaef2
:10ac0000204631b0bde8f083119b012013f0010f05
:10ac10000cd0204b2a4618702023cde920341e4b3f
:10ac2000094900932346f7f77dfde9e71b4b1870b0
:10ac3000e6e71b4b1b4a8fe71b4bfbe744cc00109e
:10ac400045800c0218d1001020740c026e800c029a
:10ac5000c4d2001010d1001051810c0276810c0278
:10ac600095800c02c4800c02dc800c02fc800c027b
:10ac7000c27f0c02d0820c0211810c0216810c02e0
:10ac800039810c02e27f0c0231800c0240800c0200
:10ac9000c07f0c0235cb00108d810c0234cb00102c
:10aca00024800c0213810c0219800c02084bc1e7ae
:10acb000084bbfe7084bbde7084bbbe7084bb9e7bc
:10acc000084bb7e7084bb5e7084bb3e7084bb1e7cc
:10acd000c57f0c02ff7f0c02cad00c0210800c0250
:10ace000ea9f0c02d97f0c02f17f0c02cf7f0c028d
:10acf00080660c02024b0021186808f0eebe00bf0f
:10ad000018d1001010b5104b8ab01b78bbb1fff7fb
:10ad1000f1ff044698b92023cde902300b4b0c49d2
:10ad2000009302aa03462820f7f7fcfc234622469c
:10ad300001212046009403f05bff0ab010bd17f01c
:10ad4000b6fb044b1860f8e736cb0010d6810c0236
:10ad500020740c022cd00010f8b50c461646114990
:10ad6000054608f0dcfb2644a64219d02746237886
:10ad700028461b0903f13001392988bf03f1570127
:10ad800008f03afc3b78284603f00f0303f130014a
:10ad9000392988bf03f15701013408f02dfce3e79e
:10ada0002846f8bd47420d020048704730d00010d9
:10adb00000487047bcd00010f0b50c461d46096c29
:10adc0003d4ba5b0994206462a9f08d12b46214605
:10add00030462a9725b0bde8f040fff734bc00208c
:10ade000019201f02dfb019a0028efd0114602a834
:10adf00008f095fb294606a808f091fb2f4b93f825
:10ae00002c203ab906a808f03ffb02a808f03cfb4a
:10ae100025b0f0bd586a1df008f805460028f1d1ac
:10ae200002a910a80f94adf8386008f0c3fb06a97a
:10ae300014a808f0bffbbdf8383010a9adf8643095
:10ae40000f9b1ba81a93189708f0b4fb14a91fa80e
:10ae500008f0b0fb189b2c2023930c9513f0b8fc42
:10ae6000044680b1bdf864301ba903801a9b0830ea
:10ae700040f8043c08f084fb1fa904f1180008f016
:10ae80007ffb239ba3620e4b1fa80d930d4b0a94cf
:10ae90000c9308f0f9fa1ba808f0f6fa0aa907487b
:10aea000f9f7f2fc0aa8f8f765fa14a808f0ecfa2a
:10aeb00010a808f0e9faa5e72d98000244d2001086
:10aec000eda50002f79b00022de9f0431f46194b48
:10aed000164693f82c2085b00446dde90c890d4612
:10aee000eab1586a1cf0a1ffc8b90290182013f00b
:10aef0006ffc28b1c0e90045c0e90267c0e90489d8
:10af00000d4b694603930d4b00900a480293f9f7e5
:10af1000bbfc6846f8f72efa05b0bde8f0833b4667
:10af2000324629462046c446cdf8309005b0bde8eb
:10af3000f043604770cc0010c1ae00021d9b0002c0
:10af400007b500684369019303690093d0e90223c0
:10af5000d0e90001fff7b8ff03b05df804fb000083
:10af60002de9f041304b174693f82c2004460e464d
:10af700088b0d2b1586a1cf058ffb0b906900c20c6
:10af800013f026fc10b1c0e900468760274b0490ff
:10af90000793274b244804a90693f9f775fc04a8e6
:10afa000f8f7e8f908b0bde8f0810023cde90333f4
:10afb000e36c25688bb1284603aa04a998470028aa
:10afc00025da00231e201a461946cde90067fff74f
:10afd0007bff0498a5f0c8f8e4e7d4f84880b8f1fe
:10afe000000f04d02a462179601dc0470546284637
:10aff0002179fff753fc8046039040b1a5f0acf8ef
:10b0000004900028ddd042462946a5f0d3f82079e7
:10b01000fff73afcdde903320146cde90067002085
:10b02000fff752ffbee700bf44d20010b5af0002e9
:10b03000dd9a000203681868d3e90112fff790bf98
:10b0400037b50c461546fff715f9034630b12a46c9
:10b05000214603b0bde83040fff782bf02460146fb
:10b0600000951d20a04703b030bd38b50023836094
:10b070008b6804460d462bb102229847eb68e360cb
:10b08000ab68a360204638bd012a70b5054603d1e0
:10b090000b680360002070bd022a0dd0032af9d18d
:10b0a0000468002cf6d004f10800f8f763f91821c1
:10b0b000204613f095fbede718200e6813f088fb8f
:10b0c000044648b1336806f108010360736808302c
:10b0d00040f8043cfff7c9ff2c60dbe7012a70b59c
:10b0e000044603d10b680360002070bd022a0cd017
:10b0f000032af9d10468002cf6d02046f8f73af973
:10b100001421204613f06cfbeee714200e6813f0b8
:10b110005ffb054620b13146fff7a7ff33692b617e
:10b120002560e1e713b56c460b460246d0e9000105
:10b1300084e8030093e8030082e8030094e8030036
:10b1400083e8030002b010bdf0b517461c4600228c
:10b1500043688fb000680d469847064627b11db179
:10b160000121284613f03cfb264b93f82c20002aa3
:10b1700039d0586a1cf059fe0546002833d12146c3
:10b1800004a8fff772ff04a909a80896fff76dff4e
:10b19000089b14200d93029513f01afb044670b11e
:10b1a0000146856009a8fff7bdff0b9ba268a3605d
:10b1b0000c9b0b92e268e3600d9b0c922361124b97
:10b1c00009a80393114b00940293f8f7d3f869464a
:10b1d0000c48f9f759fb6846f8f7ccf804a8f8f7db
:10b1e000c9f80fb0f0bd02238df81030a36809969e
:10b1f0000bb9a4f05ffa2046e36804aa09a99847ae
:10b20000efe700bf70cc0010599d00025db0000256
:10b2100030b5016885b0d1e9004568460831fff7cf
:10b2200024ff6b46012229462046fff78dff684622
:10b23000f8f7a0f805b030bdf0b591b00d4617464f
:10b24000fff7b6f80446002855d02846a6f0c2f805
:10b250002a4b064693f82c20002a40d0586a1cf04e
:10b26000e4fd054600283ad1394606a8cde9044652
:10b27000fff7fbfe049b06a90a93059b0ca80b9302
:10b28000fff7f3fe1820029513f0a2fa044688b1e6
:10b290000a9b056103600b9b00f1080143600ca849
:10b2a000fff740ff0e9b226923610e920f9b62699c
:10b2b00063610f92124b0ca80393124b00940293fc
:10b2c000f8f758f869460d48f9f7defa6846f8f7d6
:10b2d00051f806a8f8f74ef8002011b0f0bd394635
:10b2e0000aa8fff7c2fe2046012231460aabfff74b
:10b2f0002bff0aa8eee74ff0ff30eee744d2001034
:10b3000091b1000209b000022de9f84300254ff089
:10b3100014082c4b2c4cc3e900559d602b4b0a2183
:10b32000c3e900552a4a9d602046fbf7b5fe294b2c
:10b33000294a1e2104f11c002360a561fbf7acfe25
:10b34000264bdff8c090e361254b264fc4e90f83fd
:10b35000254b2946636404f13c0004f13803a364df
:10b360006563c4f83890e764f7f75afc1f4b204e2a
:10b37000e365204b2946236604f1580004f1540389
:10b38000c4e91937c4e91459a663c4f85880f7f71b
:10b3900047fc194a0d2104f170006665e566fbf76c
:10b3a0007bfe47f23052154bc4f888502367144b8c
:10b3b000c3e903551d705a601d725d729d82bde820
:10b3c000f88300bfd4d0001030d00010e0d00010bf
:10b3d00005820c02b8820c0210820c02c8820c0298
:10b3e0000e000200e96d00021f820c021d00020027
:10b3f00010790c022b820c0239820c0220790c028b
:10b40000bcd00010c4780c0209490c2008b5a4f087
:10b410004df9014650b1074b036000238360064b92
:10b420004360bde808400548fcf75abc08bd00bfb2
:10b4300055860e02dc790c02c1b30002f4d600106e
:10b4400010b510b103685b689847faf78ffc40b1fc
:10b45000fef704ffbde81040002304211a4608f05f
:10b46000f6bc10bdc0e8af1f7047002108b5034609
:10b47000c0e9001101620a460830c0e8af1f03f1bd
:10b480000c00fff7efff03f11000fff7ebff03f1f4
:10b490001401c1e8af2f03f11801c1e8af2f01215a
:10b4a00003f11c02c2e8af1f184608bd10b50a4cd4
:10b4b000d4e88f3fdb070cd4204615f027fa40b1c3
:10b4c0000648fff7d2ff204615f05afa0448a4f0c8
:10b4d0004afc024810bd00bf1cd1001020d1001052
:10b4e00085b4000210b50446006818b124f0bef916
:10b4f00000232360606818b122f0c4fe002363605b
:10b5000010bd00000148fff7edbf00bf20d10010c3
:10b510000c30d0e8af0f831e5842584170471030ae
:10b52000d0e8af0f831e5842584170471fb51c30fa
:10b53000d0e8af3f022b0fd193681b78022b0bd1c1
:10b5400000230522cde90133009320200021fbf7e1
:10b5500007fc05b05df804fbd0e8af3f002bf8d145
:10b5600092681278012af4d10322cde901330093c5
:10b57000ebe773b50024054601a8019422f064fdb1
:10b58000a04219db0198264603465bb15a682ab1ee
:10b590005278022a04d00a2a08bf01241b68f4e763
:10b5a0000126fbe722f048fd05f11403c3e8af6f65
:10b5b00005f11803c3e8af4f02b070bd002307b513
:10b5c000084669460093adf8043023f0b2fc02222d
:10b5d00068460649a6f054fc30b910f02bf810f07c
:10b5e000f5fb03b05df804fb0120fae7a8830c0229
:10b5f000f7b506460c4611bb6846009123f064fa85
:10b60000002819db2746009d9db1686878b101a923
:10b61000019723f090fb002809db019b1b0706d450
:10b6200030466968fff7caff002818bf04462d6836
:10b63000eae7009823f074fa204603b0f0bd03b0a7
:10b64000bde8f040fff7babf2de9f0430e4689b0e0
:10b650000021fff7cdff4ff00008002845d004a8d7
:10b66000cdf8108023f030fa404504da204c204613
:10b6700009b0bde8f083049d1d4cdff878902db330
:10b68000686808b305a9cdf8148023f054fb00289e
:10b690001adb059b13f0080316d16f6806a938461c
:10b6a0000693adf81c3023f044fc0eb1be420bd122
:10b6b0000222494606a8a6f0e3fb074620b90ff090
:10b6c000b9ff3c4610f074fb2d68d8e7049823f0ce
:10b6d00027fa002ccbd12346022210200021cde9ed
:10b6e00001440094fbf73cfbc1e70446bfe700bf01
:10b6f000f2feffffa8830c02006a20b183688b4230
:10b7000001d00068f9e77047f0b5002585b016460e
:10b710000c468df8075031bb02a8029123f0d4f9f2
:10b72000a8421ddb2746029dbdb1686898b103a9f8
:10b73000039723f000fb00280ddb039b1a070ad4b4
:10b7400068680df1070124f05af920b99df8073017
:10b75000b34208bf01242d68e6e7029823f0e0f920
:10b76000204605b0f0bd20460df1070124f047f951
:10b7700028b99df80740a31b5c425c41f0e72c46ca
:10b78000eee77fb500250c46019539bb02a8029172
:10b7900023f09af9a8421edb2646029dc5b16868cf
:10b7a000a0b103a9039623f0c6fa00280edb039b81
:10b7b00013f008030ad1686801a9019323f02afa5b
:10b7c00020b9019b13f4801f18bf01242d68e5e701
:10b7d000029823f0a5f9204604b070bd204601a9c7
:10b7e00023f018fa18b9019cc4f30054f3e72c466f
:10b7f000f1e738b5022204460d46fff785ff28b170
:10b8000029462046bde83840fff7bbbf38bd38b5f4
:10b81000012204460d46fff777ff30b12946204646
:10b82000fff7afff80f00100c0b238bd08b5fff7e9
:10b8300063ff00b1007908bd2de9f043002485b015
:10b84000064602a80f46029423f03ef9a04224dbec
:10b85000a146029df5b16868d0b103a9cdf80c905e
:10b8600023f069fa002813dbddf80c8018f0080fcc
:10b870000ed1696830460191fff7a0fe40b1304615
:10b880000199fff7d3ff18b137ea080308bf013465
:10b890002d68dfe7029823f043f9204605b0bde8a4
:10b8a000f08370b505460026046a4cb123792bb1ac
:10b8b0002846a168fff782fe00b101362468f4e74c
:10b8c000304670bd08b5fff717ff10b10c30d0e857
:10b8d000af0f08bd08b5fff70fff10b11030d0e86b
:10b8e000af0f08bd0a4608b5036a73b112b1996873
:10b8f000914208d103f10c000021fff7b3fd03f1e1
:10b900001000fff7affd1b68efe708bdd0e8af0ff1
:10b91000704708b50830fff7f9ff013818bf01205c
:10b9200008bd08b50830fff7f1ff043802288cbfc6
:10b930000020012008bd08b50830fff7e7ffc31f4e
:10b940005842584108bd2de9f3410546fff7e9ff8c
:10b9500058b14ff000086846cdf8008023f0b4f8e5
:10b96000002808da02b0bde8f0812846fff7e3ffbf
:10b970000028eed1f6e7009c7cb3606820b301a9f3
:10b98000cdf8048023f0d7f900281ddb019f3b0789
:10b990001ad4666828463146fff710fea0b131463a
:10b9a0002846fff7a9fe78b1037907f001076bb1cc
:10b9b00057b90121304623f017fa002804db4ff471
:10b9c0008031304623f069fa2468d5e7002ffbd098
:10b9d0000121304623f035faf6e7009823f0a0f86d
:10b9e0002046bfe708b50830fff790ff08bd00000c
:10b9f000f0b500f1080504468db028460e46fff765
:10ba000085ff072813d1072e00f0e580002104f1ff
:10ba10000c00fff727fd04f11000fff723fd04f1f0
:10ba20001402c2e8af1f04f11802c2e8af1f731e70
:10ba3000062b1ed8dfe803f00439698793c8cf00ce
:10ba4000002704f11c03c3e8af7f2a213b463a4696
:10ba50003846faf73ffe3b46022200212020cde97e
:10ba600001770097fbf77cf9fbf732fb00f1180335
:10ba70001f60202300272846cde90437fff746ff43
:10ba8000634b644953f8262053f820300292019307
:10ba9000614b1e20009304aa3b46f6f743fe04f1d7
:10baa0000803c3e8af6f0db0f0bd00232a211a468a
:10bab0000120faf70ffefbf70bfb022200f118033f
:10bac0001a602846fff722ff03280ed1072204f14f
:10bad0001c03c3e8af2f00230b22cde901330093f1
:10bae00020200021fbf73cf9c3e72846fff70effb3
:10baf0000128bed1022204f11c03c3e8af2f0023aa
:10bb00000422cde901330093eae7062204f11c0385
:10bb1000c3e8af2f2846fff7f9fe072803d1fbf74c
:10bb2000d7fa0023c36600230a22cde9013300932c
:10bb300020200021fbf714f9fbf7cafa052200f1d7
:10bb400018031a6095e700232a211a460220faf703
:10bb5000c1fdfbf7bdfa032200f11803f1e704224f
:10bb600004f11c03c3e8af2f2846fff7cffe0728d8
:10bb70000fd1fbf7adfa012200f134031a60fbf795
:10bb8000a7fa07460ef0c6fd3b6d01333b650ef08c
:10bb9000c5fd00232a211a460220faf79bfd002347
:10bba0000622cde90133009300212020fbf7d8f8cd
:10bbb000fbf78efa032200f118031a60fbf788faec
:10bbc000c36e0133c36654e700232a211a460320bb
:10bbd000faf780fd4de7052204f11c03c3e8af2fff
:10bbe00000232a211a460420faf774fdfbf770faa5
:10bbf000042200f118031a602846fff787fe072881
:10bc00003ff437af00230722cde90133009367e704
:10bc1000cc840c02ab830c02b5830c0210b5036814
:10bc2000044623b90146084823f010fe20606368eb
:10bc300023b92146054822f00ffb60602046bde88d
:10bc400010400121fff7d4be2dc1000221bf000228
:10bc500010b504460830fff759fe012803d1022130
:10bc60002046fff7c5fe6ff0d10010bd10b50446a9
:10bc70000830fff74bfe012808d0022803d101212c
:10bc80002046fff7b5fe6ff0d10000e0002010bda8
:10bc90002de9f74307460830fff738fe02284bd15d
:10bca000002504213846fff7a3fe6846009522f0e0
:10bcb0000bff041e37db2c46a946ddf80080b8f1e7
:10bcc000000f2bd0d8f8040028b301a9cdf80490b8
:10bcd00023f031f800281edb019e32071bd4d8f870
:10bce000045038462946fff769fca0b1294638467a
:10bcf000fff79cfd78b1f3070dd40121284623f00e
:10bd000073f8002807db4ff48031284623f0c5f88c
:10bd10000028a8bf0134d8f80080d0e7009822f0ae
:10bd2000fffe24b14446204603b0bde8f083052160
:10bd30003846fff75dfef6e76ff0d104f3e7f7b59d
:10bd4000054608300c46fff7e1fd0138012846d9c9
:10bd50002846fff7f0fd88b1fbf7baf906466cb14b
:10bd600000f134031c60012c01d0062c06d10ef02a
:10bd7000d1fc336d013333650ef0d0fc0027032175
:10bd80002846fff735fe6846009722f09dfe041e08
:10bd90001ddb3c46009eaeb1706888b101a90197d9
:10bda00022f0c9ff00280bdb019b1a0708d4db0730
:10bdb00006d50121706823f044f80028a8bf01349b
:10bdc0003668e8e7009822f0abfe1cb13446204606
:10bdd00003b0f0bd02212846fff70afef7e76ff037
:10bde000d104f4e710b5936804461b78083093b18a
:10bdf000fff78cfd04281ad105212046fff7f8fd36
:10be000040212046fff718fd88b106212046bde8f5
:10be10001040fff7edbdfff779fd032807d10121a1
:10be20002046fff709fd012801d80221eee710bde9
:10be30002de9f347002700210646fff753fd68462a
:10be4000009723f0a1fcb842c0f28580b846ddf827
:10be50000090b9f1000f56d0d9f8083013f008045b
:10be600034d103f04103412b30d1d9f80c306bb3fe
:10be7000196859b34d78022d2bd11a7c002a3fd076
:10be80009b68002b3ad0a845b8bfa84699f8100087
:10be9000a74201a9b8bf274622f088feb0b93046b4
:10bea0000199fff729fc034680b10c30d0e8af2f91
:10beb000954202dd2946fff7d5fa03f11000d0e8dc
:10bec000af3f9c4202dd2146fff7ccfad9f8009043
:10bed000bfe70a2d15d1da681c7c8b6943b984b1a0
:10bee00072b1147814f002040bd002240025cae7c2
:10bef0003cb12ab11478c4f34004f7e71c46f5e7d7
:10bf000000242546bfe7009823f051fa06f10c0af9
:10bf1000dae8af9f06f11004d4e8af5f3046fff7d0
:10bf200028fb41465046fff79dfa39462046fff769
:10bf300099fab8f1020f11d0022f16d0002406f1a1
:10bf4000080a5046fff7e2fc072816d1acb90621d3
:10bf50003046fff74dfd02b0bde8f08706f114034f
:10bf6000d3e8af4f012ce7d1e9e706f11803d3e896
:10bf7000af4f631e5c425c41e1e75046fff7c6fcf1
:10bf8000062800d154b95046fff7c0fc0728e2d17b
:10bf9000002ce0d0c84501d1af42dcd00721d7e763
:10bfa000fff746bf38b5936804461b7800f10805d3
:10bfb000d3b12846fff7aafc052807d10621204661
:10bfc000fff716fd2046fff733ff09e02846fff78d
:10bfd0009dfc0728f6d02846fff798fc0628f1d0ec
:10bfe000bde83840fff710bafff77cfc2846fff7a2
:10bff0008dfc07280ad141212046fff71dfc0028af
:10c00000e0d105212046fff7f3fce9e72846fff7da
:10c010007dfc0628e4d1eee738b500f108050446ba
:10c020002846fff773fc072806d12046fff700ffdc
:10c03000bde83840fff7e8b92846fff767fc062857
:10c04000f6d1f2e7d0e88f0fc0b2704770b58cb070
:10c05000fff752fb0e46044670b92023cde90430a9
:10c06000254b2649009304aa03463220f6f75afbd3
:10c070006ff0a9000cb070bd00f114051ab30223d3
:10c0800028468df80c30fff7ddff022807d0284640
:10c09000fff7d8ff042802d00422c5e88f2f202103
:10c0a0000023cde90413164a0092012004aa134983
:10c0b000f6f738fb0023009301233046194603aa04
:10c0c00023f006fcd6e7012328468df80c30fff755
:10c0d000b9ff012809d02846fff7b4ff032804d090
:10c0e000032204f11403c3e88f2f20220023cde99b
:10c0f0000423044ad8e700bfcd830c02ab830c02b3
:10c10000e8830c020a840c02f0b58fb00d46164687
:10c11000fff7f2fa60b92023cde90630164b174934
:10c12000009306aa03463220f6f7fcfa0fb0f0bde2
:10c1300000f114073846fff785ffb3681b78984273
:10c14000f4d0c7e88f3f0df11701284622f0d5fd46
:10c15000202200239df81710cde90623d7e88f2f62
:10c16000d2b2cde90112064a01200092034906aa83
:10c17000f6f7d8fadae700bfcd830c02ab830c02e6
:10c180002d840c021368033b052b0ed8dfe803f067
:10c190000305070d090bfff725befff703bffff7e8
:10c1a0003bbffff7b1bffff7c1b97047fff7eabf69
:10c1b00000232de9f04f93b0054608a80591089398
:10c1c00022f082fc00285fdb089cdff8c8a0dff8c3
:10c1d000c8b0002c55d06068002850d0002309a9b1
:10c1e000099322f0a8fd002849db099b13f00808f9
:10c1f00045d1666828463146fff77efa074680b982
:10c2000059461820a3f052fa0746002837d02b6a67
:10c21000c0e9038880f8048080f814808660036099
:10c220002862059b30463b7100230df11e018df8fd
:10c230001e3023f0e4fb814608bb07f1140840469a
:10c24000fff700ff9df81e10884218d0c8e88f1f26
:10c250000df11f01304622f050fd20229df81f10e5
:10c26000cde90a29d8e88f2f094bd2b2cde90112c6
:10c27000009351464b4601200aaaf6f753fa246868
:10c28000a7e7089822f04cfc13b0bde8f08f00bf80
:10c2900052840c02ab830c0255860e0210b521b9f4
:10c2a0000121fff785ff002010bdfff725fa10b12f
:10c2b00001230371f7e76ff0a900f5e770b50546b4
:10c2c0000c461646faf704ff00f134031e602146bf
:10c2d00028461cb9fff76cff204670bdfff70cfa2b
:10c2e00010b100240471f7e76ff0a900f5e7f7b586
:10c2f000174613f0010205460e461c4605d10b46b3
:10c3000001200521009202f073fc032d0ad0042db8
:10c310000cd0022d0dd1c4f340000ef08bfb002099
:10c3200003b0f0bd00200ef06dfbf8e70ef058fbf7
:10c33000f5e70022394630460ef044fbefe700688f
:10c340000179d0e902230078fff7d1bf012a70b547
:10c35000054603d10b680360002070bd022a08d097
:10c36000032af9d100680028f6d0102112f038fa1b
:10c37000f2e710200e6812f02bfa044618b196e886
:10c380000f0084e80f002c60e6e7000010b50124e0
:10c3900000220d4b1c700d4b1a70fef709fdd0e802
:10c3a000cf3fc0e8424f002af9d1dbb2002bf6d1d3
:10c3b000c2680361c36003754375c0e88f3fd3074c
:10c3c00058bf037a10bd00bf7051001076cf001027
:10c3d0000022014b1a70704770510010024b187800
:10c3e000003818bf01207047705100100b4b28b95e
:10c3f0001a788ab901221a70fff7c8bf032818708b
:10c4000008d80128f8d00022054b1a700122054bec
:10c410001a7001e00428efd0704700bf45d100102a
:10c420007051001076cf0010014b1878704700bf94
:10c4300045d10010014b1870704700bf44d1001067
:10c44000014b1878704700bf44d10010f0b51c466e
:10c45000431e032b06460d46174685b04fd8294a82
:10c46000d35c002908bf1d46274b5b68c3f3080354
:10c470005bb144f00104e9b223463a46f0b2fff75b
:10c4800036ff0025284605b0f0bdf9f76ffc0028ff
:10c49000efd0fef78dfc037a002bead0e307ead455
:10c4a0001a4b93f82c20002ae5d0586a1bf0bdfceb
:10c4b0000028e0d10290102012f08af918b1c0e9ea
:10c4c0000065c0e90274124b00900393114b69465a
:10c4d0000e480293f7f746f8044670b100224ff079
:10c4e000ff3140691bf0bafd236820469b68a569af
:10c4f00098476846f6f73effc4e70546f9e7064d5c
:10c50000c0e700bfec840c0200ed00e070cc00102e
:10c51000bfc20002cdc20002f2feffff70470176eb
:10c520007047417670470368db69184780f825102b
:10c5300070478163828770470164a0f84420704788
:10c540008164a0f84c207047c161704710b5036842
:10c550001446db689847031b5842584110bd08b584
:10c560004068fff7f3ff08bd70b5037a04460d4637
:10c5700016462bb9d0e90312fff7f1ff012323720e
:10c58000324629462046fff7eaff70bd70477047e4
:10c5900070470139012908b505d800211030f7f797
:10c5a00091fa012008bd0020fce713b504460846b7
:10c5b0000191f4f7e7fb013082b22046236801992c
:10c5c0001b6b02b0bde81040184713b5044608467f
:10c5d0000191f4f7d7fb013082b22046236801991c
:10c5e000db6a02b0bde81040184713b504460846a0
:10c5f0000191f4f7c7fb013082b22046236801990c
:10c600009b6a02b0bde81040184710b504460846c2
:10c61000216311b9a086204610bd002a02daf4f782
:10c62000b1fbf7e7a286f6e710b504460846a1621b
:10c6300011b9a085204610bd002a02daf4f7a2fb4a
:10c64000f7e7a285f6e710b504460846a16011b9e0
:10c65000e060204610bd002a02daf4f793fbf7e70a
:10c66000e260f6e710b504460846216111b9606141
:10c67000204610bd002a02daf4f784fbf7e7626176
:10c68000f6e7002201211046fbf78ab900220121ba
:10c690001046fbf785b910b50446502112f0a0f8fa
:10c6a000204610bd10b50446242112f099f820460a
:10c6b00010bd10b504468c2112f092f8204610bd32
:10c6c0004c2200210430a3f09cbdf8b504460d4671
:10c6d000d1b1c8b190f82570b7b101f12406304648
:10c6e000f4f750fb87423a4604f1040138bf024692
:10c6f0003046a5f0c5fb38b994f82c3085f8883061
:10c7000094f82d3085f88930f8bd002108b5022055
:10c7100002f00afd1bf079fcb0fa80f0400908bd78
:10c7200008b50021022002f0fffcbde808401bf024
:10c7300074bc38b500f1100504462846fff7e5ff44
:10c74000e8b1284606f06dfcb0b1284606f05afc68
:10c75000011e11db236820465b69c9b2984758b9ae
:10c76000284606f05efc38b1284606f043fc2368f4
:10c77000c1b21b69204698472846fff7d1ff38bd54
:10c7800038b50c46054601462046a3f013fd284661
:10c790001349f4f7edfa28b912492046a4f001fe36
:10c7a000002038bd28461049f4f7e2fa08b90f49cd
:10c7b000f3e728460e49f4f7dbfa08b90d49ece730
:10c7c00028460d49f4f7d4fa08b90c49e5e728469c
:10c7d0000b49f4f7cdfa0028e2d10a49dde700bfa2
:10c7e000f0840c02f5840c02fa840c0200850c0221
:10c7f0001c820c0206850c0214850c0217850c02a3
:10c8000025850c022c850c0238b503460446124ad5
:10c8100004f1100543f8042b07c983e807002846f4
:10c8200006f046fc0021022002f07efc1bf0e6fb35
:10c830002846fff775ff284606f02efc20b94ff476
:10c840001651284606f024fc044b20462360ff23a3
:10c85000a4f8883038bd00bf54880c02e0880c0270
:10c860004ff0ff30704770b50d46002400f1100600
:10c870002846f4f787faa04205d9295d304606f02c
:10c88000d7fb0134f4e770bd38b5044600f110055c
:10c890002846002306f022fd20460649fff7e3ff65
:10c8a000284606f0befb002803dd284606f0a2fb62
:10c8b000f6e738bd88870c022de9f0436929044664
:10c8c000a5b070d1142500212a4607a8a3f099fc31
:10c8d0000022012107a8adf81c500ef0c9fd00256b
:10c8e0002023cde90c35bdf82c3001200193914b6c
:10c8f000914900930caa2b46f5f714ffbdf82c3094
:10c90000002b3fd08d492046fff7adff03a8f9f774
:10c9100053fa20460399fff7a6ff20468849fff700
:10c92000a2ff2427dff85c82dff81492bdf82c30d8
:10c93000ab421cdd07fb05f60a9b142298590ca993
:10c94000fff71eff88b920460ca9fff78cff414670
:10c950002046fff788ff0a99204631440431fff74b
:10c9600082ff49462046fff77eff0135dee703a838
:10c9700006f08afd002207a811460ef079fd25b0c9
:10c98000bde8f0836f492046fff76dff0ca8f9f76b
:10c9900013fa20460c99fff766ff20466849fff717
:10c9a00062ff0ca8e4e76d293ed16749fff75bff02
:10c9b0005d2200210ca8a3f024fc002204201146d3
:10c9c000faf75afd014638b102882ab15d2a28bf1c
:10c9d0005d220ca8a3f0eefb01220df1870107a850
:10c9e000fef7baf920460799fff73dff07a806f0c2
:10c9f0004bfd0525554f0df18d0639462046fff7b5
:10ca000032ff0122711b07a8fef7a6f920460799fd
:10ca1000fff729ff07a806f037fd013dedd12046bd
:10ca20004749fff720ffaae766290bd110342046bb
:10ca3000474906f0c7fc0021204625b0bde8f04379
:10ca4000f7f740b8782905d10368db6825b0bde861
:10ca5000f0431847732919d13e4b00220f9301234d
:10ca600010933d4b1034119303230d943b4c0ca9b0
:10ca70003b488df838200c941293fcf713fddde948
:10ca800011120ca80c94fff76ffd78e7762908d1f6
:10ca9000344b0c9300f110030ca80d93fcf724fd0c
:10caa000bde74c290ad1002201210420f6f79affa4
:10cab000002025b0bde8f04306f03bbe632910d14d
:10cac000002016f0eafc054627492046fff7cbfe7a
:10cad0002649274b002d08bf19462046fff7c3fe05
:10cae0009de7432917d12349fff7bdfe3f2220468a
:10caf0000ca9fff7c9fe0ca8f4f744f93f2808d1a8
:10cb00000ca816f08bfc1c492046fff7acfe0ca9c4
:10cb1000e3e71a49e1e764297ff431af002200f12d
:10cb20001003009311461046154b0192fcf7e4fcec
:10cb300075e700bf46850c0220740c0266850c0266
:10cb400088870c0272850c0285850c025e730c02cc
:10cb5000a2850c02dca30c02e2850c02d4880c0234
:10cb600021450002c8880c02e6850c023f850c02b4
:10cb700043850c02f7850c0213860c0227860c02f3
:10cb8000cdc400029a9e0c022de9f041044600f14a
:10cb90002407bab021220021384604f14505a3f04c
:10cba00030fb412200212846a3f02bfbff2300216c
:10cbb000a4f88830674b4c22a4f8861027a8269347
:10cbc000a3f01ffbdff8bc8104f186064146204636
:10cbd000fff749fe202239462046fff755fe94f81c
:10cbe0002430002bf2d021465b480ff07bff94f8f5
:10cbf0008830ff2b12d1dff8908141462046fff7a5
:10cc000032fe012231462046fff73efe94f8863080
:10cc1000303bdbb2032bf0d884f8883094f88830ae
:10cc200013b1312384f845304ff0ff32394626a83e
:10cc3000fff709fd4ff0ff32294626a8fff712fd46
:10cc4000b4f888304c22adf8b030032327a90deb9f
:10cc500002008df8bc302792a3f0acfa4c22684653
:10cc60000deb0201a3f0a6fa01226946a368e06871
:10cc70009847023002d094f88930e3b9374f3946eb
:10cc80002046fff7f0fd012231462046fff7fcfd6c
:10cc900094f88620a2f13103022bf0d8322aa2f1b7
:10cca000300302d0032b18bf012384f8893094f895
:10ccb00089308df8b13094f88830013b022b0ed8c2
:10ccc00020462749fff7cffd402229462046fff79f
:10ccd000dbfd4ff0ff32294626a8fff7c3fc2046b4
:10cce0002049fff7c0fd4c22032327a90deb0200ca
:10ccf0008df8bc302792a3f05dfa4c2268460deb0c
:10cd00000201a3f057fa00226946a368e068984739
:10cd1000f0b920461449fff7a6fd20461349fff756
:10cd2000a2fd20461249fff79efd20461149fff75c
:10cd30009afd11492046fff796fd10492046fff75e
:10cd400092fd236820469b6998473ab0bde8f08180
:10cd50000b49f3e778880c024bc600029e860c0252
:10cd6000ca860c02d5860c0208870c0228870c02a2
:10cd700058870c028b870c02ca870c02fe870c02b4
:10cd800017880c026a860c0271860c02772908b596
:10cd900003d1bde80840fff7f7befff78dfd08bde2
:10cda000d0e88f0fc0b2003818bf012070470000d4
:10cdb0000048704748d1001008b5fff7f1ff08bde3
:10cdc0007fb50546fff7ecffe0b1686810b1036876
:10cdd0009b68984715f06bfbeb68c01ab0f57a7f3b
:10cde0000ed315f064fb00240646aa682346821a77
:10cdf00000210420cde901440094f9f7b1ffee6071
:10ce0000002001e06ff0d10004b070bd38b51420ef
:10ce10000d460021144602f05ff9014640b1054b72
:10ce20000573046143600448faf75aff002038bdd7
:10ce30000248fce721d00002f4d60010fcfeffff00
:10ce400010b514466ab971b1134604200a4621464a
:10ce5000faf714fc002805db224602210348fff7fd
:10ce6000d5ff002010bd0846fce700bf48d10010e8
:10ce700030b58bb0fff794ff002857d00024202353
:10ce8000cde902342b4b1e202b49009302aa2346e6
:10ce9000f5f748fc21460920f9f7d0fc08b30469ee
:10cea000002214210120f9f7d3fc28220221034695
:10ceb000cde9002102a82146012206f05dfc0022f6
:10cec000012103a8f5f712fd1a24013c0bd09df8af
:10ced0001a30322083f002038df81a3012f0adfbc5
:10cee000f3e7ff24dce7fef7e1fa2146fef7acfbaf
:10cef0000446a8b14ff47f031a2507939df81a3012
:10cf000003f0fd038df81a30013d09d09df81a3069
:10cf1000322083f002038df81a3012f08efbf3e713
:10cf200002a8fcf70dff20460bb030bd6ff0d10416
:10cf3000f9e700bf0a890c02fc880c020368016053
:10cf40001bb11a68184652681047704730b58db04b
:10cf50000546fff769fa042807d12846fff720ffa6
:10cf6000044650b16ff0d10049e009200df06cfe8d
:10cf70000028f2d06ff0810041e00123c5e88f3f27
:10cf80002023cde904301f4b1f49009304aa034618
:10cf90001e20f5f7c7fb23462246042101200094fa
:10cfa00001f026fefef782fa0721fef7c8fe2346af
:10cfb0002246a2210920f9f78dfb234622460021b3
:10cfc0000220cde901440094f9f7cafe15f06ffa8a
:10cfd000c5e9020000f0c4f800f0c6fc0b4b8c2041
:10cfe00004940694059311f0f3fb044610b104a9d0
:10cff000fff70afc281d2146fff7a0ff00200db017
:10d0000030bd00bf24890c02fc880c02c1cd000297
:10d0100030b58db00546fff7c3fe48b3002420238a
:10d02000cde90434144b04aa00931e20234613496f
:10d03000f5f778fb224621460920f9f75dfb2146ea
:10d04000281dfff77bffc5e88f4f15f030faaa685f
:10d050002346821a00210820cde901440094f9f703
:10d060007ffe00f07df800f013f920460db030bdd2
:10d070006ff0d100fae700bf3c890c02fc880c027b
:10d08000022906d0032906d0012906d10021fff785
:10d090005dbffff7bdbffff7ebbe6ff077007047d6
:10d0a00013b5047b02690021019202f027f82146a2
:10d0b000019a034802b0bde81040fff7e1bf00bf8e
:10d0c00048d100100022024b1a705a60704700bf0e
:10d0d00048d1001010b50378044613b100201cf0ad
:10d0e00035fb204610bd00004ff0fa73194a10b509
:10d0f000c0e90023184b00f10d0283600023037385
:10d10000164b03f1100153f8044b8b4242f8044bc9
:10d11000f9d102220023426540f26262c0e908337d
:10d12000c0e90a33c0e90c33c0e90e33c0e9173354
:10d13000c0e91933c0e91b33036480f84430c0f8f8
:10d140004630c0f84a30c0f84e30a0f85230a0f84f
:10d15000582010bd18002800200064004b610c020c
:10d1600010b50a4cd4e88f3fdb070cd4204613f0ef
:10d17000cdfb40b10648fff7b7ff204613f000fc97
:10d180000448a2f0f0fd024810bd00bf58d10010c5
:10d190005cd1001015d5000290f85700704780f858
:10d1a00057107047a0f858100020704773b5374be0
:10d1b00005461e78002e65d130468df804601cf0bf
:10d1c00097fad5e90801012332468df804301ef0a4
:10d1d00037fa041e2bdbd5e90b0132461ef07afa32
:10d1e000041e24db314605f146001cf0a2fb041ea0
:10d1f0001ddb314605f138001ef0daf9041e16db9e
:10d20000314695f944001cf0dcfb041e0fdb31466f
:10d2100095f854001cf037fc041e08db95f85210fa
:10d2200059b1314630461ef049fc90b1002401a8a6
:10d23000fff750ff204602b070bd95f853306bb138
:10d2400008461ef03bfc0028f0d195f85430022b24
:10d2500014d11ef07cfa00eae074e8e7194618469b
:10d260001ef02cfc50b195f85430022bded1012079
:10d27000002185f854001cf006fcece700201cf0af
:10d2800018fce8e76ff0d104d4e700bf715100103b
:10d2900070b51b4e044635788cb06dbb28468df8b2
:10d2a0000c501cf025fa012328468df80c301cf098
:10d2b00071fa94f8563083b1204684f85650fff73f
:10d2c00075ff50b12023cde904350e4b3220009379
:10d2d0000d492b4604aaf5f725fa002221460b48f2
:10d2e0001cf07bfa01233370002303a863622363dd
:10d2f0002366e366fff7eefe00200cb070bd00bfb2
:10d300007151001065890c0253890c027dd4000212
:10d31000f0b52d4b06461d7889b0002d50d128461a
:10d320008df804501cf0e4f9012328468df80430f0
:10d330001cf030fa041e38db0c2733882946adf880
:10d340000c30738802a8adf80e30f388adf80850a1
:10d35000adf81230b388adf80a70adf810301cf09b
:10d36000e8fa041e21db33892946adf818307389a9
:10d3700005a805950795adf81670adf81a301ef0a2
:10d3800017f9041e11db294602201cf07cfb041e49
:10d390000bdb294696f90c001cf013fb041e04db82
:10d3a00028461cf0f5f9041e08da3046fff770ff36
:10d3b00001a8fff78ffe204609b0f0bd2c46f7e725
:10d3c0006ff0d104f7e700bf71510010037a2bb959
:10d3d00003681b7813b94068fff75abf7047000015
:10d3e000f0b52a4b05461b7885b0002b3fd190f84d
:10d3f000523013b990f85330cbb395f855607ebbdb
:10d40000012730468df800601cf072f90df103031e
:10d410003046cde901358df800708df803608df848
:10d420000c601cf0b7f9041e24dbd5e90801324674
:10d430001ef006f9041e1ddbd5e90b0132461ef075
:10d4400049f9041e16db30461cf0a2f9041e11db5c
:10d4500001a88df80370fff7b9ff6846fff73afea1
:10d4600095f8553083f0010385f855305bb96ff0be
:10d47000d10405e001a8fff7a9ff6846fff72afedf
:10d48000204605b0f0bd0024fae700bf715100103e
:10d4900073b5194b06461d7855bb28468df80450c8
:10d4a0001cf026f9012328468df804301cf072f98f
:10d4b000041e12dbd6e917012a461ef0c1f8041e2d
:10d4c0000bdbd6e91a012a461ef004f9041e04db20
:10d4d00028461cf05df9041e08da3046fff7d8fe36
:10d4e00001a8fff7f7fd204602b070bd2c46f7e714
:10d4f0006ff0d104f7e700bf7151001030b5144b45
:10d500000c461d788bb0adb90368012b12d10846cb
:10d51000fff766ff80b12046fff7baff60b1202316
:10d52000cde902350b4b00932b4632200a4902aa63
:10d53000f5f7f8f80bb030bd00201ef008f9002810
:10d54000f8d020220023cde90223044a0092ece720
:10d55000715100108b890c0253890c02c1890c0295
:10d5600010b504460068a2f0fffd204610bd10b5be
:10d5700004466830fff7f4ff04f15c00fff7f0ffaa
:10d5800004f12c00fff7ecff04f12000fff7e8ffa7
:10d59000204610bd0148fff7eabf00bf5cd1001074
:10d5a00003680a6802600b6043684a6842604b6027
:10d5b00083688a6882608b607047002310b50446d8
:10d5c000c0e900338360fff7ebff204610bd38b59c
:10d5d0000d1e0446006803dda3f094fd18b938bda4
:10d5e000a2f0c2fd00202060a5600120f7e770b521
:10d5f00000260d1e0446c0e9006686600bddfff7bd
:10d60000e6ff40b123685a199a4203d003b11e7055
:10d610000133f9e76560204670bdf8b5d0e90153e4
:10d620009d4204460e460cda276862687919521b3f
:10d63000481ca2f0ccfd01207e5563680133636075
:10d64000f8bd691cfff7c3ff0028edd1f8e72de90d
:10d65000f041476883688846b918994204461546e0
:10d6600012dc266862683e443146d21b7019a2f073
:10d67000aefd2a4641463046a2f09cfd012062687c
:10d680002a446260bde8f081fff7a1ff0028e8d1dd
:10d69000f8e7000070b5674b06461c7898b0002c80
:10d6a00040f0c580022104a8cde90444cde9064438
:10d6b000cde90844fff7b1ff48b95f4d07a8fff770
:10d6c0004fff04a8fff74cff284618b070bd01219a
:10d6d00004a8fff7a2ff0028efd0062104a8fff757
:10d6e0009cff0028e9d01122214613a81294a2f031
:10d6f00088fd2246152112a81cf0ddf8051edddb91
:10d7000012a8f3f73ffb0130c1b204a8fff785ff71
:10d710000028d2d0092104a8fff77fff0028ccd031
:10d7200012a8f3f72ffb12a9024604a8fff78ffff8
:10d730000028c2d02023adf80430b6f858300621b6
:10d7400002a8adf806300294adf80c4018f05ffc6a
:10d75000051eb3db0b2104a8fff75fff0028acd048
:10d76000ff2104a8fff759ff0028a6d002220df1df
:10d77000060104a8fff76bff00289ed0022201a932
:10d7800004a8fff764ff002897d0062202a904a886
:10d79000fff75dff002890d0f6f7d8ff00f11801e1
:10d7a0000da802f001fc9df84430012b2fd111216e
:10d7b00007a8fff732ff00283ff47faf072107a833
:10d7c000fff72bff00283ff478af10220da907a820
:10d7d000fff73dff00283ff470af04a90aa8fff748
:10d7e000ecfe0aa906f15c00fff7dafe0aa8fff7d3
:10d7f000b7fe07a90aa8fff7e0fe0aa906f168002c
:10d80000fff7cefe0aa8fff7abfe002556e703217f
:10d8100007a8fff702ff00283ff44faf032107a836
:10d82000fff7fbfe00283ff448af0222cee76ff07f
:10d83000d10549e771510010fcfeffff38b5436880
:10d8400005468b420c4612da836899420adcd5e918
:10d8500000230021134422449a420ad003b11970d4
:10d860000133f9e7fff7b3fe0028f0d138bd0029f6
:10d87000fcdb6c60fae70000f0b53a4b05461e7819
:10d880008bb0002e6ad11f2101a8fff7b0fe1f2127
:10d8900004a8fff7acfe32461f2101981cf0bff828
:10d8a000041e52db214601a8fff7c8ff32461f21a4
:10d8b00004981cf0cef8041e47db0c27214604a870
:10d8c000fff7bcff31466f8705f138001cf08ff879
:10d8d000041e3adb314605f144001cf07df8041ebd
:10d8e00033db3146a5f8487005f146001cf039f8e5
:10d8f000041e2adb314605f154001cf0cff8041e4b
:10d9000023db30461cf0ecf8314685f852003046f7
:10d910001ef0d4f801a985f8530007a8fff74dfec3
:10d9200007a905f12000fff73bfe07a8fff718fe47
:10d9300004a907a8fff741fe07a905f12c00fff78e
:10d940002ffe07a8fff70cfe344604a8fff708fed9
:10d9500001a8fff705fe20460bb0f0bd6ff0d10423
:10d96000f9e700bf7151001037b50024264b05467a
:10d9700020461c708df804401bf0bafe012320469f
:10d980008df804301df08aff20b10a201f4a20497b
:10d99000f3f706fb00201bf0fbfe041e2fdb2846de
:10d9a000fff778fe041e2adb2846fff765ff041efa
:10d9b00025db0123284685f85630fff769fd041e54
:10d9c0001ddb2846fff7a4fc041e18db00222946b5
:10d9d00010481bf0e7fe041e11db95f8523033b1fe
:10d9e000002401a8fff776fb204603b030bd95f870
:10d9f00053000028f4d11df0aafe041ef0da2846d8
:10da0000fff746fcede700bf71510010bff50102c2
:10da1000e4890c027dd40002c0687047c268406887
:10da2000101a704710b500200c4614f033fd4ff467
:10da30007a720023f2f7f8ff2060002010bd70b565
:10da4000202488b0224606460d4668460021a2f0f2
:10da5000d8fb00216846adf800400df0cdf9044632
:10da600030b96846b36998472860204608b070bd51
:10da70006ff06300fae70000012208b5094b1a7045
:10da8000fef7d2fc01280cd1f8f770f928b9064b43
:10da90001b7813b9054b1b781bb1bde80840fcf798
:10daa000afb908bdc4d2001035cb001034cb001084
:10dab000fff7e2bf438c8b422cd890f82030012b2b
:10dac00016d0022b11d03bbb90f82430013bdbb2c7
:10dad00080f82430c3b1012380f820304ff4af73b5
:10dae00043844ff420634361704790f824203ab197
:10daf000002380f82030322343844ff47f43f2e741
:10db000011460430f4f7f2be022380f8203040f2d0
:10db1000ee23e5e75b1a43847047012a08bf0160e2
:10db20000020704710b50446024b0360fcf708f96b
:10db3000204610bda08a0c020148fff7f3bf00bfca
:10db400078d2001010b50446fff7ecff20462821dc
:10db500010f046fe204610bd10b50446024b03608f
:10db6000fcf7eef8204610bdb48a0c020148fff71e
:10db7000f3bf00bfa4d2001010b50446fff7ecffbe
:10db80002046202110f02cfe204610bd028c0023e0
:10db9000042130301af09cb9024610b508b10020bb
:10dba00010bd0146f9f747fd0028f8d1054c238840
:10dbb0009bb2002bf3d014f07afc2388c01a80b2f9
:10dbc000eee700bfd8d1001070b58eb02a4905a885
:10dbd00005f0d0f905a805f04df9b5eec00af1ee53
:10dbe00010fa47db05a805f045f9b3ee047ac0ee5c
:10dbf000077af8fe677afdeee77a17ee905a1f4e25
:10dc0000d6e88f2f12f001021d4c1cd13046039232
:10dc100012f07cfe039ab0b114210f20f8f718fe21
:10dc20001e2202210346cde9002120460f226ff07b
:10dc30007f4105f0a1fd134b3046236012f0a0fe9a
:10dc40001148a2f090f8002210481146f4f74efe59
:10dc5000022384f8203040f2ee2363844ff42063e3
:10dc600000220121094884f824506361f4f73efe44
:10dc70000eb070bd0025c2e744d70010d0d100100f
:10dc800078d20010a08a0c02b9da00027cd200100f
:10dc900008b50023a2211a460c20f8f71bfd01222b
:10dca000024b1a70bde8084001f00abac5d2001054
:10dcb00010b5094c2378012bdab204d0022a07d020
:10dcc0000023237010bd0028fcd1fff77dfff7e78c
:10dcd000fff7defff4e700bfe0d100101fb500231f
:10dce00010490a780b70104902f0ff040b60bab1ba
:10dcf00001220093cde901324ff400502246002169
:10dd0000f9f72ef8094b1c70094b5868c0f308004e
:10dd1000003818bf012004b0bde81040fff7c8bfad
:10dd200004b010bde8d10010ecd10010e0d100101b
:10dd300000ed00e030b51d2885b025d9b0f5fa7f9b
:10dd400004d305b0bde83040fff7c8bf104c2378be
:10dd50000133dbb223702378042b17d814f0a7fb10
:10dd60004ff47a7200250b4b18600b4b1a6000239e
:10dd700001214ff48050cde9013122780021009338
:10dd8000f8f7eeff002ddcd105b030bd0125eee740
:10dd9000e8d10010e4d10010ecd100107fb50646a8
:10dda0002a4de0b1002211461046f9f744fc284cf8
:10ddb000207014f07cfb80b22880227802f0ff03f0
:10ddc00042b901228020cde9013200211a46009398
:10ddd000f8f7c6ff00221f4b1a7004b070bd2b88e5
:10dde0009bb2002bf9d014f062fb2c883246041b46
:10ddf00031463046a4b2f9f71efc60b90123009009
:10de0000cde901032246034600218020f8f7a8ff50
:10de10002046fff78fff41f286330022a4f6b93483
:10de2000a4b29c422a80d8d8094b1b78002bd4d0ae
:10de300011461046f9f7fffb00220028cdd0012142
:10de4000104604b0bde87040f9f7aabdd8d1001063
:10de5000f0d10010f1d10010012802d80846fff7d8
:10de60009dbf704710b5394c2288013a92b222808a
:10de70002ab911461920f4f7a5fd19232380344c43
:10de80002388013b9bb223801bbbfcf717fd4ff49b
:10de90007a7323802f4b1a68b2f57a7f51d3002210
:10dea0001a600cf041fc4ff6ff7010f04dfa2a4c4e
:10deb00012f072f82368002b47d014f0f8fa274bc1
:10dec0001a682368801a98423fd9bde81040fff7ce
:10ded00005bf002211461046f9f7adfb80b142f2b2
:10dee00010700cf05cfd58b11d4b197801f0ff0269
:10def00031b90121104619700321f9f7a3fbc9e7d5
:10df0000002211461046f9f796fb0028c2d140f6d0
:10df1000b8300cf044fd0028bcd0124b1b7803f045
:10df2000ff04002bb6d101f0cbf82046fff736fff7
:10df3000204622462146f9f733fd0120fff72eff48
:10df4000a8e71a6801321a60b1e710bd72510010db
:10df500074510010dcd10010ecd10010e4d100109d
:10df6000f1d10010f0d1001013b501200cf078ffb2
:10df7000ff281ed0c3071cd50420fef737fa002166
:10df800000240846fef756fa224604200df1070148
:10df90008df80740f5f73efd9df807304bb122465e
:10dfa00021460420f5f71efd224621462046f9f7ba
:10dfb000f7fc02b010bd000010b50446fef734fabd
:10dfc000022801d0002010bd002cfbd1fef706fa7c
:10dfd0000028f7d0f7f7cafe0028f3d1024b1878d3
:10dfe000b0fa80f04009eee776cf001030b50d4d65
:10dff00002462c7885b034b108200b4a0b49f2f761
:10e00000cfffa1f0a9fe01234ff48020cde9014309
:10e010002b70002123460094f8f7a2fe2c7005b067
:10e0200030bd00bfa0d20010bff50102268a0c024d
:10e0300001287fb50c463fd00a2843d1224dd5e8b0
:10e040008f2f12f001021cd12846039212f05efcc1
:10e05000039ab0b114210220f8f7fafb02221e2124
:10e060001a4e0346cde9001230466ff07f4105f0ad
:10e0700083fb174b2846336012f082fc1548a1f051
:10e0800072fe14f0010212d000210846f8f7d6fb08
:10e0900050b10369002201210c484361043004b0ef
:10e0a000bde87040f4f722bc6ff07f43f2e7a307ae
:10e0b00008d511460848f2e7084604b0bde87040ac
:10e0c000fff794bf04b070bdd4d10010a4d20010eb
:10e0d000b48a0c02edda0002a8d2001070b5044632
:10e0e00086b0062010f030f9002c65d1204600f0f3
:10e0f00053ff3e4b1b78002b5ad1fef76ff90028d7
:10e1000056d0f7f733fe002852d1394b1b78002b3d
:10e110004ed1fef789f901284ad106b070bdfef74d
:10e1200047fefef749fe0028f7d14ce0072010f02b
:10e130000bf9fef779f9042801d0f2f7f9fe012373
:10e140002c4e2b7096f82c303bb9fff795fc2046ef
:10e15000fff732ff0028e0d139e0706a19f065fe60
:10e1600005460028f1d1244b14200593234b04933a
:10e1700010f02efb044690b1214b02a940f8043b5d
:10e18000f7f724fb1f4b3046236001a90194f7f7f2
:10e19000a6fa40b1706a10b1294619f073fe02a8c0
:10e1a000f5f7e8f8b9e7236820469b689847f6e753
:10e1b000154b1b78002bb0d12046fff7fdfe002841
:10e1c000abd1002cabd00a4d2b78012baed108205f
:10e1d00010f0baf8fef728f904289ed0f2f7b4fe42
:10e1e000092006b0bde8704010f0aeb876cf001040
:10e1f000a1d2001070cc001031da00029bda0002cc
:10e20000f4730c0208740c0237cb00100120fff7e6
:10e2100065bf000030b593b020f032fcf2f77cfe11
:10e220000cf042fb002000f025fa052010f08cf8dd
:10e2300000232a211a461846f8f74cfa22f0fcfe71
:10e24000474bda88012a04d100229a71da7122f050
:10e250000ffff4f7a7ff002200242025114602201b
:10e26000f4f760fd06a8f7f7a7fd069b3d4901936b
:10e270003d4b0aaa1e2000932346cde90a54f4f729
:10e2800051fa20461ff026f91ff028f922460120f6
:10e290003449f4f705fbb0b1224605a904a8cde93d
:10e2a00004440cf021fc70b9049b63b1059acde9dc
:10e2b0000a50cde901322d4b2a4900930aaa0346a0
:10e2c0000120f4f72ffa10f033fcf6f73ffaf6f7d7
:10e2d00027fafff749fe18f0b3fd254818f066ff4e
:10e2e0000020fef7adf860b3fef79ef8041f18bfdc
:10e2f00001240021084614f0cbff012807d8642030
:10e3000011f09bf90022462011460cf05bfb2046e1
:10e3100000f0eef9174db4b11748fff737fc164877
:10e32000f9f790fc2846fff731fc002019f07bfd3f
:10e3300068622846f9f7bbfc06a805f0a5f813b0fb
:10e3400030bd0446d5e7204619f06dfd0a4b5862f2
:10e35000204619f068fd68620020fff7bffefbe76a
:10e36000b8000c0020740c02328a0c02448a0c02a1
:10e37000813a000244d2001070cc00102de9f04325
:10e380003d4b8db000933d4b694603933c4b04a835
:10e3900000250293f7f71afa4ff44063cde90835e8
:10e3a00041f28833374c0a930223204614268df815
:10e3b0002e30354b04a940f8043badf82c60f7f73c
:10e3c00005fa089b65626361099b04f12800a3615b
:10e3d0000a9bdff8f480e361bdf82c302b4f2384d7
:10e3e0009df82e30dff8e49084f8223019f0d1fd4a
:10e3f000274b84f82c502360256304a8f4f7baff58
:10e400006846f4f7b7ff2946224814f055f8224c25
:10e41000224b2946a360224bc4e90086c4e9033499
:10e420006761201df4f7fcfb1e4b294623601e4c40
:10e430001e4bc4e90086a3601d4b6761c4e9033429
:10e44000201df4f7edfb1b4bc4f80090a3611a4ca0
:10e450001a4b2946a3601a4bc4e90086c4e9033469
:10e460006761201df4f7dcfb164bc4f80090a36134
:10e470000db0bde8f08300bf8de10002df56000261
:10e48000cb56000244d2001088770c02e96d0002de
:10e49000908a0c02b1df0002f4d1001006000200e5
:10e4a000698a0c02c88a0c0228d2001019000100e7
:10e4b000748a0c0299d900020cd200101a000100d3
:10e4c0007d8a0c029dd90002c4780c02d88a0c0205
:10e4d000f0b50246406890b10831d46821f00303da
:10e4e0009168201a091a043399424ff0000107d3aa
:10e4f000c4e90013d1680b4401f10800d360f0bdfa
:10e500000d460846146974b166689e4205d338b159
:10e510004768be423cbf0d46204621462468f2e7cc
:10e520000d462046f9e70028e9d003684db12b607d
:10e530002b465169814208bf5361002340f8083bd4
:10e54000dde71361f5e7704710b50446182110f0b8
:10e5500047f9204610bd0000014b586a19f065bc10
:10e5600044d20010012a38b5044602d10b6823605a
:10e5700003e0022a03d0032a0dd0002038bd0c206e
:10e580000d6810f025f903460028f0d095e8070043
:10e5900083e80700ebe700680028eed00c2110f0bc
:10e5a0001ff9eae730b5002939d051f8044cc268a8
:10e5b000a1f108031d19aa4214d1121bc260002444
:10e5c000426962b35168c3685518ab4227d15b1ae0
:10e5d000c360036913b119688a421cd14361e3b96e
:10e5e0000361ede7056900222c4624b19c4238bf47
:10e5f00022462468f9e72ab905b9436141f8085c65
:10e600000361dce7146841f8084c136041699142ea
:10e61000d5d14361d3e70b46dce71c60d0e730bdc2
:10e62000438c8b4223d890f8203013b1012b0ad0b1
:10e630007047012380f82030fa234384837c43f021
:10e6400002038374704790f82420013ad2b280f814
:10e65000242042b1002380f82030fa234384837cb5
:10e6600003f0fd03ede711460430f4f73fb95b1a00
:10e670004384704738b50c4cd4e88f3f13f0010f3a
:10e680000a4d09d1204612f041f928b119f01efcbb
:10e690002860204612f074f919f018fc2b681b1a38
:10e6a0005842584138bd00bfccd2001024d70010ca
:10e6b00010b50446024b0360fbf742fb204610bd39
:10e6c000848c0c020148fff7f3bf00bffcd600109a
:10e6d00010b50446fff7ecff2046282110f080f823
:10e6e000204610bd014b586a19f09fbb70cc00103a
:10e6f000002210b5044611461046f8f7affe6cb183
:10e70000fdf792fe042805d100231a461946184643
:10e71000f9f7d0f9bde81040fcf70eb9fdf784fe1b
:10e720000128edd1f0e7000008b5064b1b78032b5c
:10e7300006d104f0d7fcbde808400021f5f7c2b9c6
:10e7400008bd00bf37cb001070b52d4a8cb01378d0
:10e75000002b52d00023157813702022cde904231a
:10e76000284aedb2009228202749019504aaf3f720
:10e77000d9ff264cd4e88f2f12f001021dd120467c
:10e78000039212f0c3f8039ab8b114210f20f8f7de
:10e790005ff81e2202211e4e0346cde900213046bd
:10e7a0000f226ff07f4104f0e7ff1a4b20463360e1
:10e7b00012f0e6f81848a1f0d6fa012d1bd8e5b101
:10e7c0004ff47f060022124c1146201df4f78ef8fc
:10e7d000fa230022012166616384a37c201d03f0db
:10e7e000fd0384f8245084f82020a3740cb0bde805
:10e7f0007040f4f77bb8094ee4e70cb070bd00bf81
:10e80000c6d20010e08a0c0220740c02c8d200109c
:10e81000fcd60010848c0c0245e600020060ff006c
:10e82000002270b5314d8cb007200df10f018df82d
:10e830000f20f5f7eff82b685a1c2a601bb913f06c
:10e8400036fe2b4b18609df80f301bb313f02ffed4
:10e85000274e3368c01a274b98421bd90024202327
:10e86000cde9043405230193234b04aa0093282007
:10e8700023462249f3f756ff0122214b34601a70d8
:10e88000204b2c601c709df80f300bb91e4a136092
:10e890000cb070bdf6f798fc1c4cc8b110f1aa0f73
:10e8a00014d01b4a1b4b10f1a00f08bf1a460023bf
:10e8b00020210192184acde90413009228200f4923
:10e8c00004aaf3f72fff02232370dce7134aeee7d5
:10e8d0002023cde90430124b0849009304aa0346d3
:10e8e0002820f3f71fff0323eee700bf28d700100f
:10e8f000d4d20010df930400fd8a0c0220740c02b5
:10e9000075cf0010d8d2001000d00010c6d2001071
:10e910003e7e0c0260680c024b8b0c02f98a0c02e2
:10e92000648b0c0208b5074a1378ff2b1cbf013318
:10e93000137013f0bcfd044b1860bde80840fff7ee
:10e940006fbf00bfd8d20010d0d2001000222de936
:10e95000f04111468cb01046f8f7b0fd00287ed08b
:10e96000404b1b78002b7ad13f4f3b7803f0ff04dc
:10e97000002b74d12346224652210520f7f7aafe28
:10e9800013f095fd394b1d68394b451b1878faf784
:10e99000a3fa854263d34ff02008364b04aa3649c8
:10e9a00000931e202346cde90484f3f7bbfefcf759
:10e9b000fbf90122054600f118031a6040202346a6
:10e9c0000021cde901440094f8f7caf9eb6e013358
:10e9d000eb66f6f7b9fa061e10db01233b70274bf6
:10e9e0001e2000932449234604aacde90484f3f7aa
:10e9f00099fe0cb0bde8f041fff7a6be204b019692
:10ea00000093282023461c4904aacde90484f3f787
:10ea100089fee63609d1224621460620f7f76cfe2c
:10ea2000224621460520f7f767fe002305f118026c
:10ea30003b70136040201a46cde90133009300215a
:10ea4000f8f78ef90f4b1b7803f0ff023bb9114624
:10ea50001046f8f7f0fd10b9fff764ffc9e70cb0f6
:10ea6000bde8f08176cf001036cb0010d0d2001078
:10ea7000d8d200108c8b0c0220740c029e8b0c02de
:10ea8000b58b0c0275cf001008b503200cf0dcf834
:10ea9000034b1870bde8084080f00100fbf766bf2b
:10eaa0002cd7001008b5fef783f9fef785f948b1b9
:10eab00009200cf0c9f828b1fef77af9bde8084042
:10eac000fef7a6ba08bd08b5002000f0e9fd40b188
:10ead00009200cf0b9f8014618b9bde8084000f06b
:10eae0004bbe08bd2de9f74f0d460446002855d012
:10eaf000dff8b8804ff47a79d8f80030dff8b0b09a
:10eb00000344c8f8003013f0d2fc064613f0cbfce7
:10eb10000746002010f091fd0bf006fe13f0c7fc35
:10eb2000a0eb060a544533d3621e924510d34ff42e
:10eb30007a7000fb04741b4d13f0b5fc201aa84238
:10eb40002cd84008012828bf012010f078fdf3e7f9
:10eb5000012010f072fd144b1a78002adcd1002d30
:10eb6000dad1ca4504d2d8f80020b2f57a7fd3d3df
:10eb70000020fdf765fc0af57a790190f7f706f9b0
:10eb800001980028c8d19bf80030002bf5d1c3e7cd
:10eb900025b903b0bde8f04ff7f7f8b803b0bde80a
:10eba000f08f00bfa086010076cf001030d7001094
:10ebb00037cb001013b50c4b0446586a019119f07d
:10ebc00034f958b1094b01995b68c3f308032bb9b9
:10ebd000204602b0bde81040fff784bf204602b0d7
:10ebe000bde8104010f029bd44d2001000ed00e057
:10ebf0002de9f04fdff8b0b193b005939bf80030ea
:10ec000080460e469246604f1bb93b78002b00f0c1
:10ec1000ad8020230024cde90a345c4b1e205c49e2
:10ec200000930aaa2346f3f77dfdfcf7bdf83b7875
:10ec30000546b3b1c4663eb100f134031e60012e37
:10ec400002bf036d01330365032205f118031a6047
:10ec50000023092240200021cde901330093f8f779
:10ec60007ff8fcf7a5f84ff00102d0e8cf3fc0e8ed
:10ec7000412f0029f9d1dbb2002bf6d1c26801691e
:10ec8000047d90f81590c360036103754375c0e877
:10ec90008f3fd3075cbf047ae4b2930758bf416843
:10eca00053073b7858bf90f8099018f0010f08bf40
:10ecb000002413b3002c5fd01023adf81830059b4f
:10ecc000adf81a60adf81e301c9badf81ca0cde964
:10ecd000083105f0c7fa0022022106ab05f0b7f8ab
:10ece00058b120220023cde90a232a4a019000923c
:10ecf000282027490aaaf3f715fdb9f1000f01d022
:10ed0000fbf740fa18f0020f02d12046f6f7fef9a1
:10ed10000024214b3c701c70204b224621460720ca
:10ed20001c708bf80040f7f7e7fc224621460620ce
:10ed3000f7f7e2fc224621460520f7f7ddfc202309
:10ed4000cde90a34164b0aaa00931e202346104927
:10ed5000f3f7e8fc224605f118031c604020234627
:10ed60000021cde901440094f7f7faff00220d4b92
:10ed70001a7013b0bde8f08f05f074fa23462246ee
:10ed8000032105f064f8b8e733cb0010d88b0c02f0
:10ed900020740c02ed8b0c0235cb001034cb00102c
:10eda0001f8c0c02c6d2001036cb0010f0b5634b9e
:10edb00005461b788db0002b00f0bd80604f3b787e
:10edc000002b40f0a1805f4b1b7803f0ff04002b69
:10edd00040f09a805c4e327802f0ff03002a3dd06a
:10ede000fbf788ff002800f097802023cde904344a
:10edf000564b04aa564900931e202346f3f792fc73
:10ee000001233b70534b34701c70fbf7cdff022283
:10ee100000f118031a600822234600214020cde9a2
:10ee200001440094f7f79cfffdf7fefa04282346ff
:10ee300022464ff052010cbf08200720f7f74afc8a
:10ee4000002205201146f7f757fc00220620114644
:10ee5000f7f752fc0022404b1a6055e01a46522147
:10ee60000620f7f737fcfff70ffe04460028f1d025
:10ee70003a4b1b7803f0ff02002b3ad111461046a3
:10ee8000f8f7d9fba8bbfff74dfd062c46d0082ca0
:10ee900014bf4ff47f074ff0ff1700262023cde962
:10eea00004362f4b28202a49009304aa33460194a4
:10eeb000f3f738fc324614210120f7f7c9fc1e2273
:10eec00002210346cde9002104a80122394604f0bd
:10eed00053fc3246012105a8f3f708fd13f0e7fac9
:10eee000064613f0e4fa831bf92bfad904a8faf7c3
:10eef00027fffbf759ff0023c0f888401a46072177
:10ef000018460093fff774fe164b1b7843b10db003
:10ef1000bde8f040fbf7f6be0a24a9e7124fbce7b4
:10ef2000002df4d1fdf780fa0328f0d12846fdf733
:10ef300087fa0128ebd00db0f0bd00bf36cb001032
:10ef400033cb001035cb001034cb0010338c0c02c7
:10ef500020740c02d8d2001028d7001075cf0010f2
:10ef6000438c0c0237cb00100060ff0013b5044641
:10ef7000fdf734fa034638b9024600900221012019
:10ef8000fff736fe02b010bdfff7e0fc204602b0ee
:10ef9000bde81040fff70abf10b504460bf0c4fbf4
:10efa0000022194b19481a60f8f7b4fe184b1b7869
:10efb00003f0ff0023bbfef77bfefff7b5fbf8f77e
:10efc000e7fdf8f798fbf8f79dfb2046fff7ceff2b
:10efd000f9f774fbf9f79cfcfdf726fa042801d039
:10efe000fff760fdf5f7b2fbf5f7adfbfdf71cfa97
:10eff000042801d0fff767fdbde81040f4f700be1c
:10f000008c20f4f7a1fdede730d70010f4d6001006
:10f01000c5d20010f0b5224e044696f82c300d46ad
:10f02000174687b0002b38d0706a18f0fefe002813
:10f0300033d104900c200ff0cbfb10b1c0e9004598
:10f040008760184b02900593174b142004930ff020
:10f05000bffb0446d8b1154b03600023c360049b7b
:10f060003bb1022202a904309847059b2361049b0f
:10f07000e3600f4bf2692360306b002301a9019418
:10f0800018f031ff18b1236820469b68984702a802
:10f09000f4f770f9002007b0f0bd2846a047f9e763
:10f0a00044d2001035f00002e5e40002f4730c02d3
:10f0b00008740c0203681868d3e90112fff7aabfad
:10f0c00008b5002301211a461846f8f764fabde88e
:10f0d0000840f6f723b8000037b501900bf01afb93
:10f0e000019905460448fff7f3f9044628460bf05a
:10f0f00015fb204603b030bddcd6001013b50190df
:10f100000bf008fb044601990448fff74bfa204630
:10f1100002b0bde810400bf001bb00bfdcd6001010
:10f120006ff0770070470000032809d8dfe800f08f
:10f130000a02040604487047f6f71abbf9f76ebadc
:10f14000002070470148704770cc001044d2001076
:10f1500013b500240b4a23460b490c480094f2f7e0
:10f16000ebf90b4b0b4a1c605c600b4bc2e904448f
:10f170005360d3604ff480639360084b136002b018
:10f1800010bd00bfd9e4000265e60002f5e500020b
:10f19000f4d60010dcd60010dcd200106c8c0c020f
:10f1a000002270b511468cb00546f8f7d6f9024634
:10f1b00090b1002228461146f8f7cff928b1002374
:10f1c00001211a462846f8f7e6f9002205212846cb
:10f1d000f8f79afa012606e001462846f8f76ef994
:10f1e0000028e6d1064600212846f8f7eff9044644
:10f1f00038bb284604a91ff0d9fc68b9fcf756f9ba
:10f2000002220499fcf780fac8b9fcf74ff90422ee
:10f210000499fcf779fa04460023032220200021f8
:10f22000cde901330093f7f79bfd0123002063f341
:10f23000070064f30f2066f317400cb070bd012483
:10f24000eae700242023cde90434054b0120009394
:10f2500004492346019504aaf3f764fae5e700bfe1
:10f260009d8c0c02908c0c02012a38b5044602d108
:10f270000b68236003e0022a03d0032a0dd000208c
:10f2800038bd0c200d680ff0a3fa03460028f0d01b
:10f2900095e8070083e80700ebe700680028eed058
:10f2a0000c210ff09dfaeae770b50446154649b106
:10f2b0000021f8f78bf928b1002320461a46194699
:10f2c000f8f784fa3db100232046bde870401a46a5
:10f2d0001946f8f7efbb70bd21b18b88834201d08e
:10f2e0008968f9e70846704708b50a46c1680e20e4
:10f2f000fff7f2ff40b1037b934202d1c389db07e2
:10f3000001d58168f3e7012008bd4ff00102d0e884
:10f31000cf3fc0e8412f0029f9d1dbb2002bf6d155
:10f32000704700002de9f04f9a4b144693f82c20bb
:10f33000054688468bb0dab1586a18f076fdb8b940
:10f3400008900c200ff044fa10b1c0e90058846016
:10f35000914b06900993914b8e4806a90893f4f7b8
:10f3600001f9044670b9064606a8f4f703f805e06b
:10f37000002128460ef0dafd061e0fda30460bb0eb
:10f38000bde8f08f00224ff0ff31406918f066feb3
:10f39000236820469b68a6699847e5e7f9f78ef948
:10f3a0000821f9f71dfb04212846fff79dff0028df
:10f3b00068d103212846fff797ff0746002861d14f
:10f3c0000420e968fff788ff002859d04ff47a73ca
:10f3d000c668b6fbf3f6ab68dc072ed5f6f7c6fcbd
:10f3e00058b3fbf7e5fc0446fff78fff0023e26804
:10f3f000d4f810a094f81590e36023612375637529
:10f40000c4e88f3fd00758bf237a910758bfd4f87c
:10f4100004a0520758bf94f80990fbf7c9fc0446b2
:10f42000fff773ff0723e3600123c4f810a02375df
:10f4300084f815900023c4e88f3f002306211a4664
:10f4400001200096fff7d4fbfcf7c8ff8146fcf7cc
:10f45000bfff04212846fff747ff68b96b88022bde
:10f4600018d9e9680e20fff737ff98b1037b042b0a
:10f470000ed1c389db070dd50024a346234611e036
:10f480003e46a8e7f6f772fc4ff000090746e0e7b2
:10f490008168e7e70420fff783fec3b2c0f3072bc0
:10f4a000c0f3074403200393fff77afe0021c0f363
:10f4b00007228df818008df819205ffa80fac0f342
:10f4c000074208468df81a20f3f754fae720f1f7bf
:10f4d000bbfe0120f3f767fe0022414628460ef0ee
:10f4e0006bfd0646f3f760fe00210120f3f742fab8
:10f4f000e720f1f785fe039b23b1224659460420fd
:10f50000fff7d2febaf1000f06d003209df81a20b3
:10f510009df81910fff7c8feb9f1000f2ed0fcf7c7
:10f5200035fffcf781ff04460020fcf789ff054604
:10f5300000287ff423af013ce4b2012c3ff61eaf5c
:10f54000fcf74cff00283ff419af284612f0a2ff49
:10f550004ef660250446002012f09cff001b61f16e
:10f560000001a84271f1000305d2f6f7fffb10b9c4
:10f57000f6f70cfcefe7f6f7f9fbffe6002f3ff498
:10f58000fdaefaf76bfe4b464a46042104f05ffce1
:10f59000f4e600bf70cc001021f50002e9f1000292
:10f5a00003681868d3e90112fff7bcbe70b50023e9
:10f5b0001646202204460d468ab0cde90223074aaa
:10f5c00001200092064902aaf3f7acf83246294618
:10f5d00020460ab0bde87040fff7a4beb98c0c020b
:10f5e000908c0c02012a034602d101600020704772
:10f5f000022a04bfd1e90001c3e90001f6e7012aac
:10f60000034602d1016000207047022a04bfd1e9fd
:10f610000001c3e90001f6e7012a034602d10160b7
:10f6200000207047022a04bfd1e90001c3e90001ac
:10f63000f6e7012a034602d1016000207047022a42
:10f6400004bfd1e90001c3e90001f6e7012a03463e
:10f6500002d1016000207047022a04bfd1e90001f5
:10f66000c3e90001f6e7012a02d1016000207047da
:10f67000022a04bf0b680360f8e7012a034602d19f
:10f68000016000207047022a04bfd1e90001c3e9ec
:10f690000001f6e700224ff0ff3118f0dfbc000058
:10f6a00070b52d4e044696f82c3086b0002b4bd00a
:10f6b0003046f6f7d5fa0546002845d1274b1c20e1
:10f6c0000593274b029404930ff082f80446002818
:10f6d00031d0244bc5600360049b3bb1022202a9d8
:10f6e00004309847059b2361049be3600025204676
:10f6f0001d4b2a462360012140f8145f18f09efc40
:10f700001a4b01a92360f2692b46306b019418f063
:10f71000eafb014650b9706a08b118f0b3fb002249
:10f720004ff0ff31606918f099fc257e2368204670
:10f730009b68984700e0054605f0010502a8f3f72d
:10f7400019fe284606b070bdfdf70afd06b0bde8fb
:10f750007040fdf721bd00bf70cc0010f1f6000233
:10f76000e7f50002a8770c02bc770c02d0770c02f8
:10f770000068fff795bf000070b5534d044695f83b
:10f780002c300e468ab0bbb12846f6f769fa98b914
:10f790004e4b284605934e4b02a98df80840039620
:10f7a0000493f3f7dffe0546c0b9044602a8f3f759
:10f7b000e1fd20460ab070bd09200bf045fab0b952
:10f7c0002023cde90230434b4349009302aa03466c
:10f7d0003220f2f7a7ff6ff08104eae74069fff7f4
:10f7e00059ff2b6828469b68ac699847dee7002cd8
:10f7f0004cd0fdf7b5fcfdf7cffc044608b1002462
:10f80000d7e7fdf7d5fafdf7d7fa90b109200bf04d
:10f810001bfa70b12023cde90234304b2e4902aae5
:10f82000012000932346f2f77dfffdf7c1fafdf7b3
:10f83000effb002520262a4b02aa2749012000932e
:10f840002b46cde90265f2f76dfffdf789fc01213a
:10f85000fdf7a5fcf4f77aff183000f0a5fcfdf7e2
:10f860007ffcfef781f804460028a2d01d4b1a4900
:10f87000009302aa2b460120cde90265f2f752ff60
:10f88000fdf76efc2946fdf78afc92e7fdf768fc60
:10f89000fdf782fc0028b2d02023cde90234124bc0
:10f8a00002aa0d49009301202346f2f73bfffdf722
:10f8b00057fc2146fdf773fcfdf752fc0ab0bde88a
:10f8c0007040fdf7e5bc00bf70cc00106df8000281
:10f8d000fbf50002d58c0c0220740c020a8d0c0280
:10f8e000588d0c026d8d0c028b8d0c0241680078d6
:10f8f000fff742bf7fb51c4d044695f82c300e46ed
:10f90000b3b12846f6f7acf990b9184b69460393a2
:10f91000174b2846cde900460293f3f723fe044631
:10f9200048b905466846f3f725fd284604b070bd82
:10f9300054b9104df9e74069fff7acfe2368204643
:10f940009b68a5699847ede709200bf07df940b168
:10f95000f4f7fcfe2146183004b0bde8704000f01a
:10f96000c3ba6ff08105e0e770cc0010f9f800022f
:10f97000cdf50002f2feffffd0e90001fff7babfac
:10f980007fb51c4d044695f82c300e46b3b1284681
:10f99000f6f766f990b9184b69460393174b28465a
:10f9a000cde900460293f3f7ddfd044648b905466c
:10f9b0006846f3f7dffc284604b070bd54b9104d1b
:10f9c000f9e74069fff766fe236820469b68a56952
:10f9d0009847ede709200bf037f940b1f4f7b6fe90
:10f9e0002146183004b0bde8704000f095ba6ff0c1
:10f9f0008105e0e770cc001085f90002b3f5000244
:10fa0000f2feffffd0e90001fff7babf7fb51c4d42
:10fa1000044695f82c300e46b3b12846f6f720f987
:10fa200090b9184b69460393174b2846cde9004619
:10fa30000293f3f797fd044648b905466846f3f785
:10fa400099fc284604b070bd54b9104df9e74069df
:10fa5000fff720fe236820469b68a5699847ede7dd
:10fa600009200bf0f1f840b1f4f770fe2146183090
:10fa700004b0bde8704000f067ba6ff08105e0e7c0
:10fa800070cc001011fa000299f50002f2feffff9f
:10fa9000d0e90001fff7babf7fb51c4d044695f8c9
:10faa0002c300e46b3b12846f6f7daf890b9184b69
:10fab00069460393174b2846cde900460293f3f7b6
:10fac00051fd044648b905466846f3f753fc2846fd
:10fad00004b070bd54b9104df9e74069fff7dafd85
:10fae000236820469b68a5699847ede709200bf03d
:10faf000abf840b1f4f72afe2146183004b0bde857
:10fb0000704000f039ba6ff08105e0e770cc00106a
:10fb10009dfa00027ff50002f2feffffd0e900012e
:10fb2000fff7babf7fb5174d044695f82c300e4647
:10fb300003b32846f6f794f8e0b9134b69460393ec
:10fb4000124b2846adf8004001960293f3f70afde8
:10fb5000044668b14069fff79dfd236820469b6815
:10fb6000a56998476846f3f705fc284604b070bdc0
:10fb70000546f7e7fdf7f4fa214604b0bde870400a
:10fb8000fdf710bb70cc001011fb000265f5000200
:10fb900041680088fff7c6bff8b5044605462f4602
:10fba00015f8016b3046a0f0b1f90028f7d15f2eaf
:10fbb000f5d0381bf8bd2de9f8430c461746994699
:10fbc00078b119b38e18a64205d9054615f8013b40
:10fbd0004bb904f8013b0023781e341b06f8013ca6
:10fbe000001bbde8f883242b0dd12846fff7d4ff76
:10fbf000804630b122460146331b2846c84745445b
:10fc000004442846dfe704f8013bfae70846e8e742
:10fc10007047704737b5044601910af07bfd0199a2
:10fc200005462046fef754fc044628460af076fdb9
:10fc3000204603b030bd10b5044604210ef0d0fdbf
:10fc4000204610bdc86910b50c4608b10ef0c6fdbf
:10fc50000023c4e90133e36110bd000010b5044b7b
:10fc600004460360406808b10ef0b8fd204610bda0
:10fc7000d88f0c0210b50446fff7f0ff204618217c
:10fc80000ef0aefd204610bd08461146a1f03aba6e
:10fc90000846a0f069ba0846a0f05eba2de9f04126
:10fca0000c461e46174605460368ddf818805b685b
:10fcb0009847c4e90968e762a86918f079f9eb6820
:10fcc00043b19c610023a361a869ec60bde8f041e9
:10fcd00018f07db9ac60f5e737b5054601910af03b
:10fce00019fd044601992846fef75cfc204603b046
:10fcf000bde830400af012bd10b5084cd4e88f3f83
:10fd0000db0709d4204610f001fe28b1204610f090
:10fd100037fe0348a0f027f8024810bd34d7001082
:10fd200091fb00027851001008b54bf085fb18b12b
:10fd3000bde8084021f022bc08bd38b504460620c5
:10fd40004bf0a0fa054668b120464bf0a7fa012215
:10fd5000294620464bf0fafa034628b1bde8384060
:10fd600021f00cbc6ff07703184638bd08b54bf096
:10fd700001fc18b1bde8084021f000bc08bd13b576
:10fd8000044608460191f0f7fdff0199024620461e
:10fd9000fff7ecff02b010bd10b5c368044623b9ed
:10fda0000a200e4a0e49f1f7fbf8e3685a681989f0
:10fdb000023a5a60e268936802339360e3685b68d2
:10fdc0001980d4e90223916a29b10b6000211960de
:10fdd0009362e16010bd5362f8e700bfbff5010216
:10fde000a18d0c0270b500250446394bc0e90255bf
:10fdf0000360c0e90455416040f8185f18f0c9f885
:10fe0000344be56163654ff6ff732562a4f86c30ef
:10fe1000a4f86e30c4e909552f4bc4e90b55c4e969
:10fe20000d55c4e90f55c4e91155c4e91355c4e98a
:10fe30001955c4e91755c4e91c55e567a56584f84b
:10fe40008050a56784f8815084f8825004f18402c0
:10fe500003f11006154618685968083303c5b34204
:10fe60002a46f7d118681d4b286004f1980203f167
:10fe70001006154618685968083303c5b3422a4668
:10fe8000f7d11868164b286004f1ac0203f1100694
:10fe9000154618685968083303c5b3422a46f7d196
:10fea0001868104b286004f1c00203f110061546d3
:10feb00018685968083303c5b3422a46f7d1186851
:10fec000002328602046a4f8d430a4f8d83070bdb0
:10fed0006c900c02d88f0c023c900c0250900c02db
:10fee00024900c0210900c0230b581b10b4600f149
:10fef000840201f11005144618685968083303c4d8
:10ff0000ab422246f7d118682060002030bd01487e
:10ff1000fce700bff2feffff30b581b10b4600f1f8
:10ff2000ac0201f11005144618685968083303c47f
:10ff3000ab422246f7d118682060002030bd01484e
:10ff4000fce700bff2feffff30b581b10b4600f1c8
:10ff5000c00201f11005144618685968083303c43b
:10ff6000ab422246f7d118682060002030bd01481e
:10ff7000fce700bff2feffff30b581b10b4600f198
:10ff8000980201f11005144618685968083303c433
:10ff9000ab422246f7d118682060002030bd0148ee
:10ffa000fce700bff2feffff70b50246054601f117
:10ffb000840601f19403344603cc9c4210605160e6
:10ffc000264602f10802f6d120681060284670bd6e
:10ffd0008b890022a0f86e301423c36780f880203c
:10ffe00090f88030dbb280f8813000f17803c3e80c
:10fff000af2f00f1740353e8001f0131c3e8e01f85
:020000040807eb
:100000000028f8d110467047b0f86e308a899bb24c
:100010009a4202bf4b68033bc36700207047b0f8a9
:100020006e308a889bb29a4212d1ca88b0f8d63014
:100030009a420dd1002380f880308a689a42c8bf66
:10004000012380f8803090f88030dbb280f8813076
:10005000002070472de9f041044690b000201bf0cd
:100060001dfc20b10a204a4a4a49f0f799ff94f84a
:100070008250002d40f089802b4601200df10202b4
:1000800004f184011cf0b2ff00287bdb424f2822e0
:10009000294606a8059708aea0f0b3f804f1980c1d
:1000a000bce80f000fc6dcf800302a46336002239c
:1000b0008df81830bdf8023001a905a8adf834302c
:1000c0001cf0c6fd00285ddb2b4601223349bdf83c
:1000d0000a0019f0c3fd002854db2022294606a897
:1000e000059708aea0f08df804f1ac0cbce80f0049
:1000f0000fc6dcf80030dff8ac80336010238df8d9
:100100001830bdf802302a4601a905a8cde90e84b1
:10011000adf834301cf09cfd002833dbbdf80a300c
:100120002022a4f8d430bdf80e302946a4f8d630e9
:10013000059706a808ae04f1c007a0f062f80fcf3b
:100140000fc63b682a4633600c238df81830bdf883
:10015000023001a905a8cde90e84adf834301cf0b9
:1001600077fd00280edbbdf80a302a4621460c48f0
:10017000a4f8d8301cf0a8fd002803db0123284692
:1001800084f8823010b0bde8f0816ff0d100f9e75b
:10019000bff50102e4890c0203002c0038900c0228
:1001a0000d0a010289040102002238b504461146f5
:1001b00010460ef05ff82046fff74cff054660b989
:1001c0004ff4806007499ff073fa40b14ff48063a9
:1001d000c4e91955a0652066e365284638bd024d7f
:1001e000fbe700bf55860e02fcfefffff8b5064692
:1001f0000d463820104917469ff058fa0446c0b102
:10020000382200219ff0fdff0b4905f110009ff0ff
:100210004ffae06148b10db1083060600020336fe3
:10022000a560236366613c60f8bd382120460ef06e
:10023000d7fa0248f8e700bf55860e02fcfeffff22
:1002400070b50d4616681446fff756fd0368314633
:100250001b6905f10c02984746b948b1066000f1e8
:100260000c03c0e901352060002070bd0028f6d1e4
:100270000048fae7fcfeffff70b5c36804460d4670
:10028000164623b10a200c4a0c49f0f789fea068f3
:1002900004f10c02b11cfff7d3ff00280adb002099
:1002a000e268536802335360e2689368023b9360ec
:1002b000e3682b6070bd00bfbff50102b78d0c0273
:1002c00030b5002585b04ff4007202a904460295ae
:1002d000fff7d2ff00280edb114b02990093019526
:1002e00003ab04f12800d1e90112039545f0e8fec3
:1002f00018b121f043f905b030bddde9023204f157
:100300001c0059689a60f8f7c3f90028f3db20460f
:10031000fff742fd03230120c4f8c831ebe700bf1b
:10032000c5140302f0b5002685b0202269460546b3
:100330000096fff7a1ff041e23db009b05f11c07bd
:1003400038465968fff7f0fc041e1adb38464af0bd
:10035000aaff01a8cde901660396fff7eefc041e93
:100360000cdb202205f5d47101a84bf0a3f858b995
:100370001b4901a8fff703fd041e0ada01a84af091
:1003800092ff204605b0f0bd21f0f8f8041ef5db21
:10039000eee7144901a8fff7f2fc041eeedb124958
:1003a00001a8fff7ecfc041ee8db009b01a8d3e9e1
:1003b0000112fff7dbfc041ee0db009b01a859687b
:1003c0004bf0e8f838b92846fff7e6fc072300248d
:1003d000c5f8c831d2e721f0d1f8041ecedbf2e730
:1003e000ce8d0c02d58d0c02b5d10c0230b5002596
:1003f00085b04ff4007202a904460295fff73cff56
:1004000000280edb114b02990093019503ab04f118
:100410002800d1e90112039545f0acfd18b121f097
:10042000adf805b030bddde9023204f11c005968b9
:100430009a60f8f72df90028f3db2046fff7acfcb3
:1004400004230120c4f8c831ebe700bfc514030240
:1004500038b515460c4601f1200205f11001fff7f1
:10046000effe002806db35b1236a5b680833002005
:10047000c4e9033538bd2b46f9e7000038b55430e0
:100480000c460c311546fff7c5fb40b10246002370
:1004900042f80c3bc0e901242860184638bd0148e9
:1004a000fce700bffcfeffff73b5b0f86e308a8832
:1004b0009bb29a4205460c461fd1b0f8d830ca8884
:1004c0009a424ff000031dd1c96801aa0193fff7ba
:1004d000d5ff002812dbd4e90321019b58689ff067
:1004e00069fe019e0af016f92b6a4bb12b6a1e6059
:1004f000002434602e620af011f9002002b070bdb1
:10050000ee61f5e71846f9e770b503680546092b73
:100510000c468cb003d00b2b26d00cb070bd01461e
:100520002046fff7c1ff0028f7d020230026cde9a1
:1005300004362b68029001930e4b04aa00933220dc
:1005400033460d49f2f7eef84ff6ff72b4f86e300d
:100550009bb29342e1d03146b4f86e0080b20cb049
:10056000bde8704019f0a0bc01462046fff757fdda
:10057000d9e700bfec8d0c02dc8d0c0210b50446ef
:10058000006808b10ef02af9204610bd03681bb1bf
:100590009a69026002b942601846704710b5037943
:1005a000044613b901209ff01cf9036823b11868b1
:1005b00017f00dfd0023237110bd03681bb11a68ed
:1005c000026002b942601846704738b505680446b3
:1005d0004db10af09ff825682b682360236803b9a2
:1005e00063600af09bf8284638bd0b46014618b1f7
:1005f0001a681846d2681047704710b50c4629b1e2
:10060000fff77afb01462046fff7efff10bd70b5fc
:100610000c46a1b1d1e90956096afff7eeffe0697e
:1006200008b10ef0dbf8382120460ef0d9f835b1cc
:1006300031462b46bde870406ff06300184770bd2f
:100640002de9f04390f8813004468bb023b90025a2
:1006500028460bb0bde8f083436c23b90a20304a2a
:100660003049f0f79dfcd4f87c8004f12409a66c95
:10067000b0451fd9656aedb1aa68a8eb0607974295
:1006800028bf1746606c3a46696830449ff092fd77
:100690006b683b446b60ab68db1bab6033b94846af
:1006a000fff78bff29462046fff7a7ffa36c3b44cb
:1006b000a364dce7beb904f17803d3e8af3f002bb5
:1006c000c5d104f110073846fff760ff0546002842
:1006d000bdd0d0e9093100209847294620466e62f6
:1006e000fff795ffefe700233246616cb4f8d400c2
:1006f00019f0c0fda36c054683424ff000030bd0f8
:100700002022cde90223084a0190009232200749b5
:1007100002aaf2f707f89be71d46a36498e700bf1b
:10072000bff50102188e0c02348e0c02dc8d0c0217
:1007300008b50346084619b103f15401fff755ff08
:1007400008bd00002de9f84f0446894617460025ec
:1007500000f11c06636bbb4228d34ff00008dff8a2
:1007600088a0dff888b0474539d9e66a26b95246ed
:1007700059460a20f0f714fcb268a7eb0805954229
:1007800028bf154671682a4609eb08009ff012fd44
:10079000b3685b1bb360f3b904f12c00fff70dffe6
:1007a00031462046fff7c4ffa844dce73046fff798
:1007b0000cff58b1236b3bb1186005602063636b7d
:1007c000826813446363c5e7e062f6e7636bbb428c
:1007d000c3d2bde8f88f73682b447360e4e7626ba3
:1007e0000120d21b6263f4e7bff50102718e0c0297
:1007f000f7b504461546002600f11c07636bab42b3
:1008000011d238460191fff7e0fe019958b1236bf0
:100810003bb1186006602063636b826813446363b6
:10082000ece7e062f6e7626b954228bf15464db1f2
:100830002a462046fff786ff20b90a20034a0449ca
:10084000f0f7aefb284603b0f0bd00bfbff50102d4
:10085000868e0c02f7b51546d0e905329a42044659
:100860000e4610d100270222806801a9adf804705d
:10087000fff768fff8b1bdf804306361013bb3f5e1
:10088000007f14d2a7616168d4e90523a068d21a59
:100890001944fff7adffa36918446369a06198424a
:1008a00009d363680020336063692b6001e06ff057
:1008b000bd0003b0f0bd0120fbe7002313b569467e
:1008c00001aa0446cde90033fff7c4ff40b9dde9d2
:1008d000001204f1280045f011fb18b120f04efe83
:1008e00002b010bd04f11c00dde90012f7f7d0fee4
:1008f0000028a2bf02230120c4f8c831f0e700237a
:1009000013b5694601aa0446cde90033fff7a2fffb
:1009100040b9dde9001204f1280045f073fb18b17d
:1009200020f02cfe02b010bd04f11c00dde9001225
:10093000f7f7aefe0028a2bf05230120c4f8c83196
:10094000f0e70000f0b5836b04468fb0d3b9022204
:1009500006a9adf81830fff7f5fe00286ad0bdf8fb
:1009600018502046294604f13802fff73ffc0028c2
:1009700060dba36bbdf81820db6910351a800223f9
:10098000e5632364a36bd4e90f21dd69521a204685
:100990002944fff72dff236c1844e36b2064984231
:1009a00047d3e36c23b90a20234a2449f0f7f8fa25
:1009b000e66ca36baa1c9f68736d01337365069385
:1009c000706cb16c07ab03c308230593fb182b4471
:1009d000cde9032302230292cde9005330460c23d4
:1009e00006aab91d4af042fc18b120f0c7fd002844
:1009f00020db6988a36baa889986a36b00255a809f
:100a00002023cde90635a36b01209a8e0c49029272
:100a10005b8806aa01930b4b00932b46f1f782feed
:100a2000606822460368a16b1b689847c4e90e55ad
:100a3000256400200fb0f0bdbff501029a8e0c02b4
:100a4000dc8d0c02b38e0c0238b5b0f86e308a899a
:100a50009bb29a42044617d100f11c052846fff7c5
:100a6000b4fd014618b12046fff762fef6e74ff6e7
:100a7000ff73743424f8063c607354e8003f01337c
:100a8000c4e8e23f002af8d1002038bd70b5036801
:100a90000546042b0c468cb027d0062b2ad0032bfe
:100aa0002dd101462046fff793fa40b320230026bc
:100ab000cde904362b6802900193124b04aa0093ef
:100ac000322033461049f1f72dfe4ff6ff72b4f88d
:100ad0006e309bb2934212d03146b4f86e0080b2b1
:100ae0000cb0bde8704019f0dfb901462046fff7b1
:100af000abffdae701462046fff786fad5e70cb0f0
:100b000070bd00bfec8d0c02dc8d0c02036801602f
:100b100013b118460df062be704710b504460021af
:100b20000430fff7f3ffd4e90201fff766fd00236d
:100b3000c4e90533e36010bd00232de9f04194b012
:100b400004aa03a90646cde90333fff783fe044652
:100b5000a0b9049a202a40f0b9805f4b06f128081a
:100b600006f5c4750590019000932946404605abf3
:100b700045f03cfb30b120f001fd0446204614b0a6
:100b8000bde8f081059f202f40f0a280404645f04f
:100b900058f906a8cde906440894f7f757fd041e56
:100ba00036db06a8f7f76bfd041e31db3a46294613
:100bb00006a8f7f76dfd041e2adb0822474906a8a0
:100bc000f7f766fd041e23db06f5d478414606a838
:100bd000fff7aaf8041e1bdb06a84af064fb06a870
:100be000f7f734fd041e13db06f11c07394606a88f
:100bf0004af086fb80b900251c2229460da80c95d9
:100c00009ff0fffa0ca906a8fff78ef8041e08da79
:100c100006a84af048fbb1e720f0b0fc041ef7db61
:100c2000e9e706a84af03ffb09a8cde909550b956d
:100c3000fff783f8041e0bdb2022414609a84af087
:100c400039fc48b9264909a8fff799f8041e08dac3
:100c500009a84af028fbdbe720f090fc041ef7db34
:100c6000f0e7204909a8fff78af8041ef0db1e49c7
:100c700009a8fff784f8041eeadb20220ca909a8c2
:100c8000fff774f8041ee3db0ca909a84af082fc04
:100c9000a8b9039c202220460ca99ff07bfa98b9a2
:100ca00021463846049af7f7f3fc041ed0db3046a1
:100cb000fff733ff06230124c6f8c831c8e720f048
:100cc0005dfc041ec4dbe4e7084cc1e7074c55e7b4
:100cd0006ff0f90452e700bfc5140302e08e0c0266
:100ce000ce8d0c02b5d10c02d58d0c02e8feffffb3
:100cf00010b5d0f8c8310446013b062b05d8dfe813
:100d000003f0070f1215181b1e006ff0d10010bd65
:100d1000fff7d3fd0028fada0823c4f8c831f6e754
:100d2000fff764fbf6e7fff7eafdf3e7fff7c8fa22
:100d3000f0e7fff701ffede7fff7f4faeae700203d
:100d4000e5e7000010b504460f4b40f8283b45f09e
:100d500078f82022002104f5c4709ff052fa202276
:100d6000002104f5d4709ff04cfa04f11c004af005
:100d70009afa064b20462360fff7cffe201dfff7af
:100d8000fdfb204610bd00bf04900c02f08f0c024a
:100d900010b50446fff7d6ff20464ff4e6710df07c
:100da0001ffd204610bd036801601bb11a6818467c
:100db0005268104770470000f0b5002689b004adb6
:100dc000074632460f2128460696cde90466cdf83f
:100dd0001b600df04ffa002852db0e2858dd4ff44f
:100de000e6702e499ef062fc044690b12c4bc0e99f
:100df0000167c0e90366c0e90566c0e907660360ec
:100e000046624ff4b072314628309ff0faf9c4f8c8
:100e1000c861214607f15000fff7c5ff3c6d002c6b
:100e200039d01e494ff400709ef042fc0146201d4f
:100e3000fff76cfe63684bb311f039fb04f11c063d
:100e400020613046f7f702fc031e17db3046f7f748
:100e500016fc031e12db04f12800039044f0c6ffc9
:100e60000f230622cde9005301210323039845f007
:100e700013f8034630b120f081fb034603eae37028
:100e800009b0f0bd0122c4f8c821f7e7054bf5e72a
:100e90006ff0f900f4e70348f2e700bf55860e0251
:100ea00004900c02fcfeffff10b50a490446f42032
:100eb0009ef0fefb014604f14400fff727fe636c41
:100ec0002bb12046fff778ff00eae07010bd024822
:100ed000fce700bf55860e02fcfeffff034607b588
:100ee0000068196048b101904af064f95c210198ea
:100ef00003b05df804eb0df073bc03b05df804fbc8
:100f000070b5036d054623b90a20214a2149f0f73f
:100f100047f82c6dd4f8c831072b26d104f5c474da
:100f20005c201d499ef0c2fb064630b144220021e0
:100f30009ff067f90023c6e9153305f14c003146ef
:100f4000fff7ccffed6c05b328464af00cf980237f
:100f50002246022128464af00af9034660b120f0f1
:100f60000dfb034603eae37070bd0a20084a0b49f3
:100f7000f0f716f80024d3e722696a646269aa646c
:100f8000a269ea64e2692a65ece70548ece700bf7c
:100f9000bff50102e98e0c0255860e02018f0c028c
:100fa000fcfeffff10b50368044613b901209ef054
:100fb00018fc02790ab12d20f9e7186816f0f8ff3d
:100fc0000123237110bd0000f0b500f1180391b0aa
:100fd00006930023064606a88df81c30fff7e2ffb3
:100fe000012306f108058df81c302846fff7cefadc
:100ff000044640b1026b336f9a4204d0014630463a
:10100000fff705fbf1e706a8fff7c8fa002c00f090
:101010008780236a2269abb9002a74d0202200237a
:10102000cde90823a28e322001923e4a3e49009229
:1010300008aaf1f777fb6ff0bd0521463046fff7b0
:10104000e6fa57e09b68103b9342e7d3236a5d685a
:1010500023692b80e36aa28e6b606a80f36c23b9ec
:101060000a20324a3249eff79bfff76cd4f810c0e0
:10107000bb6daa1c0133bb6543f000430893f86cb9
:10108000396d09ab03c30823059363442b44cde9b1
:10109000032302230292cde9005338460c2308aa09
:1010a0000cf106014af0a8f818b120f067fa051e05
:1010b000c3db2369226a10339360b36a226a5bb38d
:1010c0001a6000231360b26220222362cde9082354
:1010d000a28e01200192174a1349009208aaf1f743
:1010e00021fb656a002da8d07369bbb19c61002506
:1010f000a56174619df81c3013b106a8fff74efa84
:10110000284611b0f0bd1021304604f12002fff74f
:1011100097f8051e9ada90e77262d2e73461e6e743
:101120002546e7e7198f0c02dc8d0c02bff50102a2
:101130009a8e0c023c8f0c0273b590f882300446f4
:10114000002b58d000215030fff72dfe002104f174
:101150004c00fff7c3fe002104f14400fff7d6fc6a
:1011600004f118030093002368468df80430fff75c
:1011700019ff012304f108058df804302846fff714
:1011800005fa014618b12046fff741faf6e768462e
:10119000fff704fa04f110052846fff7f7f90146b6
:1011a00090b904f124052846fff707fa014678b9fb
:1011b00004f12c063046fff700fa054660b10146ff
:1011c0002046fff7b5faf5e72046fff720fae3e7f8
:1011d0002046fff712fae6e72046a16bfff717fa61
:1011e0009df80430c4e90e5525646563a56413b108
:1011f0006846fff7d3f902b070bd000070b5054630
:101200008cb000f17403d3e8af3f026f9a4260d014
:10121000b0f86e20b0f86c400367a0f86c20fff7c0
:101220008bff4ff6ff72b5f86c30934239d0002433
:101230002023cde90434574b01205749009304aad9
:101240002346f1f76ffa234622464ff4002000218f
:10125000cde901440094f5f783fd2846fff724fe0d
:101260000446002835d02023002601944ff6ff7451
:10127000cde90436494b322000934749334604aa4e
:10128000f1f750fab5f86c00a04204d0314618f0de
:101290000bfea5f86c4028460cb0bde87040fff787
:1012a0004bbf9c4266d000242023cde904343c4b44
:1012b00001203949009304aa2346f1f733fa234663
:1012c00001224ff400200021cde901440094f5f7fc
:1012d00047fd4ff6ff73b5f86c209a424ad0286d4f
:1012e000002849d003689b689847041e16da002638
:1012f0002023cde904362b4b322000932649334678
:1013000004aaf1f70ffa3346cde9016600960222ee
:101310004ff400200021f5f723fda4e723d1284650
:10132000fff7eefd044620b10023cde90133009321
:10133000ede7014605f15000fff735fd2023cde92b
:101340000434194b01201449009304aa2346f1f7f1
:10135000e9f9234603224ff400200021cde901449e
:101360000094f5f7fdfc2846fff76af904460028cb
:101370007ff479af0cb070bd2846fff725fe044618
:1013800000287ff470af2846fff7dcfa04460028f7
:10139000e9d068e7698f0c02dc8d0c02a08f0c028b
:1013a000738f0c02808f0c02918f0c022de9f04399
:1013b00004460f461568dff8888087b0002d3dd0c1
:1013c000d5f80c90d9f800305e78022e01d02d6847
:1013d000f4e71822002168469ef013ffd9f8003088
:1013e0005a78022a18d101225b688df800201bbab6
:1013f000019399f8103039462046059320f064fa9d
:1014000030b16a464146204620f0e8fb0028ded194
:10141000002007b0bde8f0830a2af9d103f10802e1
:101420008df800600df1040c1833664610685168a1
:10143000083203c69a42b446f7d1dae70120e8e75a
:1014400086710c0238b51468054623685bb1636881
:101450004bb120f039fa38b1d4e900122846bde882
:10146000384020f078bb012038bd00002de9f04362
:1014700004460f461568dff88c8087b0002d3ed0fb
:10148000d5f80c90d9f800305b780a2b01d02d6884
:10149000f4e71822002168469ef0b3fed9f8003028
:1014a0005a78022a18d101225b688df800201bbaf5
:1014b000019399f8103039462046059320f004fa3c
:1014c00030b16a464146204620f088fb0028ded134
:1014d000002007b0bde8f0830a2af9d102220df1fd
:1014e000040c8df8002003f10802183366461068da
:1014f0005168083203c69a42b446f7d1d9e70120b1
:10150000e7e700bf86710c0270b50c460546eff7a1
:1015100039fc06462046eff735fc8642024607d3e3
:1015200021462846a0f0acfcb0fa80f0400970bd1e
:101530000020fce710b512490446fff7e5ffb8b9f3
:1015400020461049fff7e0ffa0b920460e49fff7fb
:10155000dbff88b920460d49fff7d6ff70b920465a
:101560000b49fff7d1ff002814bf1020002010bd49
:101570000120fce70220fae70420f8e70820f6e75c
:1015800078900c02f9910d0216e80c02a8830c0267
:1015900031920c022de9f04f05460e4600271468e3
:1015a000dff88480dff884908db0002c3ad060683a
:1015b0000df10f018df80f701df09ffb70bb0490b3
:1015c000adf814000df1100b594660681df0b1fc28
:1015d000019018bb5846fff7adff8246f0b1019964
:1015e000102208a89ef00dfe5846eff7cbfb06ab85
:1015f000cde909839df80f30cde906b03146284684
:1016000008938df82ca020f05ff938b149462846a0
:1016100008aa20f0e3fa08b12468c6e700200db05c
:10162000bde8f08f0120fae7c5130102a4710c0296
:10163000002330b585b0054601a801931df044fa9a
:10164000041e0ddb019b28460393074b074902aaa2
:10165000029300f0e9f800eae07401981df060fae6
:10166000204605b030bd00bf151501024a710c02bd
:10167000f0b500269fb06a4647490546009600f03f
:101680000df9041ec0f282809df8000001a90196a8
:101690001df08cfa041e79db019b23b90a203f4a16
:1016a0003f49eff77dfc0026402200210ea89ef066
:1016b000a8fd04af009b394601980d930496adf840
:1016c00014601df036fc041e60db3846eff75afb51
:1016d00006ab0f93334bcde9067038460e93fff7f8
:1016e00029ff8df84000002853d0019802a90296e6
:1016f0001df021fb041e49db029b019802a91193f6
:101700001df088fa041e41db029b019802a9129386
:101710001df010fe041e39db029b019802a91c93e8
:101720001df03ffe041e31db029b1222314608a849
:101730001d939ef066fd019808a91df026ff041e6a
:1017400024db9df829200df12a01082a28bf082250
:101750000df165008df864209ef02cfd019803a921
:1017600003961df03cff041e10db039b0e4a1493ee
:1017700018930e4b139228460d490daa179300f0ab
:1017800053f800eae07403981df011fe20461fb0e4
:10179000f0bd6ff06304f9e772710c02bff501024e
:1017a0007b900c02c51301022d130102ed130102ff
:1017b0005e710c02002230b587b0054602a90a20ee
:1017c000cde90122f1f78efae0b9029c0cb1236950
:1017d00023b90a200c4a0d49eff7e2fb0c230393cf
:1017e00001ab04930423059301212046236903aa36
:1017f000984738b9019b2846054903aa8df80c3053
:1018000000f012f807b030bdbff50102b77c0c0242
:101810006c6d0c0208b5faf7b9fd002008bd08b5db
:10182000faf7d6fd002008bd2de9f3410024054656
:1018300001a80f469046019420f07af9f0b12246b3
:1018400028460199f2f78eff0446c8b9eff7eafd82
:101850000646f0b1d5e903122346eff7f7fd28b1ac
:1018600042463946304620f02ff908b96ff063043c
:1018700000213046eff7dafd3cb101e06ff0630480
:10188000002228461146f2f76dff204602b0bde85f
:10189000f081014cf4e700bffcfefffff8b5044601
:1018a00000200e461746eff7c7fd054698b1d4e96c
:1018b00001120023eff7e0fd80b13a463146284699
:1018c00020f004fd0028074c18bf00240021284602
:1018d000eff7b6fd00e0044c2046f8bd6ff063045e
:1018e000f4e700bfe8fefffffcfeffff70b5002439
:1018f0008ab005460c2101a8cde9014403940cf0ff
:10190000a3fb0c2826d12146182204a89ef079fcbe
:1019100001ab04a913f8012b0134160906f13000bc
:10192000392888bf06f1570002f00f02087002f153
:101930003000392888bf02f157000c2c01f1020158
:1019400001f8010ce6d12846044904aafff76cff10
:101950000ab070bd6ff06300fae700bf5c6e0c0266
:101960001fb510220021044668469ef04afc002262
:10197000102168460cf0c2fb002804db6a462046b2
:101980000249fff751ff04b010bd00bfca6e0c0240
:101990001fb5074b6a4602930523039302ab0193dd
:1019a000044b05490093fff73fff05b05df804fbca
:1019b000af730c02c5130102f26e0c022de9f04167
:1019c0008eb0074609f036fe002846d00568002d87
:1019d00043d02b6828461b6d98472b6828461b6907
:1019e0009847041e31db1c2200260deb0200314615
:1019f00006969ef006fc2b680df118082022414641
:101a000028461b6b9847041e1fdbadf802602b684d
:101a100028465b6b0df102019847041e15db40461a
:101a2000cde903660596eff7adf901ab04930c4bd6
:101a3000cde901800393bdf802303846094903aa75
:101a40000593fff7f1fe00eae0742b6828465b6d12
:101a5000984720460eb0bde8f0816ff06304f8e7c8
:101a6000c5130102ac6e0c02002307b5044901aa9c
:101a70000193fff7d9fe00eae07003b05df804fbc4
:101a8000de6e0c0210b5044690b04022002168467c
:101a90009ef0b7fb6a4620460449fff7fffe10b9e7
:101aa000684611f0bbfc10b010bd00bf2e6f0c02d9
:101ab00013b5044600208df8040011f0eefc044933
:101ac0008df8040001aa2046fff7aefe02b010bd5b
:101ad000066f0c02002208b511460120f7f7feff41
:101ae000002008bd002208b510461146f7f7f6ffa2
:101af000002008bd002213b5044611461046f5f734
:101b00009afd04498df8040001aa2046fff78cfed7
:101b100002b010bd706e0c02002307b5074901aa80
:101b20008df80430fff7bafe28b99df80430002b79
:101b300008bf6ff0770003b05df804fb426f0c0242
:101b4000012307b5044901aa8df80430fff76cfea4
:101b500003b05df804fb00bf1a6f0c0213b500243c
:101b60000a4901aa8df80440fff798fe00280adb15
:101b70009df804102246012918bf21460420f1f7e0
:101b800031ff00eae07002b010bd00bf746f0c02bc
:101b9000002307b50c4901aaadf80430fff77efe1b
:101ba00000280adb9df80430012b09d106209df89e
:101bb000051009f023f800eae07003b05df804fbbb
:101bc0006ff07700f9e700bf566f0c0237b50025bc
:101bd0006a460f4904468df80050fff75ffe002863
:101be00011db9df800308df80450012b0dd106203b
:101bf00009f02af807498df8040001aa2046fff7ea
